:100000000C94AD430C94F8440C94D3430C94D34318
:100010000C94D3430C94D3430C94D3430C9436598F
:100020000C94D3430C94D3430C94D3430C94D343F8
:100030000C94D3430C94B1540C94D3430C94D343F9
:100040000C94D3430C94D3430C94D3430C94D343D8
:100050000C946F4C0C94D3430C94D3430C94D34323
:100060000C94D3430C94D3430C94D3430C94D343B8
:100070000403090416036F0070007400690078001F
:1000800078002E006F0072006700160351005500C3
:10009000490043004B004400450056003100360043
:1000A00012011001FF000008C016DD050001010269
:1000B00000010902120001010080960904000000FD
:1000C000000000002D2D3E53776974636820544F63
:1000D000204156520A00506F6C6C205553420A0062
:1000E000416374697661746520534E45532062758F
:1000F000730A0044697361626C6520534E45532056
:1001000057520A002D2D3E53776974636820544F6F
:1001100020534E45530A0055534220706F6C6C0AB1
:100120000044697361626C6520534E4553205752F9
:100130000A004163746976617465204156522062F9
:1001400075730A0053797374656D2048773A2025DA
:10015000732053773A2025730A000A0020202020BC
:10016000202020202020202020202020202020208F
:1001700020202020202020202020207777772E6F1D
:1001800070746978782E6F72670A000A0020202048
:1001900020202020205C5F5F3E2020202020202087
:1001A0002020202020205C2F20202020205C2F20B9
:1001B000202020202020205C2F20202020205C2FA9
:1001C000202020202020202020202020202020202F
:1001D000205C2F200A00205C5F5F5F5F5F5C205C1B
:1001E0005F2F5F5F5F5F2F7C5F5F7C5C5F5F5F2087
:1001F000203E5F5F7C5F205C2F5F5F5F5F5F5F5FC4
:1002000020202F5C5F5F5F20203E5C5F2F20207CE2
:100210005F5F5F7C5C5F5F5F5F5F20202F200A0075
:10022000202F2020205C5F2F2E20205C20207C208F
:10023000202F20205C20205C5F5F5F7C202020201E
:100240003C20207C20202020602020205C20205F7B
:100250005F5F2F5C2020202F207C2020205C20202E
:100260007C5F5F5C20205C200A0020202F20202F54
:10027000205C20205C7C20207C20205C20207C2FA7
:10028000205F5F5F5C7C20207C2F202F207C202043
:1002900020207C20205C5F2F205F5F205C20205C82
:1002A0002F202F7C2020202F2020205F5F20205C0B
:1002B000200A00205C5F5F5F5F5F20205C20205F82
:1002C0005F205F5F7C5F5F7C205F5F5F5F207C20E3
:1002D000207C205F5F5C5F5F5F5F5F5F205C202052
:1002E000205F5F5F5F5F5F5F20205F2F5F202020C8
:1002F0007C2F20205F5F5F5F5F2F0A00205F5F5FC2
:100300005F5F5F5F5F20202020202020202E5F5F26
:1003100020202020202020205F5F202020205F5FE1
:100320005F5F5F5F5F5F2020202020202020202053
:1003300020202020205F5F5F5F20205F5F5F5F5F86
:100340005F5F5F0A000A004163746976617465202B
:10035000534E4553206275730A000A0049525120DA
:100360006F66660A00416374697661746520415660
:1003700052206275730A004665746368206C6F6171
:1003800064657220726F6D0A0055534220636F6E70
:100390006E6563740A0055534220646973636F6E1F
:1003A0006E6563740A0055534220696E69740A00D1
:1003B0005553425F4352435F414444523A20616483
:1003C00064723D3078256C782073697A653D256CC0
:1003D000690A005553425F4352435F414444523AD5
:1003E00020616464723D3078256C782073697A6589
:1003F0003D25690A005553425F4156525F524553AD
:1004000045543A0A005553425F4D4F44455F4156AB
:10041000523A0A005553425F4D4F44455F534E4593
:10042000533A0A005553425F4352433A2061646491
:10043000723D30782530386C78200A005553425F81
:1004400042554C4B5F55504C4F41445F454E443AEA
:100450000A005553425F42554C4B5F55504C4F413B
:10046000445F454E443A204552524F5220737461C6
:100470007465206973206E6F74205245515F535428
:10048000415455535F42554C4B5F55504C4F41447E
:100490000A005553425F42554C4B5F55504C4F41FB
:1004A000445F4E4558543A207265715F62616E6BCD
:1004B0003D30782530327820616464723D30782593
:1004C00030386C782074696D653D25690A00555394
:1004D000425F42554C4B5F55504C4F41445F414445
:1004E00044523A207265715F62616E6B3D307825CF
:1004F00030327820616464723D30782530386C7811
:100500002074696D653D25690A005553425F425567
:100510004C4B5F55504C4F41445F494E49543A2033
:1005200062616E6B5F73697A653D30782530386C37
:10053000782062616E6B5F636E743D307825782041
:10054000656E645F616464723D30782530386C7824
:100550000A005553425F42554C4B5F55504C4F413A
:10056000445F494E49543A2025692025690A00759F
:10057000736246756E6374696F6E52656164206C58
:10058000656E3D25692074785F72656D61696E697D
:100590006E673D2569200A0075736246756E637447
:1005A000696F6E5772697465205245515F535441AB
:1005B0005455535F42554C4B5F55504C4F4144206E
:1005C000616464723A2030782530386C78206C652C
:1005D0006E3A2025692072785F72656D61696E6977
:1005E0006E673D25690A004552524F523A75736253
:1005F00046756E6374696F6E5772697465206D6FAE
:1006000072652064617461207468616E2065787021
:1006100065637465642072656D61696E3A20256951
:10062000206C656E3A2025690A007372616D5F6205
:10063000756C6B5F7365743A20616464723D3078E9
:100640002530386C780A0D007372616D5F62756CCD
:100650006B5F7365743A20616464723D3078253055
:10066000386C78206C656E3D256C690A0D007372DC
:10067000616D5F62756C6B5F636F70795F696E74DB
:100680006F5F6275666665723A20616464723D30C0
:10069000782530386C78206473743D30782570206C
:1006A0006C656E3D256C690A0D007372616D5F6249
:1006B000756C6B5F636F70795F66726F6D5F62758B
:1006C000666665723A20616464723D307825303820
:1006D0006C78207372633D30782570206C656E3DB8
:1006E000256C690A0D007372616D5F7772697465BC
:1006F0003A20616464723D30782530386C7820642B
:100700006174613D25780A0D007372616D5F6275D9
:100710006C6B5F77726974655F656E643A007372C3
:10072000616D5F62756C6B5F77726974655F73741E
:100730006172743A20616464723D30782530386C9F
:10074000780A0D007372616D5F726561643A2061B1
:100750006464723D30782530386C780A0D0073720D
:10076000616D5F62756C6B5F726561645F656E641D
:100770003A0A007372616D5F62756C6B5F726561DE
:10078000645F73746172743A20616464723D30789E
:100790002530386C780A0D007372616D5F62756C7C
:1007A0006B5F616464725F726573746F72653A2027
:1007B000616464723D30782530386C780A0D0073BE
:1007C00072616D5F62756C6B5F616464725F7361AF
:1007D00076653A20616464723D30782530386C78F3
:1007E0000A0D000A0030003100737265675F73659F
:1007F000743A20616464723D30782530386C78003A
:100800006372635F636865636B5F62756C6B5F6D7A
:10081000656D6F72793A2062616E6B3D307825307C
:10082000327820616464723D30782530386C7820ED
:100830006372633D3078253034780A006372635FF9
:10084000636865636B5F62756C6B5F6D656D6F721E
:10085000793A2062616E6B3D3078253032782061C4
:100860006464723D30782530386C78206372633D63
:100870003078253034780A006372635F636865639B
:100880006B5F62756C6B5F6D656D6F72793A20623C
:100890006F74746F6D5F616464723D3078253038B9
:1008A0006C7820746F705F616464723D30782530BD
:1008B000386C780A000A002025303278000A25308A
:1008C000386C783A007C0A002E00256300207C00FA
:1008D0002025303278002530386C783A002A0A001A
:1008E0000A446F6E6520616464723D30782530384B
:1008F0006C780A002E004F727068616E6564205239
:100900004C4520636F646520617420737461727458
:100910000A00524C45206465636F6465206C656E07
:100920003D256C6920616464723D30782530386CF7
:10093000780A0000900408C230A9000020120020AC
:10094000D208286008C23129FF000A0AAABFE55769
:100950007F48BFE3577F48A68CE220A9019F932DD3
:100960007EA97F9F9A2D7EC230689F982D7E689FBA
:10097000942D7EA522290F00186A9005186900049D
:100980009F962D7E8A18690800858CA97F00855A5C
:10099000C230A9F3608558A920008500A92000294C
:1009A0001C004A4A0A0A0AAAA00000B7589D72030E
:1009B000C8C8E8E8C600C600D0F1E220E66F2860AB
:1009C0004808E2208BA97E48ABA920291C85D8A91C
:1009D0007F855AC2308A0AAABF5C7E7F8558A000F4
:1009E00000B75829FEFF8D0C02C8C8C23098C9FF55
:1009F00001B05BE220A900EBA5D7F00CA5D73A85A2
:100A0000D7C901D0174C1E01C230B75829F000D009
:100A10000BB758290F00180AAA7C7302E220B758B6
:100A2000AAADD600F035BF39827FEBA92029E305B6
:100A3000D8EBC230AE0C029F721D7E186910009F69
:100A4000B21D7EE220C8E8E88E0C024CBB00E2201A
:100A500064D79CD600E672AB286860BF39817F18E6
:100A60006930EBA920900002090129E305D8EBC207
:100A700030AE0C029F721D7EE220C8E8E88E0C02A8
:100A80004CBB00C230C8B75848C8B7588D59006829
:100A90008D5800A00000E220A90485D7B758484A25
:100AA0009004290F186930C93A90000269068D3206
:100AB0000368290F186930C93A90000269068D331E
:100AC00003A97E855AC230A9320385584CBB00C2A7
:100AD00030C8B75848C8B7588559688558A000002D
:100AE000BBE220A90A85D7C2308A0AAAE220B758F9
:100AF0007CC101D101D201D301D401D501D601D7E6
:100B000001D8014A9007182901693048C2308A4A41
:100B1000AAE220689D3203E8E00800D0C6A97E85DD
:100B20005AC230A9320385584CBB00E220C8B758DE
:100B30001A1A291F85D7C230C8B75848C8B7588D68
:100B40005900688D5800A000004CBB00C230C8B7E7
:100B50005829FEFF8D0C02C8C8A90000E2209CD6CF
:100B6000004CBB00E220ADD60049018DD600C84C38
:100B7000BB00E220C8B7580A0A291C85D8C84CBB5C
:100B8000004C1E01AE0C02E8E88E0C02C860600842
:100B9000C230E220AD1A008920F001E82090000068
:100BA00028601E011E023602FD01080252019D014D
:100BB000440293025302530253025302530253025C
:100BC0005302C230C8B75848C8B7588559688558C5
:100BD000A00000BBE220A90585D7C23164026404ED
:100BE000B75829FF008500F02CE604A500A50429CC
:100BF0000F00C90A00D008A504186906008504A5DD
:100C00000429F000C9A000D008A504186960008577
:100C100004C600D0D4E220A505290F8506D002A97C
:100C2000F01869308D3203A5044A9004290FD006CC
:100C3000C506D002A9F01869308D3303A504290F29
:100C40001869308D3403A97E855AC230A9320385D4
:100C5000584CBB0008C231AD5802F00EC90100D09B
:100C600006A2340020900000CE5802286008E2203E
:100C70008BA97E48ABA5F0D06AA97F85DBC2308AFC
:100C80000AAABFD27F7F85D9A00000B7D9C8C829DA
:100C9000FEFF85E5B7D9C818E2200A85E7B7D9C8AD
:100CA000290F1AAAA900186940CAD0FA85E9B7D94C
:100CB000C8291FD003AB286085EB64EC64EF202CBF
:100CC0000620C305205B06E220A5EC1A85ECC5EBE7
:100CD000D0EC64ECE6F0A90185EF202C0620C305DA
:100CE000205B06E220202C06205B06C231AD6203A9
:100CF000A2FFFFE8E01000F0104A9000F748DA8AFF
:100D0000180AAAFCDD03FA6880EAAB2860FF03FF3B
:100D100003FF03FF03FF03FF03FF03E80453049BE8
:100D20000400042A04FF03FF03FF03FF03FF036023
:100D300008C231E22064EF202C0620C305205B06A8
:100D4000A5EC1AC5EB900002A90085ECA90185EF7E
:100D5000202C0620C305205B06286008C231E22053
:100D600064EF202C0620C305205B06A5EC3A10DAC0
:100D7000A5EB3A85ECA90185EF202C0620C30520C0
:100D80005B0628605A08C231E220202C06A0000031
:100D9000B7DCD003287A60A00000B7DFA00300D73B
:100DA000DC90000488B7DC3AA000001A97DFB7DCBB
:100DB000C901D00CAD6303100718B7DF690F97DFC7
:100DC000A90185EF20C305205B06287A605A08C276
:100DD00031E220202C06A00000B7DCD003287A6086
:100DE000A00000B7DCC901D00CAD6303100738B711
:100DF000DFE90F97DFB7DF3AC9FFF007A00200D79E
:100E0000DCB005A00300B7DCA0000097DFA90185D6
:100E1000EF20C305205B06287A60485ADA080B8B5E
:100E2000C231E220A97E48ABA00700B7DC180AAAAD
:100E3000FC7226AB2B28FA7A686060DA5A08C23155
:100E4000A5E729FF0065ED8D2A03A00400B7DC8D1E
:100E50002F03E220C8C8B7DC8D3103A9058D2E030E
:100E6000A2020020900000287AFA60DA5A08C23103
:100E7000A5E729FF0065ED8D2A03A00400B7DC8DEE
:100E80002F03E220C8C8B7DC8D3103A9068D2E03DD
:100E9000A2020020900000287AFA60DA5A08C231D3
:100EA000A5E729FF0065ED8D2A03A90000E220A037
:100EB0000100B7DC8D2F03A00000B7DF2D2F03C288
:100EC0003129FF000A690C00A8B7DC1865D98D2FFD
:100ED00003E220A5DB8D3103A9048D2E03A20200BD
:100EE00020900000287AFA60080509053805670592
:100EF00008050805080508055ADA08C231A90000E6
:100F0000AA9D2903E8E8E008009000F6A5EC291F57
:100F100000AAA90000E00000F0061865E9CA80F503
:100F20001865E585ED8D2A03A5EF290118690800EC
:100F3000A8E220B7DC8D2D03A9048D2E03EE290332
:100F4000A9078D2C03C231A00A00B7DC65D98D2F0B
:100F500003E220A5DB8D3103A202002090000028CF
:100F6000FA7A605A08C231A5EC291F000A69050007
:100F7000A8B7D965D985DCE220A5DB85DEA006000F
:100F8000B7DC85E1C230A00400B7DC85DFE22028B1
:100F90007A605ADA08C231A0000098E220B7DC2952
:100FA000070AAAFCB30528FA7A6008C231290F00A3
:100FB0000AAABF39827F856BE220A97F856DA000D8
:100FC00000B76B851CC8B76B851DC8B76B851EC87D
:100FD000B76B851FC8B76B853DC8B76B853EC8B773
:100FE0006B8521C8B76B8522C8B76B8523C8B76BE3
:100FF0008524C8B76B8525C8B76B8526C8B76B85B0
:1010000029C8B76B202C12C8B76B8549C8B76B8548
:101010004AC8B76B854BC8B76B854CC8B76B854D55
:10102000C8B76B854EC8B76B854FC8B76B8550C8BE
:10103000B76B8551C8B76B8552C8B76B8553C23142
:10104000A5214829F000EB856568290F00EB180AF7
:1010500090048563A5224829F000EB856968290F73
:1010600000EB180A90048567A52329FC00EB855B3B
:10107000A52429FC00EB855DA52529FC00EB855FF7
:10108000A52629FC00EB8561A5292907000A900502
:10109000EB8527286008E2208502C2318A85040A90
:1010A0006504AABF94867F8504E8BF94867F850582
:1010B000E2207820890720D107582860E220A68CFA
:1010C000A9019F932D7EA5069F9A2D7EC231A00077
:1010D00000B704850765049F982D7E38C8C8B704FB
:1010E000E5079F942D7EA5022903000AA8B9630095
:1010F0009F962D7E8A18690800858C60720572158E
:10110000721D722508E2208BA98148ABA97E2901B6
:101110008D8321C231A5022903000AAABFC9077F16
:101120008D8121E220A502293C8503C231A50585D8
:1011300035A00200B704850765048534C8C8B70424
:1011400038E507850029FEFFAAA00000E220B73499
:101150008D8021C8B73429C305038D8021C8CACA30
:10116000D0ECC231A502290300AAF670E220A97EC4
:101170002901A5028902F005291C0A8005291C0AFB
:101180000A0AC23129FF00AAA5058535A00400B7C7
:1011900004850765048534C8C8B70438E5078500A9
:1011A000A00000E220B7349F72037EC231C8E8C6B7
:1011B00000D0F0E220E66FAB2860DA08C230E2200F
:1011C0009C2121A200019C2221CAD0FA28FA6008A1
:1011D000C231E220A900A00002A2720320602728E9
:1011E0006008C231E220A900A00008A272052060B8
:1011F00027286008C231E220A900A00008A27215C9
:10120000206027286008C231E220A902A00008A2BD
:10121000721D206027286008E22085008BA97E4887
:10122000ABC2317898A48C99962DA50029FF008532
:10123000000A0A186500AABF77867F850099982D55
:10124000E8BF77867F99992DE8E8BF77867F9994E4
:101250002DE220A90199932DC231981869080085C3
:101260008C58AB286008C230E220A51A253AD00C71
:10127000A520290FC90FF006E62028602860286005
:10128000A51A253AD009A520290FF004C6206060D0
:10129000E6196008E220A9808D0021286008E2207C
:1012A000AD104258A520297F8D0021286008C23149
:1012B000A9FF038D2C008D30009C2A009C2E009CE1
:1012C00030009C7E009C80002860EC1A001009A968
:1012D0000300853A204D0960A90300853A203209B0
:1012E00060088BC23148E220A97E48ABC2316885D4
:1012F00000860284042900FFEB85060A186506AA09
:10130000BF97867F8506BF98867F8507A00000B7B8
:10131000061865068509C8C8B7061865068514C885
:10132000C8B706186506850BC8C8B706850DA500A1
:1013300029030085110AAAB563850FA51D29070099
:101340000A0A186511AABF4B867F29FF008511A5DF
:101350000229FF038502A504290080D03AA90000D4
:10136000A602F006186511CAD0FA4A18650F78A6C9
:101370008C9D962DA51438E5099D942DA5099D9861
:101380002DE220A5089D9A2DA9019D932DC2318A99
:1013900018690800858C58A504290020F0034CFA30
:1013A0000AA50B8509A508850BE220A500293C8527
:1013B0000CC231A50D851229FF00850FA91F003829
:1013C000E50F0A850FA5044829FF030A8504A50037
:1013D0002903000AAABF86867F186504AA688504C7
:1013E000A00000C231B70929FF0318650229FF03D5
:1013F000EBE220050CC231EB9F00007EE8E8C8C894
:10140000E220C61210DDA50D8512C2318A18650FC3
:10141000AA9818650FA8E220C61310C7C231A50408
:10142000290010D008A500290300AAF670A50429F8
:101430000040D055A51129FF004A4A4AAABF8F0B88
:101440007F850DA00400B70618650638E51429FF4E
:1014500001A8A5004A4A290700AAF009A900001816
:10146000650DCAD0FA29FF01186972038509A50024
:101470004A9005290600AAFC590BA5078501A51469
:10148000850020E427E66FAB2860610B660B6C0BD0
:10149000710BA900008016A50D4A4A8010A50D4ABF
:1014A000800BA50D4A850F4A18650F8000850F181F
:1014B0006509AAA50F18651485149838E50FA8606A
:1014C0000000080020000002C231A900005BE220F9
:1014D000A98148AB9C0142A532C231A5498D232187
:1014E000A54C8D2621A54E8D2821A5508D2A21A5FC
:1014F000528D2E21E220A54B8D2521A5548D06214C
:10150000E220A61AE8861AA51D8D0521A51E8D2CA0
:1015100021A51F8D2D21A5218D0B21A5228D0C210B
:10152000A5238D0721A5248D0821A5258D0921A599
:10153000268D0A21AD3D008D3021AD3E008D31213B
:10154000AD4100291F09808D3221AD4000291F09BE
:10155000408D3221AD3F00291F09208D3221A52A5F
:101560008D0D21A52B8D0D21A52C8D0E21A52D8D49
:101570000E21A52E8D0F21A52F8D0F21A5308D10A9
:1015800021A5318D1021A5298D0121A5448543F088
:1015900019C231A5458D0942A5478D0742E220A514
:1015A00042093085428D0042800BE220A54229CFBE
:1015B00085428D0042E220A9808D00212008132061
:1015C000C11020EF13E220A520297F8D0021208863
:1015D0002020CC20C231A5D52903000AAAE220FC94
:1015E0000A296008C231A58CD0FC286008C231A548
:1015F0001AC51AF0FA286008C231A900008F8C00C1
:101600007E8F8E007EA00008A2932D206027286088
:10161000010D880FC20F610DB80D570E020D851117
:10162000BC11F3112E115411010D010D010D010D0D
:10163000010D60A901188D0043B79000297F00F0CB
:101640005185F3A910008D0543C8C8B7900085F5F2
:101650008D1621C8C8B7900085F78D0243C8B79092
:1016600000C8C88D0343E220A9808D1521A9018DF2
:101670000B42C6F3F01FC231A5F569100085F58D48
:101680001621A5F71869100085F78D0243A91000EF
:101690008D054380D160A901188D0043A940008DBC
:1016A0000543C8C8B7900085F38D1621C8C8B79008
:1016B0000085F58D0243C8B79000C8C88D0343E28A
:1016C00020A9808D1521A9018D0B42C231A5F36996
:1016D000000185F38D1621A5F51869400085F58D6B
:1016E0000243A940008D0543E220A9018D0B426011
:1016F000A901188D0043A980008D0543C8C8B79083
:101700000085F38D1621C8C8B7900085F58D02437A
:10171000C8B79000C8C88D0343E220A9808D152169
:10172000A9018D0B42C231A5F369000185F38D1625
:1017300021A5F51869800085F58D0243A980008DEB
:101740000543E220A9018D0B42C231A5F3690001D6
:1017500085F38D1621A5F51869800085F58D024366
:10176000A980008D0543E220A9018D0B42C231A55D
:10177000F369000185F38D1621A5F51869800085B0
:10178000F58D0243A980008D0543E220A9018D0B50
:101790004260A901188D0043A900018D0543C8C806
:1017A000B7900085F38D1621C8C8B7900085F58DD8
:1017B0000243C8B79000C8C88D0343E220A9808DBA
:1017C0001521A9018D0B42C231A5F369000185F3F2
:1017D0008D1621A5F51869000185F58D0243A90034
:1017E000018D0543E220A9018D0B42C231A5F369A9
:1017F000000185F38D1621A5F51869000185F58D89
:101800000243A900018D0543E220A9018D0B42C2CC
:1018100031A5F369000185F38D1621A5F51869003E
:101820000185F58D0243A900018D0543E220A90140
:101830008D0B42C231A5F369000185F38D1621A5F8
:10184000F51869000185F58D0243A900018D054356
:10185000E220A9018D0B42C231A5F369000185F395
:101860008D1621A5F51869000185F58D0243A900A3
:10187000018D0543E220A9018D0B42C231A5F36918
:10188000000185F38D1621A5F51869000185F58DF8
:101890000243A900018D0543E220A9018D0B42C23C
:1018A00031A5F369000185F38D1621A5F5186900AE
:1018B0000185F58D0243A900018D0543E220A901B0
:1018C0008D0B42C23160A901188D0043B79000F022
:1018D000288D0543C8C8B790008D1621C8C8B79099
:1018E000008D0243C8B79000C8C88D0343E220A909
:1018F000808D1521A9018D0B42C23160C89007600F
:10190000A901188D0043E220A9818D1521C231C89B
:10191000C8B790008D1621C8C8B79000AAC8C8C81B
:10192000BF00007E8D1821BF40007E8D1821BF8032
:10193000007E8D1821BFC0007E8D1821BF00017E62
:101940008D1821BF40017E8D1821BF80017E8D182A
:1019500021BFC0017E8D1821BF00027E8D1821BFDE
:1019600040027E8D1821BF80027E8D1821BFC002EB
:101970007E8D1821BF00037E8D1821BF40037E8D10
:101980001821BF80037E8D1821BFC0037E8D1821D2
:10199000BF00047E8D1821BF40047E8D1821BF80BA
:1019A000047E8D1821BFC0047E8D1821BF00057EE6
:1019B0008D1821BF40057E8D1821BF80057E8D18B2
:1019C00021BFC0057E8D1821BF00067E8D1821BF66
:1019D00040067E8D1821BF80067E8D1821BFC0066F
:1019E0007E8D1821BF00077E8D1821BF40077E8D98
:1019F0001821BF80077E8D1821BFC0077E8D18215A
:101A00006008E220A97E8592C231A9932D859000BD
:101A1000A48CF059A48EB790005A290F000AAAC8C6
:101A200008FCDF0C287AA90000979000C8C897909E
:101A300000C8C8979000C8C8979000C8C898858EFD
:101A4000C58C900006648E648C8028E220A9808D6D
:101A50000142EA9004AD3721AD3F21AD3D21EBAD10
:101A60003D21EBC23129FF01C9C700900005C9041F
:101A7000019000A72860E2209C2121A272038E021F
:101A800043A200028E0543A97E8D0443A9008D0068
:101A900043A9228D0143A9018D0B4260E2209C02E3
:101AA000219C0321A2732B8E0243A220028E0543A8
:101AB000A97E8D0443A9008D0043A9048D0143A98B
:101AC000018D0B42600008001000100020C231A5FB
:101AD000232903000AAABF7D117F8D0543E220A6BA
:101AE0005B8E1621A272058E0243A97E8D0443A946
:101AF000808D1521A9018D0043A9188D0143A901ED
:101B00008D0B4260C231A5242903000AAABF7D11B2
:101B10007F8D0543E220A65D8E1621A272158E02EE
:101B200043A97E8D0443A9808D1521A9018D004311
:101B3000A9188D0143A9018D0B4260C231A5252949
:101B400003000AAABF7D117F8D0543E220A65F8EA8
:101B50001621A2721D8E0243A97E8D0443A9808D99
:101B60001521A9018D0043A9188D0143A9018D0BF1
:101B70004264726008E22085438544C2312907002F
:101B80000A85F30A1865F3AABF7E127F8545BF80D8
:101B9000127F85472860C23948DA5A0B8BA90000AA
:101BA0005BE220A98148ABC231A5432907000A8521
:101BB000F30A1865F3AAFC7C12C239AD1142AB2BB3
:101BC0007AFA6840AC12C8008200C112C8008200D4
:101BD000D6128F00820007130090040713009004B0
:101BE000071300900407130090040713009004EA01
:101BF0009008E220A92F8D3221C231EE8E0260EAD8
:101C00009008E220A98F8D3221C231EE8C0260E271
:101C100020A940C6439C0F219C0F219C10219C10A1
:101C200021A521290F09708D0B21A52529FC8D08DF
:101C300021C231A9C8008D0942A982008D074260E6
:101C400060A56FF0259C2121A272038E0243A200A1
:101C5000028E0543A97E8D0443A9008D0043A9226D
:101C60008D0143A9018D0B42646FA56EF0289C0283
:101C7000219C0321A2732B8E0243A220028E0543D6
:101C8000A97E8D0443A9008D0043A9048D0143A9B9
:101C9000018D0B42646EA570F038C231A523290373
:101CA000000AAABF7D117F8D0543E220A65B8E1638
:101CB00021A272058E0243A97E8D0443A9808D1551
:101CC00021A9018D0043A9188D0143A9018D0B4263
:101CD0006470A571F038C231A5242903000AAABF97
:101CE0007D117F8D0543E220A65D8E1621A272151F
:101CF0008E0243A97E8D0443A9808D1521A9018DF3
:101D00000043A9188D0143A9018D0B426471A5728E
:101D1000F015A68CA9099F932D7EC2318A186908F7
:101D200000858CE220647260E220AD6D02300E4AC4
:101D300090000CA520C90FF010A5201A852060A5E1
:101D400020F006A5203A852060AD6D0209808D6DDA
:101D5000026008E220AD6D0210FB2860C231DAA6F5
:101D600099BD953D29FF000AAA080BFC6F202B287E
:101D7000FA6008C231BD9F3D29FF000ADAAABF51AF
:101D8000717FFA186951718534E220A97F8536C2C6
:101D900031BD9E3D29FF000AA8DAB73485A1482944
:101DA0001F000AAA685A080BE220A900EBFC821463
:101DB0002B287AFAE220A5A130B92860CA14FF14B2
:101DC000051547156A157615F9147F158A15A4159A
:101DD000BC155E15C515A914A814D315E115FB157E
:101DE000D31460A6998D0000AD0000F013BDA73D8F
:101DF000D007AD00009DA73D603A9DA73DF0016072
:101E0000FE9E3D60A699FE9E3D20FF1860C231A84F
:101E1000A699BD9A3D69800048BD9C3D1869800027
:101E200048FE9E3D9820FF18A699689D9C3D689DA0
:101E30009A3D60A6999D9E3D60A6999D933D60A6A2
:101E400099FE9E3D4829F0184A90048908F005291A
:101E50000749FF1AC2310A90047D9A3D9D9A3DE2DE
:101E60002068290F8908F005290749FF1AC231297E
:101E7000FF000A90047D9C3D9D9C3DE22060A69958
:101E8000FE9E3D187D973D9D973DBD933D8940F059
:101E900003209B1960A6999D963DFE9E3D209B19AF
:101EA00060A699FE9E3D9D973D209B1960A699FED8
:101EB0009E3D9D993D60A6999D9F3D9E9E3D640AD5
:101EC00060A699FE9E3D2901180A90058500BD93E4
:101ED0003D29DF05009D933D60A699FE9E3D2901A9
:101EE000180A0A0A8500BD933D29F705009D933D18
:101EF00060A699FE9E3D9D953D60C231A699FE9ECD
:101F00003D29FF0020072460A699FE9E3DBD933D1C
:101F100029EF9D933D60A699FE9E3D9DAA3D293FD8
:101F2000C93FD003DEAA3DBDA93D297F9DA93D60E3
:101F3000A699FE9E3D9DAC3D293F8500BDAB3D2948
:101F40003F8501C500F028B00BA50038E501C92088
:101F5000B014800738E500C92090000BBDAB3D29C7
:101F60003F09409DAB3D60BDAB3D293F9DAB3D6012
:101F7000BDAB3D09809DAB3D60BF923D7E300D8A7B
:101F800018692000AAE0E007D0EF38608699186051
:101F900008E2208BA97E48ABA56ED01AC2319CB551
:101FA0000020011D20EF1CA2000020431690000A13
:101FB00020881A6499E66EAB2860BD933D892000A5
:101FC000D062BD9A3D4A90048D0002BD9C3D4A906E
:101FD000048D0202BDA43D29FF0049FFFF186D00DA
:101FE0000218692000C57E900047BDA43D29FF006E
:101FF00018657E1869E800CD0002900035BDA53D4A
:1020000029FF0049FFFF186D020218692000C580F2
:10201000900020BDA53D29FF001865801869E000EB
:10202000CD020290000E20D11BBD933D0940009DC2
:10203000933D8009BD933D29BF009D933DBD933DD8
:10204000DA891000F003203814FA8699DABD933D3E
:10205000890800F003202214FA8699DABD933D899D
:102060000400F003204917FA8699BD943D891000B9
:10207000F0032016208A18692000AA86994C74164D
:102080002860089BA6B5E220B9A83D0980EBB9A05D
:102090003DC2319F13467EB99A3D4A9004E8E89FBD
:1020A00013467EB99C3D4A9004E8E89F13467EE8BB
:1020B000E886B5BB286008C23186A884AA29FF003B
:1020C0000AAA0BA900005BE2208BA97E48ABC231B3
:1020D000BFC8847F1869C8848534E220A97F85360B
:1020E000A20000BD933D1010C2318A692000AAE20F
:1020F00020E0E007F00280EBC23186998A184A900E
:1021000004E220859BC231A00000B7349D933DE8D6
:10211000E8C8C8C02000D0F2A699BD933D89200030
:10212000F054BD933D102CA5A829FF00180A900774
:102130009D9A3DA5A82900FFEB180A90079D9C3D9C
:10214000A5AAE2209DA63DC2318044A5A829FF0092
:10215000180A90079D9A3DA5A8EB29FF00180A9040
:10216000079D9C3D802118A5A829FF000A90079D86
:102170009A3D18A5A82900FFEB0A90079D9C3DA950
:102180000000A8E220A59B9DA03D209B19209C1843
:10219000A699DABD933D8910F003203814BD943D13
:1021A0008910F003205720FA8699E220BD933D89DB
:1021B00008F003202214AB2B2860BD943D8920D069
:1021C0005BC231BD993D8500BDA13D29FF000A0AD2
:1021D000AABF27867F186927868534BF29867F296D
:1021E000FE00C92000B003A920008501A90000E27B
:1021F00020A97F8536C231A500290E00184A18692A
:1022000008000A9005AAA00000B7349D7203E8E810
:10221000C8C8C401D0F3E220E66F6008C23129FFCC
:102220000085000AAA0BA900005BE2208BA97E486A
:10223000ABC231BFC8847F1869C8848534E220A945
:102240007F8536A20000BD933D1010C2318A6920FF
:1022500000AAE220E0E007F00280EBC23186998A12
:10226000184A9004E220859BC231A00000B7349D3B
:10227000933DE8E8C8C8C02000D0F2A699A90000A4
:10228000A8E220A59B9DA03D209B19209C18A69903
:10229000BD933D8910F003203814BD943D8910F0A2
:1022A00003205720E220BD933D8908F0032022142B
:1022B000C230AB2B286008E220BD943D8940F0027B
:1022C0002860C231BD933D290200180A0A8500A585
:1022D0002929E000184A9005050085000A186500C4
:1022E000DAAABFCC857F8508BFCE857F850EFA1818
:1022F000A50829FF001A4A90058500A50929FF00B5
:102300008502A90000A8C402F005C8650080F78511
:1023100000BD973D29FF008502A90000A8C402F076
:1023200005C8650080F78502BD963D29FF0085043C
:102330000A1865049BAABF24867F8504BF25867F73
:10234000BB8505A502180A9005186504900002E6F1
:10235000068504E220BD993D2901EBBD983DC231BF
:102360000A9004186527850ADAA68CA50829FF00BB
:102370001A850CC231A50E9F932D7EA50A9F962D1E
:102380007EA5049F982D7EA5059F992D7EA50C9F67
:10239000942D7E8A18690800858CFA286008C2315D
:1023A000E220A20000A5A0D0022860850285036477
:1023B000009BB97725100FB97825C50090000885D6
:1023C00000C231989D732AC23198690600A8E220A4
:1023D000C602D0DFA5A0850264005ABD732AA8B941
:1023E0007725297F9977257AE8E8A00000C603D0F1
:1023F000C26402A69CC231A50229FF00A8B9732AB3
:10240000A8B973259D732BB975259D752BDA5A8A4A
:1024100029F0014A900485008A18290C004AAAB9BB
:102420007725A4002903007C151B231B211B1F1BE0
:102430001D1B0A900619732D99732D7AFAA90000B5
:10244000E89004E220A5021A1A85024AC5A0D0A08D
:10245000869C286085000A0A186500A8B97325F0D3
:102460000F9838E90600900003A880F1A0EC0480E2
:10247000EC60E220BDA63DF04FA49EBD943D30210E
:10248000BDA63D997825C231BD9A3D4A9004997305
:1024900025BD9C3D4A9004E2209974254C3B1CBD0F
:1024A000A63D49FF997825C231BD9A3D4A9004E284
:1024B00020997325C231BD9C3D4A9004E220997455
:1024C000254C3B1CC231BD9A3D4A900499732BBDEB
:1024D0009C3D4A9004E22099742B4C911CA49CBD15
:1024E000933D892000D085BDA63D29FF00F073A44F
:1024F0009EBD9C3D4A90048500BDA63D29FF001865
:10250000650038E580E220997825C231BD9A3D4AC0
:10251000900438FDA43D38E57E997325B00BBD933A
:102520003D0901009D933D8009BD933D29FEFF9D1E
:10253000933DBD9C3D4A900438E58038FDA53DE2C1
:1025400020997425BD933D29030980997725E6A03C
:10255000C231BD983D99752598690600859E60BD7C
:102560009A3D4A90041838FDA43D38E57E99732BB6
:10257000B00BBD933D0901009D933D8009BD933D86
:1025800029FEFF9D933DBD9C3D4A900438E580386F
:10259000FDA53DE22099742BC231DA5A9829F00149
:1025A0004A900485009818290C004AA8BD933DBBA9
:1025B000A4002903007CB21CC01CBE1CBC1CBA1C9D
:1025C0000A900619732D99732D7AFAC231BD983D80
:1025D00099752BC89004849C6008201C1D20EF1C5A
:1025E000205A1DE2209C8602646EA90120FF182853
:1025F0006008C231E220A900A02000A2732D206053
:1026000027286008C231E220A903A49CF006A27327
:102610002B206027C231649C649E64A0286008C29D
:1026200031E220A903A00002A2732B206027C2314F
:10263000649C649E64A0286008C231E220A900A0C6
:10264000C000A21346206027286008C231E220A9FA
:1026500000A00006A27325206027286008C231E28E
:1026600020A900A00008A2933D206027286008C28E
:10267000318500A20000BFA23D7EC500D007A900A1
:10268000009F933D7E8A18692000AAE00008D0E6EA
:10269000286008C2318500A20000BFA23D7EC500AF
:1026A000D0032818608A18692000AAE00008D0EA40
:1026B00028386008C231850080E008C231E220A6D7
:1026C00099BDA93D3045293F8500BDAA3D48293F18
:1026D0008501682A2A2A0AC231290600DAAAE220DC
:1026E000FC451FFA8502A501C500B00DA50038E51F
:1026F00002C501300DB0118009A500186502C501A1
:10270000900006A501293F09809DA93DC231A699E7
:10271000BDAA3D30490A0A2900FC8500BDAD3D0A2D
:102720000A29E00305008500BDAC3D48EB0A0A29F3
:1027300000FC8502684A9005290600DAAAFC711F90
:10274000FA8504BDAB3D894000D01FA500C502B08D
:102750000E38E504B03CC50290002C80364CAE1E0D
:1027600038E504900022C50290001E8028A500C50F
:102770000290000B18650490001DC502B00D801773
:10278000186504B006C502B002800CA5022900FC41
:102790004A4A090080800529E0FF4A4A8500E22074
:1027A000BDAB3D294005019DAB3DBDAD3D290705B4
:1027B000009DAD3DC231BD943D290F008500BDADEA
:1027C0003D2907008502BDA93D293F0048BDAB3D1D
:1027D000293F000A9005650018695169AAA02003E5
:1027E00068186502482907008502684A4A4A29078D
:1027F0000048F0323A547EC0A96B00990000A699B7
:10280000BD9C3D4A9004A8BD9A3D4A9004DAAA2294
:1028100020037E8AFA0A90049D9A3D980A90049DAE
:102820009C3D68186500290F008500E220A699BD2F
:10283000943D29F005009D943DBDAD3D29F805026C
:102840009DAD3D28604D1F501F531F561FA940606E
:10285000A90160A90860A50138E500900002800583
:10286000A50038E5014AD003A90160C9089000021B
:10287000A90860791F7D1F811F851FA900FC60A921
:10288000200060A9000460A50238E50090000280E5
:1028900005A50038E5024AC92000B004A92000605F
:1028A000C90004900003A900046008C231DAE220E4
:1028B00048A5B4290385AE6829031865AEF058858C
:1028C000AEC231BD9C3D4A900729FF00EB8500BD9B
:1028D000A43D29FF008502BD9A3D4A900438E90ACB
:1028E000004A4A4A1A29FF000500AAA93600207F9B
:1028F00017E220FABD993D290E8500DAA699BD9907
:102900003D29F105009D993D208820208820C6AEF4
:10291000D0AAFA2860BDAD3D29FF00F032DEAD3D02
:10292000BDA93D29FF00186980FF187D9A3D9D9A39
:102930003DBDAC3D29FF00187DAA3D9DAA3D187DF7
:102940009C3D9D9C3D4A9004CD8402B00160CE86A2
:10295000029E933D6008E220AD8602CD8702900082
:10296000089E933D9E943D2860EE86022860872055
:102970007320E220A699AD11020A90049D9C3DA906
:10298000FF9D9A3D606008E220A5B385B4A5B2859D
:10299000B3A5B185B2C5B33024A5B31865B4184D3D
:1029A00042034D44034D46034D48034D4A034D4CED
:1029B000034D4E034D5003451A85B128601865B488
:1029C000184D4A03451A85B1286008E220AD41211F
:1029D00029E0C9E0D011C231AD41212907000AAA7E
:1029E000AD42219F5B5F7EC231A5C5291F000AAAA7
:1029F000FC1021E220286008E2209C120220C7235C
:102A0000A5C9C5CAD0FAA5C5C901D0F428606C22F1
:102A10000323392345238D219921A824E824392231
:102A20005E2219222B2270217F2153216221342121
:102A30004521C231A5C68D4121E220A9FE8D40214C
:102A4000E6C560E220AD4021C9FED004A90185C5DC
:102A500060E220A5C68D4121A9FD8D4021E6C5601B
:102A6000E220AD4021C9FDD004A90185C560E22066
:102A7000A5C68D4121A9FC8D4021E6C560E220ADAF
:102A80004021C9FCD004A90185C560E220A9F88DC8
:102A90004021A90585C560E220AD4021C9F8D0706C
:102AA000A5C685CFC23129FF0085CB0A1865CBAA00
:102AB000BF91867F85CBBF92867F85CCA00000B773
:102AC000CB3A3A8DD100C8C8E220B7CB8D4121C89E
:102AD000B7CB8D4221C8B7CB8D4321C8A9F28D4019
:102AE00021CD4021D0FBB7CB8D4121C8B7CB8D4242
:102AF00021C8B7CB8D4321C8A9F38D4021CD4021FA
:102B0000D0FBCCD1009000C3A9F98D4021A901854B
:102B1000C5A5D3094085D360C2319C41219C422187
:102B2000E220A9FB8D4021E6C560E220AD4021C92D
:102B3000FBD004A90185C560C231A5C68D4121A580
:102B4000C729FF7F0D71028D4221AD7102490080BE
:102B50008D7102E220A9FA8D4021E6C560E220AD28
:102B60004021C9FAD004A90185C560E220A97FA24D
:102B7000522B85CD86CBC231A00000A9AABBCD4087
:102B800021D0FBE220A9CC8026B7CBC8EBA90080DE
:102B90000BEBB7CBC8EBCD4021D0FB1AC2208D4048
:102BA00021E220CAD0EBCD4021D0FB6903F0FC48E4
:102BB000C220B7CBC8C8AAB7CBC8C88D4221E22073
:102BC000E00100A9002A8D4121697F688D4021E044
:102BD0000100900007CD4021D0FB70AEE220A5425D
:102BE000E6C5A9A08D1502A90F8D160220F022605E
:102BF00008C231A90000A210009F595F7ECACAD046
:102C0000F82860E2209C4021A5C9C5CAF02AC2313B
:102C1000293F00AABD180285C5BD1A0285C7A5C5F2
:102C2000291F00C90100F0100AAAFC1021E220A50A
:102C3000C9186904293F85C960E220A9F18D4021A6
:102C4000A90385C560E220AD4021C9F1D072A5C6B7
:102C500085CEC23129FF0085CB0A1865CBAABF8E6D
:102C6000867F85CBBF8F867F85CCA00000B7CB3A0F
:102C70003A8DD100C8C8E220B7CB8D4121C8B7CB6F
:102C80008D4221C8B7CB8D4321C8A9F28D4021CDFB
:102C90004021D0FBB7CB8D4121C8B7CB8D4221C895
:102CA000B7CB8D4321C8A9F38D4021CD4021D0FB66
:102CB000CCD1009000C3A9F48D4021A90185C5A500
:102CC00042A5D3098085D36008C231A5CA29FF0077
:102CD000AAE220A90A9D1802A5CA186904293F85FD
:102CE000CA286008C23148DAA5CA29FF00AA689D2F
:102CF0001A0268E2209D1902A9089D1802A5CA18A7
:102D00006904293F85CA286008C231DA48A5CA2962
:102D1000FF00AAA900009D1A0268E2209D1902A9DD
:102D2000089D1802A5CA186904293F85CAFA2860B7
:102D300008C23148A5CA29FF00AA68E2209D1902ED
:102D4000A9029D1802A5CA186904293F85CA9C12C8
:102D500002A5D3297F85D3286008E22048C2319C90
:102D60006F02A5CA29FF00AAE220689D1902A906E0
:102D70009D1802A5CA186904293F85CAE2209C1241
:102D800002286008C23148A5CA29FF00AA68E220CB
:102D90009D1902A9049D1802A5CA186904293F8536
:102DA000CAA5D329BF85D32860E220A97F8D12024E
:102DB000A5C685C4C23129FF0085BC0A0A1865BCB6
:102DC000AABF9D867F8D4121E220A9F58D4021AFCC
:102DD000402100C9F6F004A90785C560E220A532AC
:102DE000297F8532A90185C560E220AD4021C9F661
:102DF000F0EAC9F5D0F2A5C4C23129FF0085BC0AAA
:102E00000A1865BCAABF9A867F85BEBF9B867F8550
:102E1000BFAD412185C18D6F0248AD120229FF006F
:102E2000D0039C6F0268C9C70190000CE220E6C085
:102E3000C23138E9C70180EF0A900485BE0A0A0A48
:102E40001865BE85BEA9120085BCA90500A20000B8
:102E50009B9F535E7EA9F7009F545E7EA5C19F5540
:102E60005E7EAD12029F575E7EE89005A901009F2D
:102E7000535E7EB7BE9F545E7EC8C8B7BE9F565E87
:102E80007EE89005C8C8A901009F535E7EB7BE9F2B
:102E9000545E7EC8C8B7BE9F565E7EE89005C8C81F
:102EA000C6BCD0C464BC64BEA901009F535E7EA5AD
:102EB000BC9F545E7EA5BE9F565E7EE89005A9002D
:102EC000009F535E7EA9535E8F724300E220A532BD
:102ED00009808532A97E8F744300A9048F70430056
:102EE000A9408F7143006008C231A5CA29FF00AA1A
:102EF000E220AD15029D1902A90C9D1802A5CA1861
:102F00006904293F85CA286008C231A5CA29FF0083
:102F1000AAE220AD16029D1902A90E9D1802A5CAAB
:102F2000186904293F85CA286008C231A5CA29FF4B
:102F300000AAE220AD170229079D1902A9109D18C9
:102F400002A5CA186904293F85CA28606008C231F1
:102F500048A699BD9A3D4A9005297F00090F00EBCC
:102F6000AA68E22020E22328602027D226D626362F
:102F700027DB26FE2604270C27C723EE250F263045
:102F8000269A2621272827E526EC26F326522759BC
:102F900027E2204B688502C23164009C900002A0A9
:102FA0000000C231B70029FF006D9000028D900033
:102FB00002C8D0F0A0DEFFB700CD900002F007A25B
:102FC00011002090000060A2100020900000605CC2
:102FD000DA267F5CDA267F60E220AD8B028F00303C
:102FE0000060E220A90285FB60E220A90485FB6065
:102FF000E22064FB60A5C420582460A5CE202F24C5
:1030000060E220A5CF20822460E220AD1302EBAD68
:103010001402C231AAE220A5D020E2236060E2209F
:10302000A900851960E220A90A851960E220A90893
:10303000851960E220A902851960E220A90485199A
:1030400060E220A902851960E220A91C851960E2CE
:1030500020A925851960E220A924851960088BE242
:103060002048A98048AB68C2312907000A69962721
:103070008500E220A97F8502C2319829FEFFA85A67
:10308000A00000B7007A9F00007EE8E88888D0F6AC
:10309000AB28600000EAEA8024C900072948DA0862
:1030A000C230E220A9808D00219C00428D1521A212
:1030B00009188E1043A200008E162186008E12433E
:1030C000A9008D1443A2FFFF8E1543A9028D0B4268
:1030D0009C1921A5208D0021A5428D004228FA6867
:1030E00060088BE22048A98048AB68C2316403E2E3
:1030F000205AA403B700C884037A9F00007EE888A2
:10310000D0EFAB2860088BE22048A98048AB68C2AA
:10311000319C15439C12439C8121E220A9C08D144F
:1031200043A9018D8321A202808E1043A9028D0B39
:10313000425C38287FAB28604328AC28D328E82895
:10314000C231A9C8008D8402E220A9008520A9808F
:103150008F00210020D71C207A0920C60C20361DA4
:1031600020481D20D20820C00820AE08E670E67175
:10317000E67264A3A90085D5A9808D6D02A9148D7E
:103180008702A90020730620040020D208A900208D
:103190002F2464F0A90F8520E619C231A92400A2CA
:1031A0000000A0000020AE0960205A16A2000020F6
:1031B0003E03E220A51A2903D015A2130020900097
:1031C00000A2140020900000A21500209000002012
:1031D000D82960E22020D20820C00820AE08A2032F
:1031E000002090000064F0E619205A16A201002089
:1031F0003E03A20D0020900000A20E0020900000CF
:10320000A21E0020900000A21F002090000060B4C9
:103210002913291229122960AD12428901D0F9C25D
:1032200031AD18428D4203AD1C428D4403AD1A42AC
:103230008D4A03AD1E428D4C03E220A9C08D014290
:10324000A9018D16409C1640C231A21000AD164057
:103250004A2E46034A2E48030A0AEB4A2E4E034AD8
:103260002E5003CAD0E7E220A9018D1640EAEAAD4C
:103270001640AD16402902D0069C46039C4703AD7C
:103280001740AD17402902D0069C4E039C4F039C6B
:103290001640C231A20000BD520349FFFF9D6203E8
:1032A000BD42039D52033D62039D6203E8E8E010C6
:1032B00000D0E4E2209C014260AD12428901D0F9C5
:1032C000C230AD520349FFFF8D6203AD18428D42FB
:1032D000038D52032D62038D6203E2206008C23128
:1032E000AF0100C08500AF0000C0CF000040D0207B
:1032F000E220C9A5D01AA50089F8D014A9A58F008D
:1033000000C0C231A500482907000AAA68FC0D2A9E
:1033100028601E2A252A1D2A1D2A1D2A1D2A1D2A2B
:103320001D2A60E220EB8D920260E220EB8F0242C8
:1033300000A9648F034200EA9004C231AF16420034
:103340008F044200E220AD92028F064200EA90080C
:10335000C231AF1442008D9302A2180020900000E9
:1033600060A217002090000060E220A9808D00215B
:10337000200828C231A900005BA9FF011BE220A997
:1033800000A0F001A20000206027A900A00060A218
:103390000002206027A201217400E8E00D21D0F88E
:1033A00074007400E8E01521D0F6A9808D15219CE9
:1033B00016219C17219C1A21A21B2174007400E87D
:1033C000E02121D0F6A223217400E8E03421D0F8D6
:1033D000A9FF8D0142EAEAAD1042AD1142208708F3
:1033E000209C0820AE0820C00820C60C20D71C2036
:1033F000361D20481DC231A9341285B1A9AA5585B0
:10340000B2E220A9018D42008D0042AD1C008D3337
:1034100021206A09AD104230FBAD104210FB20970D
:103420000BA5190AC23129FF00AAE220AD1C008FAA
:1034300033210008FC3B2828A9808F014200EA9034
:1034400004AF372100AF3F2100AF3D21008D1102B5
:1034500080C161190003208FF0F1E8FFC5F0FFCDB6
:10346000FFBDE8005D5F24036D6174744064666FA6
:10347000726365333030302E6465AFC8F0D0FB8F97
:103480007F9C8F7F9D8F009E8F009F8F0FA08F0F3F
:10349000A18F00B28F7FB88F7FB98F5F838F1C841D
:1034A0003FB7133F550C3F020C3F0B13E4FDE4FD07
:1034B000F0FC3FFD033F4314E4F428F068F0D0EC47
:1034C000E4F4280F1C5D1F7303F1139303F113F150
:1034D00013F1139211F113F1139E0FF11347101F03
:1034E000140614F4132E1437143F170F3FB7133F6D
:1034F0000B0D3F550C3F020C3F0B132FAF3FC51276
:103500002FAA8D00CBF4CBF5CBF6CBF7E86C8DE092
:10351000DAF2E80CDAF2E81CDAF2E82CDAF2E83C4B
:10352000DAF2E84CDAF28DFFE85CDAF28D00E80DB1
:10353000DAF2E82DDAF2E83DDAF2E84DDAF2E85DA7
:10354000DAF2E86DDAF2E87DDAF28FF0F15FC0FFCF
:103550005FC0FF03EF016FAB60698F60D01A8F000F
:1035600060EB9000E85CDAF2E4FE8D02E4FEF0FC31
:10357000FEFA3F57043F210E6FBAA4DA6A8F007833
:103580003F2406BAA6DA6A8F10783F2406BAA8DA72
:103590006A8F20783F2406BAAADA6A8F30783F24EF
:1035A00006E4B7F0088F4CF2C4F38F00B76FBA622D
:1035B000DA963AB38F0077BAA4DA6A8F00783FAF11
:1035C000043FCB0DBAA6DA6A8F10783FAF043FCB29
:1035D0000DBAA8DA6A8F20783FAF043FCB0DBAAAA4
:1035E000DA6A8F30783FAF043FCB0D3F8B0D3F9EA3
:1035F0000E5F3C133A628D00E8FFD76AFCD76AFC85
:10360000D76AFCD76A6F8D00F76AC46CFCF76AC48E
:103610006DFCF76AC470FCF76AC471096D6C0970BF
:103620006C09716CE46CD0033F0E068D00F7626884
:10363000FFF0C1D76AFCF762D76AFCF762D76AFC71
:10364000F762D76A3A623A623A623A628D02F76A80
:10365000280FC46C8D03F76A28F0046C68DEF00351
:103660003F0D056F8D00F76AF01A9C8D08CF7A87A1
:10367000DA6C8D02F76C8D04D76A8D03F76CC47910
:103680008D05D76A8D01F76A68FFF0338D02F76AFE
:1036900068FFF02E280FC46CFCF76A28F0046C9FBA
:1036A00068E5F0108D02F76A280F6803F00B6805D3
:1036B000F0072F0E3FD70B2F093F4A085F82065FA6
:1036C00082068D01F76A8D11D76AFD6D8D04F76A48
:1036D0008D48CF7A81DA7FEEF77FC46CC48CFCF71B
:1036E0007FC46DC48DEB6DE46C7A6C7AA2DA6C8D5C
:1036F00000F76CC47AFCF76CC47B8D06E47AD76A59
:10370000FCE47BD76A8D13E48CD76AFCE48DD76A1E
:103710008D0EF76A6804D0068D0DE800D76A8D0E0D
:10372000F76A6840D0068D0FE800D76AE47808028F
:103730005D8D06F76AD8F2C4F3FC3DF76AD8F2C48F
:10374000F33D8D00F76AF01AD8F2C4F33DD8F28F3A
:1037500000F33DD8F28F00F33D3D8D17F76A0477F3
:10376000C4775F8206E47808025D8D06F76AD8F2B6
:10377000C4F33DFCF76AD8F2C4F36F8D02F76A68B0
:10378000FFF0E2280F1C5D1F3306E2067F07EC07FF
:103790009A084009FB060107150A53065306EB0A6F
:1037A000530653065306540653066F8D03F76A28D3
:1037B000F05C5C5C5D1F6106810681068106810606
:1037C00081068106810681068106E60E8106810654
:1037D000BD0EE60E810681066F8D02F76A68FFF066
:1037E00027280F1C5D1F91060E060E060E060E06FC
:1037F0000E060E060E060E060E06320B0E06890B80
:10380000A90BB70BB406240B5F0E068D03F76A28CD
:10381000F0FD9F1C5D1FC106C10B7707E407E106A1
:10382000C40BD70B730EE106E106AF0EE20BF20BF1
:10383000AF0EAF0EE106E1066F8D04F76A8D48CF3B
:103840007A81DA7F8D06F76AC47AFCF76AC47B5FF7
:1038500007073FAA085FEB0A3F70095FEB0AE460C5
:103860008D00CD039ECB6C78016CF00B78026CF070
:103870000F78006CF0126F8D03F76A9F280F2F15D9
:103880008D03F76A280F2F0D8D06F76AC46CFCF7BD
:103890006AC46D2F291CC46C8D11F76A60846CFD9D
:1038A000F77FC489FCF77FC48AEB8AE4897A897A36
:1038B000A2DA898D00F789C46CFCF789C46DE478BD
:1038C0000802C4F2FA6CF3BCC4F2FA6DF36F78002C
:1038D00060D0648F0F7DE8718D00DA708D13F76A08
:1038E000C46CFCF76AC46D8D03F76A247D8D00DA21
:1038F0006EBA6C9A6E5A701002BA70DA6C8D13E45C
:103900006CD76AFCE46DD76AEB6DE46C7A6C7AA2D2
:10391000DA6E8D00F76EC46CFCF76EC46D8D06E434
:103920006CD76AFCE46DD76AE4780802C4F2FA6CDA
:10393000F3BCC4F2FA6DF38FFF7D6F780060D0F7AF
:103940008F0F7DE8588D03DA708D13F76AC46CFC15
:10395000F76AC46D8D03F76A247D8D007A6C5A7006
:103960003002BA70DA6C8D13E46CD76AFCE46DD760
:103970006AEB6DE46C7A6C7AA2DA6E8D00F76EC435
:103980006CFCF76EC46D8D06E46CD76AFCE46DD7F1
:103990006AE4780802C4F2FA6CF3BCC4F2FA6DF37C
:1039A0006F8D01F76AFD6D8D04F76A8D48CF7A81BE
:1039B000DA7FEEF77FC48CFCF77FC48D8D15E48C25
:1039C000D76AFCE48DD76A8D13F76AC46CFCF76A7A
:1039D000C46D8D0BE800D76ABA8C5A6CF0093006BA
:1039E0008D0BE801D76A6F8D15E800D76AFCD76A9E
:1039F0006F8D03F76AF00A8D0AD76A8D03E800D746
:103A00006A8D15F76AC46CFCF76AC46DBA6CF0D69F
:103A10008D0AF76A8D00DA6E8D0BF76AD0208D1350
:103A2000F76AC470FCF76AC471BA709A6E5A6C1067
:103A30002B8D15E800D76AFCD76ABA6C2F1E8D1340
:103A4000F76AC470FCF76AC471BA707A6E5A6C3047
:103A50000B8D15E800D76AFCD76ABA6CDA6C8D1347
:103A6000E46CD76AFCE46DD76ABA6C7A6C7AA2DA35
:103A70006C8D00F76CC470FCF76CC4718D06E4703B
:103A8000D76AFCE471D76AE4780802C4F2FA70F3EA
:103A9000BCC4F2FA71F36F8D03F76AF02AC46C8D1F
:103AA0000CF76AC46D380F6CF00638F06D096C6D58
:103AB0008D03F76AC46C38F06CF006380F6D096C32
:103AC0006D8D0CE46DD76A8D0DF76AC46D4B6D4B2F
:103AD0006D381F6D8D0EF76A2803C46EF0230B6DD1
:103AE0000B6D0B6D6801F0058FFF6E2F1B8D0DF7B1
:103AF0006A10098FFF6E80A96D6E2F0CFA6D6E2F04
:103B000007F86DF5C714C46E8D0CF76A280FEB6EBD
:103B1000CFDA708D074B716B70FEFA8D13F76AC4A4
:103B20007AFCF76AC47B8D0DF76A3006BA7A9A7010
:103B30002F04BA7A7A70DA7A9004A2DA898D00F7C3
:103B400089C47AFCF789C47BE4780802C4F2FA7A63
:103B5000F3BCC4F2FA7BF38D0CF76A5C5C283CC4BE
:103B60006C8D0DF76A60846CD76A6F8D03F76AF00D
:103B70002AC46C8D10F76AC46D380F6CF00638F0EB
:103B80006D096C6D8D03F76AC46C38F06CF0063803
:103B90000F6D096C6D8D10E46DD76A8D0FF76AC4D7
:103BA0006D4B6D4B6D381F6D8D0EF76AC46E4B6E8D
:103BB0004B6E4B6E4B6E38036EF0260B6D0B6D0B20
:103BC0006D0B6D78016EF0058FFF6E2F1B8D0DF75D
:103BD0006A10098FFF6E80A96D6E2F0CFA6D6E2F23
:103BE00007F86DF5C714C46E8D10F76A280FEB6ED9
:103BF000CFDA708D064B716B70FEFA8D05F76AC4D3
:103C00006C8D0FF76A30066089706C2F0480A97084
:103C10006C10038F006C78406C30038F406CE4783C
:103C20000800C4F2FA6CF3BCC4F2FA6CF38D10F71E
:103C30006A5C5C283CC46C8D0FF76A60846CD76A40
:103C40006F8D03F76A9F280FF016C46C8D05F76A15
:103C5000846C68403002E840D76AC4793FAB0D6F8E
:103C60008D03F76A280FC46C8D05F76AA46C1002E7
:103C7000E800D76AC4793FAB0D6F8D03F76A680F10
:103C8000B005C48F9CC4916F8D03F76A5DE8008D09
:103C9000008F90006E8F006FC800F0057A6E1D2FA8
:103CA000F7DA6C8D00F76A1C1C5DF50002C470C564
:103CB0008002F50102C471C58102F50202C58202CB
:103CC000F50302C58302BA707A6CDA70E470C580BD
:103CD00002E471C58102E4780804C4F28F20F36F16
:103CE0008D03F76AC47C5DF5591D1C5DF5D91DFD7A
:103CF000F5DA1D7A64DA62AE90065F56038D03F73B
:103D00006A8D05D76AC4793FCB0D6F8D03F76AD0F2
:103D1000038F019B6FABB56F8D03F76A280FC46CDF
:103D20008D0EF76A28F0046CD76A6F8D03F76A2846
:103D30000F8D04D76A6FE460D00B8D03F76A280FEC
:103D4000C46C5FF60A6FE460D00B8D03F76A280F2E
:103D5000C46C5F120B6F8F0060E806C48F9CC49127
:103D60008F009A8F007C8FFF7DE5571DC48E8FFCDE
:103D70006C8F016DBA85DA877A6CDA62DA64DA9868
:103D8000E5591D1C5DF5D91DFDF5DA1D7A64DA6271
:103D9000E8E7C481E814C482E85FC4A2E815C4A3BC
:103DA0008F009B8F00B56FE3018F00F1E4FDE4FE0F
:103DB000E4FF8F0FB18FA0B0FAB0FA8F10FB0000B4
:103DC0008F03F1E8005DC86CD006D8F28F20F33D78
:103DD000D8F2C4F33D10EF8F5DF28F02F38F6CF2D7
:103DE0008F20F38F0CF2FA9CF38F1CF2FA9DF38F65
:103DF0003DF28F00F38F7CF2C4F38F0FF28F30F31C
:103E00008F1FF28F00F38F2FF28F00F38F3FF28F0F
:103E100000F38F4FF28F00F38F5FF28F00F38F6FFD
:103E2000F28F20F38F7FF28F30F3E4782D8F0078BC
:103E30003FF30C8F10783FF30C8F20783FF30C8FFB
:103E400030783FF30CAE6FE80504785DD8F28F0E42
:103E5000F33DD8F28F2DF33D7D28F05DE8406FCD26
:103E6000008D00FCF785DC608485D50402F785842D
:103E700086D50502FC9005F785DC608485D50602B1
:103E8000F7858486D50702FC90043D9004C87CD059
:103E9000CE6F60F5601C885FD60402F55F1C881C3D
:103EA000D605023D900460F5601C885FD60602F5D9
:103EB0005F1C881CD607023D9004FC9004AD7CD0AA
:103EC0009B6FE8211C1CFDE880D60002D60202E8A8
:103ED000FBD60102D603026F8D00E85CDAF28F4C4C
:103EE000F2E47724B1C4F36FE8070478C4F28F9F3B
:103EF000F38D05E800D76A6FE8070478C4F2E47927
:103F0000287FC4F3E4786800F0306820F02CEBB828
:103F1000DAF2BCEBB9DAF26FE8070478C4F28D0587
:103F2000F76A287FC4F3E4786800F00E6820F00A8E
:103F3000EBB8DAF2BCEBB9DAF26FEBB9DAF2BCEB60
:103F4000B8DAF26FE478C4F2E4F3C476697679F013
:103F50001C300DAB76E478EB76DAF2BCDAF22FECBB
:103F60008B76E478EB76DAF2BCDAF22FDF6F8D0035
:103F70008F0090008F01783F3E0E8F02783F3E0EFB
:103F80008F04783F3E0E8F08785F3E0EF762680020
:103F9000F02A68FFF029FCF76268FFF020FCF76266
:103FA0006803F01A280FC46CFCF762DC28F0046C7C
:103FB00068DEF00AE490000478C490002F02FC90C0
:103FC000046F8D03F76A280FD005BA96DA986FE46C
:103FD0009A2820D00B8D03F76A280F0830C49A6FF7
:103FE000E49A280F9CC49AF00318309A6FE49A2838
:103FF00010F00ABA98DA62E49A28EFC49A6F8D0337
:10400000F76A280FF0019C8D12D76A6F8D12F76A3C
:10401000280FD01DD76A3F9B0D8D17F76A48FFC444
:10402000892989778F00793FCB0D8D03E800D76A06
:104030006F9CD76A6F8D12F76A280FD0123F0D055B
:104040008D17F76A04B7C4B78D03E800D76A6F9C71
:10405000D76A6F8F2CF28F00F38F3CF28F00F38FB3
:104060004DF28F00F36F8F0CF28F00F38F1CF28FE5
:1040700000F38F2CF28F00F38F3CF28F00F38F6CE4
:10408000F28F20F3E8F1C4F4E800C4F5C4F6C4F7F5
:104090008F5F838F1C848F5F858F1C868D0078F4E3
:1040A000F4F03678F2F4D0F6E4F5D7833A83E4F608
:1040B000D7833A83E4F7D7833A838FF2F478F3F423
:1040C000D0FBE4F5D7833A83E4F6D7833A83E4F769
:1040D000D7833A838FF3F42FC5E800C4F4C4F5C442
:1040E000F6C4F78F00B38F00B48F01EF6FE8F8C408
:1040F000F4E800C4F5C4F6C4F78F5CF28FFFF3BA9E
:1041000083DA6C8D0078F9F4F03678F2F4D0F6E4C6
:10411000F5D7833A83E4F6D7833A83E4F7D7833A33
:10412000838FF2F478F3F4D0FBE4F5D7833A83E499
:10413000F6D7833A83E4F7D7833A838FF3F42FC516
:10414000E800C4F4C4F5C4F6C4F7BA6CDA83180204
:10415000EF3F08105F5603CD888D00F783281FC4FA
:104160006CFCF783FC608483D50002F7838484DCD5
:10417000D50102FCFCF783FC608483D50202F7833F
:104180008484DCD50302DD60880EFD3D90046E6CF6
:10419000D06F5F5603BAF4DA6CBAF6DA6E8FFAF4BF
:1041A00033EFEFE46F288044B6D0E75880B68D0037
:1041B000F783C470E46D6470B0D8E4AFBC2803C466
:1041C000AF5DF5BF14C470F5C314C4718F5CF2C445
:1041D000F3E4FE8D04E4FEF0FCFEFAF870E46D1CDE
:1041E0009004BCFDFC9004E46F287FF021280FC4EC
:1041F00072601C1C1C380F720472C4723F4711D8C5
:10420000F2C4F3FC3D3F6411D8F2C4F32F0EF783E0
:10421000D8F2C4F3FC3DF783D8F2C4F3FC3DE46E5E
:10422000F0326D1CFDF781C472FCF781C473EB732F
:10423000E4727A727AA2DA728D00F772C47AFCF7AD
:1042400072C47BEEE47AD8F2C4F3FC3DE47BD8F28E
:10425000C4F32F0EF783D8F2C4F3FC3DF783D8F2F2
:10426000C4F33DE46D608822D8F2C4F3FC3DF783CB
:10427000D8F2C4F3FC3DF783D8F2C4F3FC3DF783D6
:10428000D8F2C4F38F5CF28F00F38F4CF2FA71F323
:104290005F5603E46F9F28074D1C5DE4721F5411A5
:1042A0008111821183118411851186118711881162
:1042B000E46F9F28074D1C5DE4721F711188118700
:1042C000118611851184118311821181115C90076F
:1042D00000C473E47280A473CE6F8F5CF28F0FF30F
:1042E0008F00AC8F00AD3F750DBAF5DA6CE800FDBC
:1042F000DA6EDAF58FF5F478F7F4D0FBBAF55A6E8A
:10430000D064E4F7C4AEF068E4AC1C5D1F411278E1
:10431000F7F4F0FBBAF42D6DBAF62D6DE46CE46C95
:10432000E46CE46CE46CE46CE46CE46CE46CE46C0D
:10433000E46C6E70DFE824C4708D8FAED772DCAE93
:10434000D772DCAED772DCAED772DC6E70ED780758
:10435000ADD0088D87F7720803D7723A6EABAD38CF
:1043600007ADE4FDF0FCBA6EDAF5BA6C5A6ED08790
:104370008F5CF28F01F38FF6F48F00F10000FAB03A
:10438000FA00008F03F15F5603661245128F8072A8
:104390008FFB73E4AD8D9000CF7A72DA72E800EB98
:1043A000AEDAF2BCDAF28D00E824C4705FC7118F78
:1043B00080728FFB73E4AD28078D9000CF7A72DA9C
:1043C000728D00E824C4707807ADD040E800EBAEF1
:1043D000DAF2BCDAF2BC8D00DAF2BC8D04DAF2BC9F
:1043E0008D21DAF2BC8D00DAF2BCDAF2BC8D7FDA14
:1043F000F28F5CF28F00F38F4CF28F01F38F00F19C
:1044000000008F00FA00008F03F1ABAC5FC7118F83
:104410009C858F00868D008F01F47800F4D0FBE43A
:10442000F5D7853A85E4F6D7853A85E4F7D7853A16
:10443000858F00F47801F4D0FBE4F5D7853A85E464
:10444000F6D7853A85E4F7D7853A85E800C4F4C401
:10445000F5C4F6C4F78F6DF28FF8F38F7DF28F01FC
:10446000F38F0DF28F04F38F0CF2FA9CF38F1CF292
:10447000FA9DF38F2CF2FA9EF38F3CF2FA9FF38FA2
:104480004DF2FAA1F36FE49BF027AB7CF87C3E8EF3
:10449000D0058F007CF87CF5591D1C5DF5D91DFDFC
:1044A000F5DA1D7A64DA628F009BAE90045F5603E2
:1044B000F87CF5591DBC1C5DF5D91DC46DF5DA1DE0
:1044C000C46CBA629A645A6C10016FAB7CE47C6471
:1044D0008EF0145DF5591D1C5DF5D91DFDF5DA1D35
:1044E0007A64DA62DA986F8F50F68F007CF87CF588
:1044F000591D1C5DF5D91DFDF5DA1D7A64DA626F70
:10450000E8008D00DA6CDAA4E8013FDA13DAA6E8F5
:10451000023FDA13DAA8E8043FDA13DAAAE8083F20
:10452000DA136F8D17D76C1A6CE800D76CFEFC3A63
:104530006CE8188D007A6CDA6C6F5F5603FAF5B18F
:104540008F5CF2E4B1480FC4F38FFDF45F5603FAB9
:10455000F5B08F00F10000FAB0FA8F10FB00008F69
:1045600003F18FFCF45F560338FEEF8F5CF28F0F80
:10457000F38FFBF45F5603FAF5B28FFEF45F560338
:10458000FAF5B8FAF6B98FFFF45F5603E4B22807DC
:104590001C5D1F4C145C1465147314B1145C145C22
:1045A000145C145C14E800C4F5C4F6C4F76F8F0003
:1045B000F5BAB3DAF6E4B208E0C4F56F8F09F2E4B5
:1045C000F35C5C5C280FC46C8F19F2E4F31C28F0D8
:1045D000046CC46C8F29F2E4F35C5C5C280FC46D3E
:1045E0008F39F2E4F31C28F0046DC46DBA6C8F00AF
:1045F000F5DAF6E4B208E0C4F56F8F00F5E4B5C46F
:10460000F6E4B208E0C4F56F4050607010204080BE
:104610000018314A61788DA1B4C5D4E0EBF4FAFDFD
:10462000FFFDFAF4EBE0D4C5B4A18D78614A3118EE
:1046300058032803FA02D002A60280025C023A0262
:104640001A02FC01E001C501AC0194017D01680181
:10465000530140012E011D010D01FE00F000E2009A
:10466000D600CA00BE00B400AA00A00097008F00C8
:1046700087007F00780071006B0065005F005A00C2
:10468000550050004B00470043003F003C003800FD
:10469000350032002F002D002A00280025002300BD
:1046A00021001F001E001C009011D7F7DBD8C2C0EC
:1046B0007BADB59D900090007185E87BA5736A6C19
:1046C00009665D604B5BBA569852D74E694B4448B9
:1046D0006045B542EA3FB63DA83BBB39ED373B36B6
:1046E000A3342233B6315E30182FE32DBE2CA62B17
:1046F0009C2A9F29AC28C527E8261426492586240C
:10470000CB2317236A22C42124218A20F51F661F88
:10471000DB1E551ED41D571DDD1C681CF71B881B96
:104720001E1BB61A511AF01991193519DB18841885
:104730002F18DD178C173E17F216A7165F161816DE
:10474000D3159000154E150E15CF14921456141C47
:1047500014E313AB1374133E130A13D712A412738A
:104760001243121412E511B8118C11601135110B9E
:1047700011E210BA1092106B1045101F10FB0FD6EB
:104780000FB30F90000F6E0F4C0F2B0F0A0FEA0E96
:10479000CA0EAB0E8D0E6F0E510E340E170EFB0DA2
:1047A000E00DC40DA90D8F0D750D5B0D420D290D8A
:1047B000100DF80CE00CC80CB10C9A0C840C6E0CAB
:1047C000580C420C2D0C180C030CEE0BDA0BC60B1C
:1047D000B20B9F0B8C0B790B660B540B410B2F0B01
:1047E0001E0B0C0BFB0AEA0AD90AC80AB70AA70A69
:1047F000970A870A770A680A580A490A3A0A2B0A66
:104800001C0A0E0AFF09F109E309D509C809BA090A
:10481000AC099F099209850978096B095F0952095A
:1048200046093A092D09210916090A09FE08F30863
:10483000E708DC08D108C608BB08B008A5089B0833
:1048400090000886087B08710867085D08530849CE
:10485000083F0836082C082208190810080608FD29
:1048600007F407EB07E207D907D107C807BF07B767
:1048700007AE07A6079E0795078D0785077D077575
:10488000076D0765075D0756074E0746073F073761
:10489000073007290721071A0713070C070507FE2A
:1048A00006F706F006E906E206DB06D506CE06C7E1
:1048B00006C106BA06B406AD06A706A1069B069475
:1048C000068E06880682067C06760670066A0664F0
:1048D000065E06590653064D06480642063C063754
:1048E0000631062C06260621061C06160611060CA5
:1048F0000607060106FC05F705F205ED05E805E3E8
:1049000005DE05D905D405CF05CB05C605C105BC17
:1049100005B805B305AE05AA05A505A1059C059832
:104920000593058F058A05860582057D0579057540
:104930000571056C056805640560055C055805543E
:10494000054F054B054705430540053C0538053433
:104950000530052C052805250521051D0519051619
:104960000512050E050B05070503050005FC04F9F6
:1049700004F504F204EE04EB04E704E404E004DDCF
:1049800004DA04D604D304D004CC04C904C604C297
:1049900004BF04BC04B904B604B204AF04AC04A957
:1049A00004A604A304A0049D049A0497049404910B
:1049B000048E048B048804850482047F047C0479BB
:1049C000047704740471046E046B04680466046361
:1049D0000460045D045B0458045504530450044D02
:1049E000044B0448044504430440043E043B04399A
:1049F000043604330431042E042C0429042704252E
:104A000004220420041D041B0418041604140411B9
:104A1000040F040D040A040804060403040104FF3F
:104A200003FC03FA03F803F603F303F103EF03EDCA
:104A300003EB03E803E603E403E203E003DE03DB46
:104A400003D903D703D503D303D103CF03CD03CBBE
:104A500003C903C703C503C203C003BE03BC03BA33
:104A600003B803B703B503B303B103AF03AD03AB9F
:104A700003A903A703A503A303A1039F039E039C0C
:104A8000039A03980396039403920391038F038D73
:104A9000038B038903880386038403820381037FD6
:104AA000037D037B037A0378037603740373037136
:104AB000036F036E036C036A036903670365036492
:104AC00003620360035F035D035C035A03580357EB
:104AD0000355035403520350034F034D034C034A41
:104AE000034903470346034403430341033F033E93
:104AF000033C033B033903380337033503340332E4
:104B00000331032F032E032C032B03290328032730
:104B100003250324032203210320031E031D031B7B
:104B2000031A0319031703160315031303120310C3
:104B3000030F030E030C030B030A03090307030609
:104B4000030503030302030103FF02FE02FD02FC4F
:104B500002FA02F902F802F702F502F402F302F295
:104B600002F002EF02EE02ED02EB02EA02E902E8D5
:104B700002E702E502E402E302E202E102DF02DE12
:104B800002DD02DC02DB02DA02D802D702D602D54D
:104B900002D402D302D102D002CF02CE02CD02CC87
:104BA00002CB02CA02C902C702C602C502C402C3BE
:104BB00002C202C102C002BF02BE02BD02BB02BAF3
:104BC00002B902B802B702B602B502B402B302B229
:104BD00002B102B002AF02AE02AD02AC02AB02AA59
:104BE00002A902A802A702A602A502A402A302A289
:104BF00002A102A0029F029E029D029C029B029AB9
:104C000002990298029702960295029402930292E8
:104C10000291029000028F028E028E028D028C029F
:104C20008B028A0289028802870286028502840238
:104C3000830283028202810280027F027E027D0261
:104C40007C027B027B027A0279027802770276028A
:104C500075027402740273027202710270026F02B2
:104C60006E026E026D026C026B026A0269026902D8
:104C700068026702660265026402640263026202FD
:104C80006102600260025F025E025D025C025C0221
:104C90005B025A0259025802580257025602550244
:104CA00055025402530252025102510250024F0265
:104CB0004E024E024D024C024B024B024A02490286
:104CC00048024802470246024502450244024302A6
:104CD000420242024102400240023F023E023D02C5
:104CE0003D023C023B023B023A02390238023802E2
:104CF00037023602360235023402340233023202FF
:104D00003102310230022F022F022E022D022D021B
:104D10002C022B022B022A02290229022802270236
:104D20002702260225022502240223022302220250
:104D30002102210220021F021F021E021E021D026A
:104D40001C021C021B021A021A0219021802180283
:104D5000170217021602150215021402130213029B
:104D6000120212021102100210020F020F020E02B2
:104D70000D020D020C020C020B020A020A020902C9
:104D800009020802070207020602060205020502DE
:104D900004020302030290050102000200020090D7
:104DA00005030800080F280F200700902601900433
:104DB0000F0B0F0F7F5F009008010307070F1F3FC6
:104DC0003F0090043C163F7FFF90080090040D03C5
:104DD000FF900A00900468FDFFFFFEFFF2F8E8D0A4
:104DE0008080009004F1FEFFFFFEFFF8FCF0E04041
:104DF00080009004E040A080808000000101020358
:104E00000090048000E0C000900601010000000155
:104E100005071F075F3EB43440F0E3800000010047
:104E200007031F0F1D3E7878F0E080C1780FFF90D8
:104E30000491DF0F033F0F7F3FFFFF271F7FFFFF1F
:104E4000FFE3FF0F073F1FFF7FFFFF00DCFDFCFFBD
:104E5000900CE8F0FFFEFF900C009005C0F0E0E839
:104E6000F8F8F8FEFEFDFE009004C080C0E0F0F00F
:104E7000FCF8FCFCFEFE00900401000603020F1685
:104E80000F3F3F1C1E00900501010306071F0E1E69
:104E90001E1E3E010000010F83070F3F1F90043FBD
:104EA0007F3F0000030103071F0F1F1F1F3F3F3FEE
:104EB0007F3FFF7FFF900E7FFF900FFEFFFDFEFC08
:104EC000FEFCFCF4F8F2F8E5E3EFEFFEFFFEFEFE79
:104ED000FCF8FCF8F8F8F1F7F3F7EF0090080100A0
:104EE000FC67FEFCF8F000900A1FFEF8FCF0F805E5
:104EF0000307070E0F0C1C0E1C3C381839783903B9
:104F00000302070E060C0E0C1C181C1C38383985C1
:104F1000831A0D2F115B051367465EEECE98DC8772
:104F200003040E181933332F674EEFDEDC98FCBFF5
:104F3000BF7FFFF5F2E0D0C0800090067FFF7FFFCB
:104F4000FBFCC0E00080009006FF90041F9F071F3D
:104F50000703030100010001FF9004BF7F070F0753
:104F600003030100010000FF9010FEFF900F0000FE
:104F700080008000C080C0C0E0C0C0E0E0C0000091
:104F800080008080C08080C0C0C0E0C0C0E00090D1
:104F90000402020301030103010301030100900461
:104FA000010003900A009006FF900A009004FF00A1
:104FB000FF900A00900680C081C081C183C387C76B
:104FC000009004800080808180818383878F8700A8
:104FD00090040B10FF5F7FFF9005F9FD009004081F
:104FE000077F3FFF9006FDFE009004A820FCFCFE1A
:104FF000FF90057FFF00900430C0FAFCFEFF900593
:105000007FFF00900A8080C0C080C000900B80C0ED
:1050100080C0C000900A020004060C0400900C0638
:105020000006061F1E7F3F7F3E7F3F7F3F7F7F3F03
:105030007F3F7F3E3E3F3E7F3F3F7F7F7F3F7F7F83
:105040003F3F3F7F7F7FFFFF7FFF900A3F7F9004BE
:10505000FF902BEFDFFF901EE0E0D0E0C0C080802B
:10506000C0C0C08000808000F0F0E0E0E0C080C000
:105070008090083B73737B7B7BFFF37FF77F900609
:105080007939317B7F737F77F77F7FFF7FFF7FFFEA
:10509000F0F8B0F0E0E0E0F0F0E0C0E0C0C0E0E048
:1050A000F8B8F8F09004E09007C0E000900C060615
:1050B0000090100404FF90057F9006FF7F7FFF7F24
:1050C0007FFFFF7FFF7FFF7FFF7FFF7F7FFFFFFF70
:1050D000C0C0C0E0900AC0DEE0900FE2FC00900E7D
:1050E0000F1000900F0F10100F1F0F1F0F1F0F1F1B
:1050F0000F000000EF000F001F9008001F000020AD
:10510000DF0000C09009000000C000C000C090088F
:1051100000C0000000C000900ED30D00900EBE7FB6
:105120000000010001000100010001000100C100B8
:10513000900401000100010001000100014081FC18
:1051400000FEFCFEFCFEFCFEFCFEFCFEFCFEFC0089
:1051500000FC900E00900F0F00900E1F00900F1299
:10516000F100900EE100000001900C857900000133
:10517000030103010301030103010303FF0000F81E
:10518000FCF8FCF8FCF8FCF8FCF8FCF8FC0000FC6F
:10519000F8FCF8FCF8FCF8FCF8FCF8FCF800900CC3
:1051A0000100130F00900E170F00900C8000D4F830
:1051B00000900EE8F000900EFF0100900E7EFE00C1
:1051C000900E0700900F0303010300900CF0000302
:1051D00000900DF0F8FFFF7F900FFF7FFF7FFF7FB4
:1051E000FF7FFF7FFF7FFF7FFF8FC79FCF9FDF9FE7
:1051F000DFBFFF9FFFBFDF9FFF8F8F9F8F8F9F902E
:1052000005BF9F9FBF9FBFF8F8E8F0E0F0F0F0E126
:10521000EFFF9006F0F8F0F0F0E0E0E0F0E0FF9053
:10522000067F3F1F1F001F0000D0E0FEF4FCFFFFC1
:10523000FF7F3F9004009005FCF8FFFEFFFFC0C019
:10524000C0E020C000900AE0C0C0E0E000900A800A
:10525000060F0E0E0E0790040F0F07030F0703062D
:105260000E060F070F070F0F070F079004031F3FCE
:105270001F3F3F9FDFFFEFDFFF90063F3F1F3F3F96
:105280001FDF9FFF90088080820086841C0C38D826
:10529000B8F8FCF8FAFC008000808804089898B8F8
:1052A000F8F8FCF8FCFC7F9005FF7F7FFF7F3F3F15
:1052B0007F7F7F3F7FFF7FFFFF7FFF7F90063F3F26
:1052C0003FC0C0E0C0F0E0E0F0F0E0F8F8FCF8FE2D
:1052D000FDE09006F0E0F0F0F8F0FCF8FCFE009045
:1052E0000A0301000500900D0101020000080919E0
:1052F000182B335179A377E78F8F2F7FBF0C0408CA
:105300000D19193333F36787CF1F1F3F7FFEFCFE54
:10531000FCFEFCFEFCFEFCFEFCFEFCFEFCFCFEFCBF
:10532000FEFCFEFCFEFCFEFCFEFCFEFCFE0F9010F4
:105330001F0F1F0F1F0F1F0F1F0F1F0F1F0F1F0FFD
:10534000EFDFEFDFEFDFEFDFEFDFEFDFEFDFEFDFED
:10535000DFFFDFFFDFFFDFFFDFFFDFFFDFFFDFFF5D
:10536000C2C1C7C3C7C7DF9004FFDFFFFFFFDFC3B2
:10537000C1C3C7C7CF9004DF9005FFDFFF9006F5DC
:10538000F7E1D1C0E08080C080FF9006FBFFE1E044
:10539000C0900480C0C1F0F1F0F9F8FDF8FDFEFD09
:1053A0000201000100F0E1F0F9FCF9FCFDFEFD7CDA
:1053B000FF00010001FEFCFEFCFEFCFFFDFCFDFD0C
:1053C000FF9005FC9008FFFDFF90061F3F7F3F7F89
:1053D0007FFFFFFCFEF8FCF8FCFCFC3F1F7F3FFF5B
:1053E0007FFEFFFCFEF8FCF8FCFEFCD3C3AF8FCFC2
:1053F0008F3F1F3F90041F3F3F3FE3E7C7CF0F9F03
:105400001F1F3F1F1F3F9005FF9009F787C783C1EC
:105410000381FF9008D7EF83C381838381F8FCF871
:10542000FCF8FDFAFDFBFFFBFDFFFFFBFBFCF8FCBE
:10543000F8FDF8FDF9FFF9FFFBFFFBFBFF5F3FFF06
:105440009005FEF8FCF0F8F8F7FFFF7F3FFF7FFFC5
:10545000FFFEFCFCF8F8F8FFF8FFFFFAFEFEFFFF86
:10546000FFDF3F1F1F1F0F1FEFFFFFFEFCFEFFFFB1
:10547000FF7F3F3F1F1F1FFF1FFFFFFE7E3F7E7FFF
:105480007FFFFF9FBFDF9FFFCFDFFFFE7F9004BF47
:10549000BFBF9FFFFFDF9004CF030707070F87877A
:1054A0008F8F8FCF8FDF8F8FDF0703030707078F64
:1054B00007078F8F8FDF8F8FDFF8F8E0E0E0F0C015
:1054C000E0C0C0C0E0C0C08080F09005E0E0E0C077
:1054D000E0C0C080C0C0807F9011FF7FFF7FFF7F52
:1054E000FF7FFF7FFF7FFF7FFFBFFF9FDF9FDFBF4C
:1054F000FF9FFFBFDFBFFF9FDF9FBF90059FBF9F45
:10550000BF9FBFBF9FBF9FFFFFFCFFFCF4E8F0E021
:10551000F0E0F0E0E0F0E0FF9004F8F8F0F0F0E008
:105520009007FF90047FFF1F90070F1F0FFF90044D
:105530003F7F3F3F3F1F9007C0C0E09005F0E0F085
:10554000F0E0E0F0E0F0C080C0C0C0E0E0E0F0E0FB
:10555000E0F0E0F0E0F00303000101006000280843
:10556000181E0F1E071F03010001000060003030ED
:10557000381C0E1F0F0FFF90047F7F3FFF1F7F1F00
:105580002FFFEFFF90087F7F3F3F1F1FEF1FFFFFA1
:10559000FCFEFEFF900DFCFEFF900E1F3FDF9FFF05
:1055A000900C1F3F3FFF900D473CFF9008FEFEFF11
:1055B0009004BDC3FF90160F7F030F01858180FF0C
:1055C0009008AFDF0F0703038001FEFEFC9005F09B
:1055D000F8E1D0C0C080FF00FEFFFDFEF9FCF9F845
:1055E000F0F0E0E080C080FFFEFCFEFCFEFEFF90DD
:1055F000067FFFFFFFFCFEFCFEFCFEFEFEFF9004AC
:105600007FFF7FFF0F0F0F1F0F1F1F1F7F3FFF9099
:10561000061F0F1F0F0F1F3F1FFF9008EFDFEFDF69
:10562000EFDFEFDFEFDFEFDFEFDFFFDFDFFFDFFFDA
:10563000DFFFDFFFDFFFDFFFDFFFFFFFDFFFFFDF5A
:10564000DFDFFFDF9005C7C7FBC7FFDFFFDFFFDF3F
:10565000DFDFCFDFCFCFC7CFC7FF809004C0C0C090
:10566000E0F3D1F7FBFF900480C080C080C0C0C0D1
:10567000E0E1FF90060100010001027FFCFFFCF960
:10568000FCF9FCF7F800010001827DFCFFFEFDFC47
:10569000FDFCF9F9FF9008FEFEFCFEFCFEFCFFFCA1
:1056A000FF9007FEFEFC9006FFFEFCFFFF7EFF3F23
:1056B0003F7F7F1F3F1F3FEF1FFEFEFFFE7FFF7FED
:1056C0007F3F3F1F3F1F1F1FFF7F3F3F3F9F3F3FCA
:1056D000BFFFFF9FBFDFEFCFFF3F90061FBFBF9F02
:1056E000DFDFEFDFEFFF810101818183C383A3E36C
:1056F000F7EFFF9004838183818381C183C3C7FF58
:105700009006FB9004F9FFFBFFFBFDF8FCF8FDFFA2
:10571000FCFBFFFBFFFFFBFDFBFFF9FDF9FCF8F8CD
:10572000FFFFFFF8FFF0F0FCF8FCFCFEFC7FFF7FC2
:105730007FFF9004F89005FCFEFF900700FF00003B
:10574000100F1F3FFF9004FEFF90050090043F1FC5
:10575000BF7FFF9005EF27EF0F0F03C3C3C785C3BC
:105760000381FF03CFCFC7CF07900487C383838113
:105770000301FF8FDFFFFFFEFFFFFEFEFFFEFEFEC9
:10578000FCFFFCDFDFFFDFFFFFFEFFFEFEFCFEFE97
:10579000FCFCFF8000808080009009FF00808080FA
:1057A00000900CFF7F9011FF7FFF7FFF7FFF7FFF47
:1057B0007FFF7FFFFFFFBFDF8FCF8FDF87CF8FC7D9
:1057C00083C783C3BFC19F90058F90048783878160
:1057D0008381FFE0F0F0F0E8F0F8F4FDFDFF9006C3
:1057E000E0E0F0E0F0F0F8F8FEFF90070F1F1F3F39
:1057F0003F1F7F7F7FFF90071F90053F7F3FFF90F8
:1058000008F0E0E0F0E0F0C0900480C08080E0109C
:10581000E0F0F0E09006C080C0008000E00F0F07CD
:1058200003060200900A0F070707030100900AFF12
:1058300090069F5F140C009006FF90067F3F0B07B9
:10584000009006FF9008009008FF900A009008C0A2
:105850008080C0C1C06FC3EF5FF07A4010809004B9
:10586000C08080C0C5C3CE7F787C70603F7F7F3FA3
:105870002F3FFFBF80C080009005FF7F1F3F1F1F8D
:10588000FF7FFFFF80009005E09008101000900659
:10589000F0E0F0E0F0E0F0E0E0E0009006400090A2
:1058A0001F1F7C630C8514E71C29256B2DAC31EF81
:1058B0003D1146724A9556F75E39677A6BBD77FFA0
:1058C0007F0090460100020003000400050006006E
:1058D00007000800902D09000A000B000C000D00C5
:1058E0000E000F001000110012001300901D140094
:1058F000150016001700180019001A001B001C00E4
:105900001D001E001F0020002100000022002300B7
:105910002400250026002700280029002A002B004B
:105920002C002D002E002F003000310032003300FB
:105930003400350036003700380039003A001D00C9
:105940001D001D003B003C003D003E003F001D00CF
:10595000400041004200430044004500460047002B
:10596000480049004A004B004C004D004E004F00DB
:1059700050005100520053005400550056001D00C5
:105980001D001D00570058001D0059005A005B0003
:105990005C005D005E005F0060006100620063000B
:1059A0006400650066006700680069006A006B00BB
:1059B0006C006D006E006F0070007100720073006B
:1059C000730073007300730073007300740075003C
:1059D000730073007300730073007300730073002F
:1059E000730073007300730073007300730073001F
:1059F000730073007300730076009013770090FFBC
:105A00000090FF00902FF3570009F3600000F3604F
:105A10000000F3600090142D367E7F7D266A4CFDD9
:105A2000FEFA4C4C009005DAECD4F828F0DA7CBA97
:105A3000DC4498AACC54F8A870FAFCFC20FAFCECE0
:105A40003010200090061018383C34181800000060
:105A5000383C5C666A0C14181018180010181800EE
:105A60000000507850787800900B707850787078FB
:105A7000780090072030FCFEEC362436243654663D
:105A8000AACCCC002030FCFEEE303018FCFEF6181C
:105A9000180C0C007C7E5C664466A4C6CA0C080C1C
:105AA0003438380040607C7E5A6CA8CCC80C14187E
:105AB000283030000000F8FCF80C080C080C080C2A
:105AC000F8FCFC00486CFCFEDA6C486C680C14189E
:105AD000283030000000C4E6E406C4E6EA0C1418DE
:105AE000E8F0F000F8FCF80C080C14183038586C8A
:105AF000ACC6C6004060FEFFDE634D6E4E60426382
:105B00007D3E3E0084C6C46644666A0C080C1418C8
:105B1000687070007C7E5C664466B4FEFA0C1418F3
:105B20002830300004063A3C380CFEFFFB0C080C11
:105B3000141818000406A4F6A4F6FA0C080C14189D
:105B400068707000FCFEFE00FCFEF61810181018BD
:105B5000283030004060406040606070587C5C607D
:105B6000406060001018FCFEF6181018101828305D
:105B7000D0E0E0000000787C7C009007FCFEFE0096
:105B8000F8FCF80C080C54787038283CD8ECEC0081
:105B90002030F8FCF80C1418787CACF6E6303000B5
:105BA000080C080C080C14181018283050606000FD
:105BB00010181018586C486CACC684C6C406060091
:105BC00080C080C0F8FCBCC080C080C0F8FCFC0075
:105BD000FCFEFC06040604060A0C1418687070002B
:105BE0002030587CBCC6C60090091018FCFEF61880
:105BF0001018547EB6DB92DBDB00FCFEFC060406CC
:105C0000DAFCEC70603030181800E0F0FC1EEEF0AA
:105C1000FC1E1E00E0F0FC1E1E001018101828309C
:105C200020305466FEFFBEC3C300040604064A6C5F
:105C3000683C3418283CDCE6E600FCFEEE30203000
:105C4000FCFEEE3020303C3E3E004060FEFFEE3376
:105C5000253626303018101818000000787C780C93
:105C6000080C080C080CFCFEFE007C7E7C0604067A
:105C70007C7E7C0604067C7E7E00787C7C00FCFEBC
:105C8000FC0604060A0C3438380044664466446650
:105C9000446664060A0C14181800101850785078DE
:105CA000527B527B557EDAFCFC00406040604060D5
:105CB000446644665A7C6C7070000000FCFEBCC6F2
:105CC00084C684C684C6FCFEFE000000FCFEBCC682
:105CD000C40604060A0C343838000000E4F6F40662
:105CE000040604060A0CF4F8F8009005383C3C065B
:105CF0003C3E5C667C3E3E0040604060787C5C667A
:105D0000446644667A7C7C009005383C5C6646605C
:105D100044667A3C3C00040604063C3E5C664466ED
:105D200044667C3E3E009005383C5C667A7C5C6054
:105D30007C3E3E001C1E2E3020307C7E6E3020309B
:105D40002030300090053C3E5C667C3E3C067A7C10
:105D50007C0040604060787C5C66446644664466D3
:105D60006600101818003038301810181018383C19
:105D70003C00080C0C00181C180C080C080C3438DB
:105D8000380040604060486C547868705078586CB7
:105D90006C00303830181018101810181018383CD3
:105DA0003C009005787C547E547E547E547E7E0068
:105DB0009005787C5C66446644664466660090059F
:105DC000383C5C66446644667A3C3C009005787CCE
:105DD0005C6644667A7C5C60600090053C3E5C6674
:105DE00044667C3E3C0606009005587C6C76566006
:105DF00040604060600090053C3E5E60783C3C0640
:105E00007A7C7C0020302030787C6C302030203050
:105E1000381C1C00900544664466446644667A3C1F
:105E20003C0090054466446644666A3C3418180099
:105E3000900544664466547E6A3C283C3C009005CC
:105E400044666A3C3418283C5C66660090054466EB
:105E500044667C3E3C067A7C7C0090057C7E7A0C15
:105E6000141828307C7E7E00900510182830506071
:105E700060303018180090054060603030182830CD
:105E800050602040009006F0F8F800F0F8F80000AC
:105E900000383C3C202030203020302030383C3C42
:105EA00000383C380C080C080C080C080C383C3C3A
:105EB00000900DFAFCFC00383C5C6644667C7E5C1D
:105EC00066446644666600787C5C6644667A7C5C00
:105ED0006644667A7C7C00383C5C66466040604084
:105EE0006044667A3C3C00787C5C66446644664468
:105EF0006644667A7C7C007C7E5E604060787C5C78
:105F00006040607C7E7E007C7E5E604060787C5C71
:105F100060406040606000383C5C6646605C7E5C6F
:105F20006644667A3C3C004466446644667C7E5C1B
:105F3000664466446666007C7E7618101810181059
:105F40001810187C7E7E000406040604060406046D
:105F50000644667A3C3C0044664A6C54786870504B
:105F600078586C4C6666004060406040604060401D
:105F70006040607C7E7E00446644666C7E547E5C3D
:105F800066446644666600446644666476547E5C95
:105F90006E4C6644666600383C5C66446644664403
:105FA0006644667A3C3C00787C5C6644667A7C5C3D
:105FB00060406040606000383C5C66446644665403
:105FC0007E5A6C743E3E00787C5C6644667A7C5CEB
:105FD000664466446666003C3E5E604060783C3CD9
:105FE0000604067A7C7C007C7E7618101810181047
:105FF0001810181018180044664466446644664435
:106000006644667A3C3C004466446644666A3C28C2
:106010003C341810181800446644664466547E5494
:106020007E6A3C283C3C00446644666A3C3418283E
:106030003C5C66446666004466446644666A3C347A
:10604000181018101818007C7E7C060A0C141828EA
:106050003050607C7E7E00FEFFFE03121B1D1E166C
:106060001810182830300006070D0E1A1C687C78AE
:106070000C080C080C0C0010187E7F5E6362030590
:106080000604061A1C1C0000007C7E7618101810EE
:10609000181018FEFFFF0004067E7F7D0E0C0E1404
:1060A0001E2C365466660010183820203020302010
:1060B00030203030181800383C5C66446644664432
:1060C0006644667A3C3C00101830383018101810BE
:1060D000181018383C3C00383C5C6664060A0C1406
:1060E0001828307C7E7E00383C5C6664061A1C1CD6
:1060F0000644667A3C3C00486C486C486C486C7CB2
:106100007E7A0C080C0C007C7E5E604060787C7CA3
:106110000644667A3C3C00383C5C664660787C5CB1
:106120006644667A3C3C007C7E7C060A0C080C14B3
:1061300018101810181800383C5C6644667A3C5CED
:106140006644667A3C3C00383C5C6644667C3E3C77
:106150000644667A3C3C00020305060A0C14182823
:10616000305060A0C0C00000003038687C763B5DD5
:106170007E5A6F753E3E00900B203050606000608C
:1061800070603050606000900920301018101810B6
:106190001810181018283030001018383C383C34CB
:1061A000181018180010181800900B40606000902C
:1061B000097E7F7F00900D4060600040606000902D
:1061C000076476BADCDC0090072030383C5C6070F5
:1061D00038380C7478683030000000101810187CC3
:1061E0007E7618101818009005FCFEFC061A1C1488
:1061F00018101818009005101828306070A0F0E0F2
:10620000303000000020302030F8FCB8CCD4182802
:106210003030009005F8FCEC3020302030F8FCFCE9
:106220000090051018F8FCF4385078B0D8D80090D9
:1062300005A8FCA8FCF80C34382830300090054044
:1062400060F8FCD86C4C60603030009005E0F0E005
:106250003020302030F0F8F8009005E0F0E030E039
:10626000F0E030E0F0F0000000787CB4DEBCFEEC42
:10627000FEBCFEFA7C7C009005AC31734EFF7F1FA4
:106280007C08218D35734E1F7C0D0834001F011FC3
:106290007C02344050E07D3E0804F7004004F700E3
:1062A00040053F0040053F002005630015056300E1
:1062B00020058700400587004005CF003505CF0049
:1062C0000008060032080600100818000E08180022
:1062D00010082A0040082A00100090B8010090839E
:1062E00002FB00907E024C0A0504180F0600FF0016
:1062F0004700FF0F84033C0A01FF00FF0047FF0235
:106300003E0A0500FF0C0006300047FF034C0A015F
:10631000FF07300047FF02380A050534FFFF00FF82
:106320000047FF033E0A0105340C0600FF0047FF4B
:10633000023E0A050418FFFF00FF0047FF03380A6A
:1063400001FF00FF0047FF024C0A0500FF0C00069A
:10635000300047FF033E0A01FF07300047FF023EBF
:106360000A050418FFFF00FF0047FF034C0A01FF66
:1063700006300047FF02380A050534FFFF073000EA
:1063800047FF033E0A010418FFFF00FF0047FF021A
:106390003E0A05FF06300047FF03380A0100FF0CE4
:1063A0000007300047FF02480A050418FFFF00FFFE
:1063B0000047FF033E0A01FF00FF0047FF023E0ABD
:1063C0000500FF0C0006300047FF03480A01FF07E5
:1063D000300047FF02380A050534FFFF00FF004781
:1063E000FF033E0A0105340C0600FF0047FF023E92
:1063F0000A050418FFFF00FF0047FF03380A01FFEA
:1064000000FF0047FF02480A05FF06300047FF0370
:106410003E0A01FF07300047FF023E0A050418FF4D
:10642000FF00FF0047FF03480A01FF06300047FF57
:1064300002380A050534FFFF07300047FF033E0A14
:10644000010418FFFF00FF0047FF023E0A05FF0698
:10645000300047FF03380A0105340C240730004799
:10646000FF02460A050420FFFF00FF0047FF033E2E
:106470000A01FF00FF0047FF023E0A0500FF0C0073
:1064800006380037FF03460A01FF07380037FF02CE
:10649000380A050534FFFF00FF0037FF033E0A01FD
:1064A00005340C0600FF0037FF023E0A050420FFFA
:1064B000FF00FF0037FF03380A01FF00FF0037FF2E
:1064C00002460A0500FF0C0006380037FF033E0AAB
:1064D00001FF07380037FF023E0A050420FFFF00D6
:1064E000FF0037FF03460A01FF06380037FF023876
:1064F0000A050534FFFF07380037FF033E0A010491
:1065000020FFFF00FF0037FF023E0A05FF063800AC
:1065100037FF03380A0100FF0C0007380037FF027D
:10652000420A05041CFFFF00FF0037FF033E0A017B
:10653000FF00FF0037FF023C0A0500FF0C00063495
:106540000047FF03420A01FF07340047FF02340AF5
:10655000050534FFFF00FF0047FF033C0A01053437
:106560000C0600FF0047FF023C0A05041CFFFF0069
:10657000FF0047FF03340A01FF00FF0047FF02420C
:106580000A0500FF0C0006340047FF033C0A01FF28
:1065900007340047FF023C0A05041CFFFF00FF0010
:1065A00047FF03420A01FF06340047FF02340A0591
:1065B0000534FFFF07340047FF033C0A01041CFFBA
:1065C000FF00FF0047FF023C0A050534FFFF0634C9
:1065D0000047FF03340A0105340C3207340047FF3B
:1065E000A2000BBBBCCCCCCDDD92BBBCCDDDDEEFC5
:1065F000F000A2000443333332222292433332218B
:1066000011100000A200044333333222229243339C
:10661000322111100000A2000BBBBCCCCCCDDD930D
:10662000BBBCCDDDDEEFF000A2000BBBBCCCCCCD03
:10663000DD92BBBCCDDDDEEFF000A20004433333BE
:10664000322222934333322111100000A2000BBBEF
:10665000BCCCCCCDDD92BBBCCDDDDEEFF000A2002A
:10666000044333333222229343333221111000008A
:10667000A20009999006A2999008A294449007A2BA
:10668000449008A2449008A2449008A2449008A311
:1066900044900700B000A9ECDDFD297127B0FA672E
:1066A0007EB374A7306EB032E02BB2888FA8A9B049
:1066B0003BE8928A121DD5F0A0E3A68EEDE02014EF
:1066C00024B01346667777677766B0674422100F69
:1066D000EEEDDCB0DCCBBB89889004B0998899AA38
:1066E000ABFBDDFDB0E0F1112223243457B07790ED
:1066F0000457767416B020422F3E1B1DDDDAB0CA57
:10670000ADCABD8ED9FB9DB0C90BAE9CF91BFBE099
:10671000B0CB00AE2D31131225B01072235151357C
:106720000632B024423120321F3D41B0F131F4EF46
:106730001100F0DDB00BFDDDD9FBC9E99BB0ABBEAC
:106740009CA9B9DFF8C1B0F1F0D30421602064B096
:10675000F606273607F72154B02242043FE4103DE5
:1067600000B00A0DCDB09BAAD8BBB0BE9EB9BBEBA2
:10677000C0AFFBB0E1E01002112D6133B011315216
:106780002155215241B0404231211310121FB00156
:10679000D0FD0CF9D0D9FBB0CDBDE8FCAECCDBFD13
:1067A000B0BE0EFEF5B011020FB021031F123E2243
:1067B0001410B04F4E21311105E2309000532D647A
:1067C000287FF08FD1A0B0DFBCCFB09C9000AAB0E2
:1067D000EDD0EFD09000DFC1DFB00C0B11C1F001A4
:1067E000F0F0B0011202F303204130B04212230254
:1067F0001201102EA050FFDFC3BDFDCAB4B0CEEE13
:10680000C0FBEFB0DCE0B0CEFDD0C2B3FC0FE0A027
:10681000E2C3E3D522024123A005316F073035D60C
:10682000F3A03F521F6D13B5F1FEA00F1C0EE0B197
:10683000CEDDDFA0CDCEAD0CC0AD081CA0CDFDEDF2
:10684000390F1EF1C1A01020002004F04240A02109
:1068500040403213013050A0305EF6D01210F1D01B
:10686000A0EB10FDEEDAE0BCD2A0ACFCCEBDEFC1D7
:10687000DEDE90009F3E93D0ED797D22A00F2011A7
:10688000204D320422A022323023312105F1900024
:1068900041F402FF1FE1A1DAA0FFB2CEEEDDECDF92
:1068A000CD9000F9BE9DADBBFDC0EC9000FC4B1F30
:1068B000F0F2233F409000513413454255F5339098
:1068C00000154314F302E1100051449008A2009017
:1068D0000401111AAAA3ABC21111009004A20090E6
:1068E0000401111AAAA3ABC21111009004A20FEE69
:1068F000A2ACC0AEEED993FEDAAAA988EEEEF0887B
:106900009028E888900FE888900BE8889007E8883E
:106910009007E8889007E8889006E8889004E8885F
:106920009004E8889005E8889004E8889004E88856
:106930009004E8888888E8888888E8888888E888D3
:106940008888E8888888E8888888E8888888E88847
:106950008888E88888E88888E88888E88888E888D7
:106960008888E88888E88888E88888E88888E888C7
:106970008888E888E88888E88888E88888E888E857
:106980008888E888E88888E88888E88888E888E847
:1069900088E888E88888E888E888E88888E888E8D7
:1069A00088E888E88888E888E888E88888E888E8C7
:1069B00088E888E888E888E888E888E888E888E857
:1069C00088E888E888E888E888E888E888E888E847
:1069D000E888E888E8E888E888E888E8E888E888D7
:1069E000E888E888E8E888E888E888E8E888E888C7
:1069F000E8E888E888E8E888E8E888E8E888E88857
:106A0000E8E888E888E8E888E8E888E8E888E88846
:106A1000E8E888E8E888E8E888E8E888E8E888E8D6
:106A2000E8E888E8E888E8E888E8E888E8E888E8C6
:106A3000E8E888E8E8E888E8E8E888E8E8E888E856
:106A4000E8E888E8E8E888E8E8E888E8E8E888E846
:106A5000900488E8900488E8900488E8900588E825
:106A6000900488E8900488E8900688E8900788E811
:106A7000900788E8900788E8900B88E8900F88E8EE
:106A8000902FC8E8900FC8E8900BC8E89007C8E8B6
:106A90009007C8E89007C8E89006C8E89004C8E8DE
:106AA0009004C8E89005C8E89004C8E89004C8E8D5
:106AB0009004C8E8E8E8C8E8E8E8C8E8E8E8C8E812
:106AC000E8E8C8E8E8E8C8E8E8E8C8E8E8E8C8E8C6
:106AD000E8E8C8E8E8C8E8E8C8E8E8C8E8E8C8E8D6
:106AE000E8E8C8E8E8C8E8E8C8E8E8C8E8E8C8E8C6
:106AF000E8E8C8E8C8E8E8C8E8E8C8E8E8C8E8C8D6
:106B0000E8E8C8E8C8E8E8C8E8E8C8E8E8C8E8C8C5
:106B1000E8C8E8C8E8E8C8E8C8E8C8E8E8C8E8C8D5
:106B2000E8C8E8C8E8E8C8E8C8E8C8E8E8C8E8C8C5
:106B3000E8C8E8C8E8C8E8C8E8C8E8C8E8C8E8C8D5
:106B4000E8C8E8C8E8C8E8C8E8C8E8C8E8C8E8C8C5
:106B5000C8E8C8E8C8C8E8C8E8C8E8C8C8E8C8E8D5
:106B6000C8E8C8E8C8C8E8C8E8C8E8C8C8E8C8E8C5
:106B7000C8C8E8C8E8C8C8E8C8C8E8C8C8E8C8E8D5
:106B8000C8C8E8C8E8C8C8E8C8C8E8C8C8E8C8E8C5
:106B9000C8C8E8C8C8E8C8C8E8C8C8E8C8C8E8C8D5
:106BA000C8C8E8C8C8E8C8C8E8C8C8E8C8C8E8C8C5
:106BB000C8C8E8C8C8C8E8C8C8C8E8C8C8C8E8C8D5
:106BC000C8C8E8C8C8C8E8C8C8C8E8C8C8C8E8C8C5
:106BD0009004E8C89004E8C89004E8C89005E8C8A4
:106BE0009004E8C89004E8C89006E8C89007E8C890
:106BF0009007E8C89007E8C8900BE8C8900FE8C86D
:106C0000902FCAC8900FCAC8900BCAC89007CAC8AC
:106C10009007CAC89007CAC89006CAC89004CAC8D4
:106C20009004CAC89005CAC89004CAC89004CAC8CB
:106C30009004CAC8C8C8CAC8C8C8CAC8C8C8CAC8C8
:106C4000C8C8CAC8C8C8CAC8C8C8CAC8C8C8CAC8BC
:106C5000C8C8CAC8C8CAC8C8CAC8C8CAC8C8CAC8AA
:106C6000C8C8CAC8C8CAC8C8CAC8C8CAC8C8CAC89A
:106C7000C8C8CAC8CAC8C8CAC8C8CAC8C8CAC8CA88
:106C8000C8C8CAC8CAC8C8CAC8C8CAC8C8CAC8CA78
:106C9000C8CAC8CAC8C8CAC8CAC8CAC8C8CAC8CA66
:106CA000C8CAC8CAC8C8CAC8CAC8CAC8C8CAC8CA56
:106CB000C8CAC8CAC8CAC8CAC8CAC8CAC8CAC8CA44
:106CC000C8CAC8CAC8CAC8CAC8CAC8CAC8CAC8CA34
:106CD000CAC8CAC8CACAC8CAC8CAC8CACAC8CAC822
:106CE000CAC8CAC8CACAC8CAC8CAC8CACAC8CAC812
:106CF000CACAC8CAC8CACAC8CACAC8CACAC8CAC800
:106D0000CACAC8CAC8CACAC8CACAC8CACAC8CAC8EF
:106D1000CACAC8CACAC8CACAC8CACAC8CACAC8CADD
:106D2000CACAC8CACAC8CACAC8CACAC8CACAC8CACD
:106D3000CACAC8CACACAC8CACACAC8CACACAC8CABB
:106D4000CACAC8CACACAC8CACACAC8CACACAC8CAAB
:106D50009004C8CA9004C8CA9004C8CA9005C8CA9A
:106D60009004C8CA9004C8CA9006C8CA9007C8CA86
:106D70009007C8CA9007C8CA900BC8CA900FC8CA63
:106D8000902F88CA900F88CA900B88CA900788CA2B
:106D9000900788CA900788CA900688CA900488CA53
:106DA000900488CA900588CA900488CA900488CA4A
:106DB000900488CACACA88CACACA88CACACA88CA3B
:106DC000CACA88CACACA88CACACA88CACACA88CA2B
:106DD000CACA88CACA88CACA88CACA88CACA88CA5D
:106DE000CACA88CACA88CACA88CACA88CACA88CA4D
:106DF000CACA88CA88CACA88CACA88CACA88CA887F
:106E0000CACA88CA88CACA88CACA88CACA88CA886E
:106E1000CA88CA88CACA88CA88CA88CACA88CA88A0
:106E2000CA88CA88CACA88CA88CA88CACA88CA8890
:106E3000CA88CA88CA88CA88CA88CA88CA88CA88C2
:106E4000CA88CA88CA88CA88CA88CA88CA88CA88B2
:106E500088CA88CA8888CA88CA88CA8888CA88CAE4
:106E600088CA88CA8888CA88CA88CA8888CA88CAD4
:106E70008888CA88CA8888CA8888CA8888CA88CA06
:106E80008888CA88CA8888CA8888CA8888CA88CAF6
:106E90008888CA8888CA8888CA8888CA8888CA8828
:106EA0008888CA8888CA8888CA8888CA8888CA8818
:106EB0008888CA888888CA888888CA888888CA884A
:106EC0008888CA888888CA888888CA888888CA883A
:106ED0009004CA889004CA889004CA889005CA8819
:106EE0009004CA889004CA889006CA889007CA8805
:106EF0009007CA889007CA88900BCA88900FCA88E2
:106F0000900744009A009E00EE000A010E0146011F
:106F10004A018E01F40144028E02B4020E032803DA
:106F20007603C003020402041E044E048A04C20451
:106F3000DC04FE04680584059E05AC05BA05D4058D
:106F4000EC05FC0512060D000D000D000D000D00F6
:106F50000D000D000D000D00830102100D008301D6
:106F600002100D00830102100D00830102100D00BC
:106F7000830102100D008401857602100D0083014B
:106F800002100D00830102100D00830102100D009C
:106F9000830102100D0084018536060680058702F4
:106FA00003010D0003010D0003010D0003010D009D
:106FB00003010D0003010D0003010D0003010D008D
:106FC00003010D0003010D0003010D0003010D007D
:106FD00003010D0003010D0003010D0003010D006D
:106FE00003010D0003010D0003010D0084020604DE
:106FF00003020A02030103010D0103FF0D0103FF58
:107000000D0103FF0D0103FF0A0D0E0004000E0029
:1070100003010D0003010D0003010D0003010D002C
:1070200003010D0003010D000A020D0003010D0014
:107030000D0003010D000D0003010D000D00030103
:107040000D000D000A0E0E008007870403010D00DD
:1070500003010D0003010D0003010D0003010D00EC
:1070600003010D0003010D0003010C0003010D00DD
:1070700003010A0503010A0203010D000D000301CB
:107080000D000D0003010D000D0003010A0D0E009F
:1070900003010D000D0003010D000D0003010D00A3
:1070A0000D000D0003010D000D000D000D000D0081
:1070B0000D000D000D000D0003010D000D000D0071
:1070C0000D000D000D000D000D000D0003010D0061
:1070D0000D000D000D000A020D0003010D000D0052
:1070E00003010D000D0003010D000D0003010D0053
:1070F0000D000A0E0E000D0203010D0203010D0228
:1071000003010D0203010D0203010D0203010D0233
:1071100003010D0203010D0203010D0203010D0223
:1071200003010D0403010D0403010D0403010D040B
:1071300003010D1003010D0403010D0403010D04EF
:107140000301840B061603010D000D0003010D0061
:107150000D0003010D000D000D0003010D000D00D9
:107160000D000D000D000D000D000D000D000301C0
:107170000D000D000D000D000D000D000D000D00A7
:107180000D0003010D000D000D000D000A0A0E0098
:1071900003010D0503010D0503010D0503010D0597
:1071A00003010D0503010D0503010D2004000D056C
:1071B0000D050D050600040B0D0103010D01030172
:1071C0000D0103010D0103010D0103010D01030177
:1071D0000D0103010D0203010D0203010D02030164
:1071E0000D0203010D0203010D0203010D02030153
:1071F0000D0203010D0303010D0503010D0503013C
:107200000D0503010D0303010D020A070D00060021
:107210008A0204050D0603010D0603010D0803FF94
:107220000D0003FF0D000A0A0E000D0303010D03FC
:1072300003010D0303010D0303010D0303010D03FE
:1072400003010D0303010D0303010D0303010D03EE
:1072500003010D0303010D0303010D0303010D03DE
:1072600003010D0303FF0D0303FF0D0303FF0D03D4
:1072700003FF0D0303FF061203020D0003020D00BE
:1072800003020D0003020D0003020D0003020D00B6
:1072900003020D0003020D0003020D0003FE0D00AA
:1072A00003FE0D0003FE0D0003FE0D0003FE0D00A6
:1072B00003FE0D0003FE0D0003FE0D0003FE0D0096
:1072C000060003010D0003010D0003010D00030181
:1072D0000D0003010D0003010D0003010D0003016A
:1072E0000D0003FF0D0003FF0D0003FF0D0003FF62
:1072F0000D0003FF0D0003FF0D0003FF0D0003FF52
:107300000D0006000D0103040D0103040D0103042B
:107310000D0103040D0103040D0103040D0101001F
:107320000D0503010D0403010D0403010D03030109
:107330000D0303010D0303010D0203010D020301FF
:107340000D0203010D0103010D0103010D020616DB
:107350000D0003010D0303010D0303010D030301E0
:107360000D0303010D0303010D0303010D030301CD
:107370000D0303010D0303010D0303010D030301BD
:107380000D0403010D0403010D03061D0301030198
:1073900003010D0003010D0003010D0003010D00A9
:1073A00003010D0003010D0003010D0003010D0198
:1073B00003010D0103010D0203010D0203010D0084
:1073C0000A0D0E0003010D0003010A0F03010D0A4F
:1073D00003FF0D0103FF0D0203FF0A0D0E00030260
:1073E0000D00030203010A0F03FF0D0003FF0D0050
:1073F00003FF0D0003FF0D0003FF0D000A0D0E003B
:107400000D0702010D0702010D0302010D0102012A
:107410000D0002010D000201020102010201020140
:107420000D0002010D0002010D0102010D03020118
:107430000D0702010D0702090D0702090D030209DC
:107440000D0102090D0002090D00020902090209DD
:10745000020902090D0002090D0002090D010209CD
:107460000D0302090D0702090600100111B40D02F7
:1074700010C30D0411E40D0810C10D0B113410C31D
:1074800011E40D0B010011DB0D0210DF0D0411E002
:107490000D0810F00D0B111910D811DC0D0B0100A7
:1074A00011840D0810C80D0810C30D1801001197A4
:1074B0000D0810C80D0810C30D12010011B80D02FF
:1074C00010DF0D0211E00D0810F00D08113910D772
:1074D00011E20D06010011C60D0510D911E00D05D0
:1074E0000D080D05110210C611D70D2401001199C8
:1074F0000D0510DF11DD0D0810D50D24010011F46C
:107500000D0610DF11F00D0410CF11E90D0810C3A6
:107510000D08010011FF0D0310DF11FC0D0210CF4B
:1075200011FB0D0510C30D080100F502011100113A
:10753000007F7F000400001F00900580F00F10F016
:107540000F00012E9000FD3E14D28BD5B756B0F23D
:107550002ED4E3BF2DDB65C8BC55C6B7A5B9F84D21
:10756000C434A1BBBCFE2F13F0B42C1E1E0F3F135E
:10757000E294A0531FAA0989CDB326A436B54C10B6
:10758000E15BDCBFB4F0862A5ED0F03371B41DF24B
:10759000B62030E38785B4BC7B3BD6DD2A07CDCC53
:1075A0004C21FF03FE2FF5B1B422C310E1E04A1FC6
:1075B00010A4B815CDF934A2EF4DA44FE403F400A4
:1075C000272A41A43B30E5FE3E5815DBA42A13CB05
:1075D00052EC3C6DFDA0A8D8B889BFCA6F31B0236A
:1075E00042232342435437B4D012FE0093F2D2F028
:1075F000B4E4C101D3B3D3D002A4F016B71E25E181
:1076000012DFA47D1F011F396FFE2BA03F4C0FCA54
:107610000AA919B9A41F01C012B5B2D41BAC61A547
:107620002B131C15B14C94F333E13A55FF02F0AC27
:107630001E03B5D0FD3F011C9402CDF7AA7C2E019C
:10764000F4A411F1302C51EF72EFA86A112FE3F07E
:10765000100001A4B4E2FD1D5DCF3F3E94C3853808
:1076600000E1C5C1C09411C3E1003E213F6AA0659D
:1076700064655464556457A4EFD50000F2F1C20E5E
:1076800094D7B901C79000E2DEF6948F00C16A3F3B
:107690002F7C20A415CD7102F11F301FA0647360F0
:1076A000F2DCEDACCD94830FB5964FF6F117A4E262
:1076B000F3ED40A25900E49000A8C88818BF7EE30B
:1076C00074A4040E13E3E111B4FDA0FE4DD0EB1F32
:1076D000BEFBCDA0CEBEE0FB0EC31CD1A4EF22E0CA
:1076E0002E3C42CF689000155E63DB530843B8A47C
:1076F0002EF0F4EE24C312F190005374F512BB0681
:10770000E4D690003BE5340E11B72E3EA41F5D1168
:10771000E040E22C01900003FC2FBEEB9E188B9002
:1077200000EC8AABEACEEA005394E7970D24864E2C
:10773000BD4F900001FD04A2E02FE54394B51B2E40
:10774000F2DE4F010D90005CE31D12F1DE1AFE9493
:10775000B5DF22ED5EB42FF08420017E1430B457E3
:10776000AB8465912ECDF58A7E82941E1FFF2EE19B
:107770002FE3F594FF15E1E32CF5E100941D3FC4E0
:10778000C30B3D219680C0BD58B0D8C880BD80E8ED
:10779000580F28F0380FFF80707F71F6252F2717BC
:1077A00080C45E122B00A9DE9E80D98C08CCE8FE36
:1077B000FB1D80F222E7F70052104080306F220458
:1077C000F0E5BFDE80CDA0D828DDDDEFF08003122C
:1077D00005040303224E803120101E21DF0CF080AF
:1077E000E3E1FFF2C3C4C04F80F2030233E61F3F60
:1077F0003E8042E2F11F2D2D01CF80F1D0EE10FF2F
:10780000F1ED1080FEF01FE12F1D31FF802E32F1CF
:10781000312201020E8021001F0FF1E00000010063
:107820009008141C24345F6FBFC1B1815F4F2C24BA
:1078300014140800180030007E007E00300018008C
:10784000080090FF0090E24C002D20517569636B99
:1078500064657620313620555342202D01D00044F6
:10786000656275673A204D61696E0046015669642C
:10787000656F20495251733A015C01058D027E000B
:1078800000000429037E4C002D204F5054495858C5
:107890002074657374202D01D00044656275673AC9
:1078A00020417564696F0086014558542049525142
:1078B000733A019C01058E027E00C6012430303AE5
:1078C0003330303001DC0105003000009401054305
:1078D000037E00C6014A6F79323A0544037E00D424
:1078E000010545037E0006024A6F79333A054603D7
:1078F0007E0014020547037E0046024A6F79343A3F
:107900000548037E0054020549037E004601546980
:107910006D65636F64653A015801055E5F7E005CCA
:1079200001055D5F7E004C002D204E776172702056
:1079300044616973616B7573656E202D01D00044DD
:10794000656275673A205461626C69737420526590
:10795000636F72646572000602636873756D206FF1
:107960006B20000602636873756D206261640060BD
:1079700001058C027E004602050000C0004A020597
:107980000100C0004E02050200C000860245786575
:10799000637574696E67205144313620434D44202D
:1079A00031008602457865637574696E67205144BD
:1079B000313620434D44203200C60250726F677248
:1079C0006573733A2090042501DA020893027E0061
:1079D0008601566F6C6F75743A01980105605F7E81
:1079E000009C01055F5F7E009E014A6F79353A0574
:1079F0004A037E00AC01054B037E00DE014A6F792D
:107A0000363A054C037E00EC01054D037E001E0353
:107A10004A6F79373A054E037E002C03054F037EEB
:107A2000005E034A6F79383A0550037E006C030507
:107A300051037E006E7C927CA77CAD7CCE7CE17C89
:107A4000F37CFA7C067D0D7D197D207D2C7D337DB8
:107A5000467D4D7D7E7D8A7D967D9D7DA47DAB7D21
:107A6000B27DC97DE07DF87DF87DF87DF87DF87DFB
:107A7000F87D097E107E1C7E237E2F7E367E427E20
:107A8000497E557E5C7E5C7E5C7E5C7E5C7E5C7E40
:107A90005C7E5C7E5C7E5C7E5C7E5C7E5C7E5C7E16
:107AA0005C7E5C7E5C7E5C7E5C7E5C7E5C7E5C7E06
:107AB0005C7E5C7E5C7E5C7E5C7E5C7E5C7E5C7EF6
:107AC0005C7E5C7E5C7E5C7E5C7E5C7E5C7E5C7EE6
:107AD0005C7E5C7E5C7E5C7E5C7E5C7E5C7E5C7ED6
:107AE0005C7E5C7E5C7E5C7E5C7E5C7E5C7E5C7EC6
:107AF0005C7E5C7E5C7E5C7E5C7E5C7E5C7E5C7EB6
:107B00005C7E5C7E5C7E5C7E5C7E5C7E5C7E5C7EA5
:107B10005C7E5C7E5C7E5C7E5C7E5C7E5C7E5C7E95
:107B20005C7E5C7E5C7E5C7E5C7E5C7E5C7E5C7E85
:107B30005C7E5C7E5C7E5C7E5C7E5C7E5C7E5C7E75
:107B40005C7E5C7E5C7E5C7E5C7E5C7E5C7E5C7E65
:107B50005C7E5C7E5C7E5C7E5C7E5C7E5C7E5C7E55
:107B60005C7E5C7E5C7E5C7E5C7E5C7E5C7E5C7E45
:107B70005C7E5C7E5C7E5C7E5C7E5C7E5C7E5C7E35
:107B80005C7E5C7E5C7E5C7E5C7E5C7E5C7E5C7E25
:107B90005C7E5C7E5C7E5C7E5C7E5C7E5C7E5C7E15
:107BA0005C7E5C7E5C7E5C7E5C7ED87F3F801F81DD
:107BB00006031000030B00350050000307000144CA
:107BC000007E0001001B0025002D00566964656FD2
:107BD0002D4952510044697361626C6500456E61C4
:107BE000626C652000010000FF8B027E04010041F1
:107BF000002430303A3330303020577269746500D9
:107C000090047F13027E0C01005C0043616C6320D2
:107C1000436873756D00060314000611002E0044BE
:107C2000005F007D00CD009005CE007E0501001DA7
:107C30000055706C6F61642C706C617920736F6E8D
:107C4000670090043B14027E0801003A0053746FF1
:107C50007020736F6E6700010000FF15027E09013E
:107C600000500053657420736F6E672073706565F4
:107C700064000200000F16027E0A01006B00536FC1
:107C80006E67206368616E6E656C206D61736B005A
:107C90000307000717027E0B01009900A900B2003C
:107CA000BB00C400A900A900A900A900537063206B
:107CB0005265706F72742054797065004E6F6E65F6
:107CC0002090040054696D65636F646500566F6CA5
:107CD000204F757420004D6F6420436D6420009028
:107CE000040F16027E0D0100D90052657475726E84
:107CF00000060310000107009004FF67027E0D01DB
:107D000000130052657475726E005055901F50CF6D
:107D10005651D452CBCDBFCE57D5CCD1D0CAC0C18D
:107D2000C2C3C4C5C6C7C8C9D2D29A9C9B55DFA0DE
:107D3000A1A2A3A4A5A6A7A8A9AAABACADAEAFB0BB
:107D4000B1B2B3B4B5B6B7B8B99D539E6F9FCD80ED
:107D50008182838485868788898A8B8C8D8E8F909B
:107D600000919293949596979899BFCFCED35555FD
:107D70009B55559A559009BA5590059C559004BB52
:107D8000BC55900A5455D6D7D8D9DADCDBDDDED124
:107D9000BABBBCBDBE58595A5B5C5D5E5F60616238
:107DA000636465666768696A6B6C6D6E6F7071722B
:107DB000737475767778797A7B7C7D7E7F5657559C
:107DC00090204B8264827D829682AF82C882E1825B
:107DD000FA82138300091500003F250100081018DE
:107DE00023000000200100900704031111A000707F
:107DF000005C7C0000230103000310EF00900411DD
:107E00000004031313A0004000593C000023013379
:107E1000003310EF0090041300040310110231002E
:107E2000005C000000430103000310EF0090041108
:107E30001104031313A0A150005C4C000043013354
:107E4000003310EF009004130000091100003325E7
:107E500001000810184301000020010090070403EE
:107E60001313A03F50005C4C00004301330033105B
:107E7000EF0090041300000B130000331200010CFC
:107E800000002301000020010090080B13000033C4
:107E90001200000C000043010000200100900C01C2
:107EA000009005020090050400900508009005165A
:107EB00000900532009005640090040128009004B1
:107EC0000256009004051200900410240090042033
:107ED00048009004409600900481920000000163E5
:107EE00084000000032768000000065536000000EB
:107EF0001310720000002621440000005242880046
:107F00000001048576000002097152000004194343
:107F10000400000838860800001677721600003347
:107F2000554432000067108864000134217728002E
:107F300002684354560005368709120010737418FE
:107F400024002147483648FC83FC83FC83FC83FCE7
:107F500083FC83FC83FC8360900450900440900475
:107F600030900420900410900401901002901003AF
:107F700090100490100590100690100790100203C6
:107F8000FF000313FF000423FF000633FF00084334
:107F9000FF000B53FF000F63FF001273FF001783F6
:107FA000FF001B93FF0023A3FF002DB3FF0039C385
:107FB000FF0046D3FF0058E3FC0063F3FC0063F3CB
:107FC000FC0004002400DA00020000083680008073
:107FD00000901007009005E820010000FF3110001C
:107FE000010090160200020001000100900D010046
:107FF0000100020002000200020002000200020072
:1080000001000100900D01000100020002000200C9
:1080100090811F01011F01011F01013F02033F0267
:10802000037F04043F04003F04003F02037F040475
:10803000FF08057F0404FF0805FF08057F08007F8F
:10804000040408000800080028000000210C0314A4
:10805000221023246520861CA620C644C928C830C7
:108060002B31AD49324E73665B776E7AC0040020C7
:10807000001F7C6B45B05E586F59301F002E258F56
:1080800029773A1E537E5FFF77FF7F6027E0033139
:108090004D109004202010002020000040200000FF
:1080A000401000002010000020000000F0F1F2F36A
:1080B000F4F5F6F7F8F9B0B1B2B3B4B58C857F003A
:1080C000008C857F00008C857F40007205721572E0
:1080D0001D722513617F79777FFC857FBB44C000CB
:1080E000FF90FFFF90FFFF90FFFF90FFFF90FFFFCB
:1080F00090FFFF90FFFF90FFFF90FFFF90FFFF902A
:10810000FFFF90FFFF90FFFF90FFFF90FFFF90FFAA
:10811000FF90FFFF90FFFF90FFFF90FFFF90FFFF9A
:1081200090FFFF90FFFF90FFFF90FFFF90FFFF90F9
:10813000FFFF90FFFF90FFFF90FFFF90FFFF90FF7A
:10814000FF90FFFF90FFFF90FFFF90FFFF90FFFF6A
:1081500090FFFF90FFFF90FFFF90FFFF90FFFF90C9
:10816000FFFF90FFFF90FFFF90FFFF90FFFF90FF4A
:10817000FF90FFFF90FFFF90FFFF90FFFF90FFFF3A
:1081800090FFFF90FFFF90FFFF90FFFF90FFFF9099
:10819000FFFF90FFFF90FFFF90FFFF90FFFF90FF1A
:1081A000FF90FFFF90FFFF90FFFF90FFFF90FFFF0A
:1081B00090FFFF90FFFF90FFFF90FFFF90FFFF9069
:1081C000FFFF90FFFF90FFFF90FFFF90FFFF90FFEA
:1081D000FF90FFFF90FFFF90FFFF90FFFF90FFFFDA
:1081E00090FFFF90FFFF90FFFF90FFFF90FFFF9039
:1081F000FFFF90FFFF90FFFF90FFFF90FFFF90FFBA
:10820000FF90FFFF90FFFF90FFFF90FFFF90FFFFA9
:1082100090FFFF90FFFF90FFFF90FFFF90FFFF9008
:10822000FFFF90FFFF90FFFF90FFFF90FFFF90FF89
:10823000FF90FFFF90FFFF90FFFF90FFFF90FFFF79
:1082400090FFFF90FFFF90FFFF90FFFF907E407830
:1082500018FB4BABC230E2209C0042A9018D0D42BD
:108260005C682AC0405C4E12C0FF9005517569637E
:108270006B646576203136205553422090063100DC
:108280000800013301DCBC2343FF9004A0FFA0FFE2
:10829000A0FFB6FF0000B7FF9005A0FF0000A0FF01
:1082A000A0FFA1FFA0FF7368617265645F6D656DDB
:1082B0006F72795F726561643A2030782530347866
:1082C0003D307825303278203078253034783D3094
:1082D0007825303278200A007368617265645F6DBA
:1082E000656D6F72795F77726974653A20206C6F83
:1082F000636B65645F74780A007368617265645FBC
:108300006D656D6F72795F77726974653A202030A0
:1083100078253034783D3078253032782030782513
:108320003034783D307825303278200A0073686127
:108330007265645F6D656D6F72795F777269746580
:108340003A20206C6F636B65645F74780A00736811
:10835000617265645F6D656D6F72795F7363726181
:108360007463687061645F726567696F6E5F74786B
:108370005F736176653A206C6F636B0A00736861A6
:108380007265645F6D656D6F72795F73637261743E
:1083900063687061645F726567696F6E5F74785F50
:1083A000726573746F72653A206C6F636B0A007349
:1083B00068617265645F6D656D6F72795F7363721A
:1083C000617463687061645F726567696F6E5F7224
:1083D000785F736176653A20756E6C6F636B0A0027
:1083E0007368617265645F6D656D6F72795F7363E9
:1083F00072617463687061645F726567696F6E5FF4
:1084000074785F736176653A20756E6C6F636B0A82
:10841000007368617265645F6D656D6F72795F731B
:108420006372617463687061645F726567696F6EBF
:108430005F736176655F68656C7065723A206F7016
:10844000656E20727820616464723D307825303624
:108450006C780A007368617265645F6D656D6F7238
:10846000795F736372617463687061645F7265677A
:10847000696F6E5F736176655F68656C7065723A8F
:10848000206F70656E20747820616464723D30786E
:108490002530366C780A0053657420776174636800
:1084A000646F672E2E2E0A00436174636820534E5A
:1084B000455320726573657420627574746F6E0A1B
:1084C0000053657420534E4553206869726F6D20C8
:1084D0000A0053657420534E4553206C6F77726FBA
:1084E0006D200A00526573657420534E45530A008F
:1084F000454E4400746573745F6372633A20636829
:1085000065636B0A00746573745F6372633A20631A
:1085100072630A00746573745F6372633A20636CFC
:108520006561720A002D2D2D2D2D2D2D2D2D2D2D1A
:108530002D2D2D2D2D2D2D2D2D2D2D2D2D2D2D2D6B
:108540002D2D2D2D2D2D2D2D2D2D2D2D2D2D2D2D5B
:108550002D2D2D2D2D2D2D2D2D2D2D2D2D2D2D2D4B
:108560002D2D2D2D2D0A00746573745F6D656D6F53
:1085700072795F7061747465726E3A2064756D70A3
:1085800020626F74746F6D5F616464723D30782532
:1085900030386C7820746F705F616464723D30783D
:1085A0002530386C780A00746573745F6D656D6F83
:1085B00072795F7061747465726E3A207772697453
:1085C0006520616464723D30782530386C782070A5
:1085D00061747465726E3D30782530386C780A00AD
:1085E000746573745F6D656D6F72795F70617474BB
:1085F00065726E3A20626F74746F6D5F616464724D
:108600003D30782530386C7820746F705F61646419
:10861000723D30782530386C780A00616464723DB0
:1086200030782530386C7820633D307825780A0022
:10863000616464723D30782530386C782025780A82
:10864000007265616420616464723D307825303861
:108650006C782025780A006E616E00696E660000F5
:10866000407A10F35A00A0724E18090010A5D4E801
:108670000000E87648170000E40B54020000CA9A94
:108680003B000000E1F505000080969800000040E6
:10869000420F000000A0860100000010270000002B
:1086A00000E803000000006400000000000A000071
:1086B0000000000100000000002C76D888DC674F25
:1086C0000823DFC1DFAE59E1B1B796E5E3E453C655
:1086D0003AE651997696E8E6C28426EB898C9B624D
:1086E000ED407C6FFCEFBC9C9F40F2BAA56FA5F4F7
:1086F00090055A2AF75C936B6CF9676DC11BFCE01F
:10870000E40D47FEF520E6B500D0ED902E03009471
:108710003577050080841E080000204E0A00000006
:10872000C80C333333330F986E12831141EF8D2110
:1087300014893BE65516CFFEE6DB18D1844B381B77
:10874000F77C1D901DA4BBE424203284725E22813C
:1087500000C9F124ECA1E53D270011241FBECFEF95
:10876000D0E1DEBFCDBF14BE88E10FB6F894809390
:108770006000109260000FBE12E0A0E0B1E0E8E2FD
:10878000F0ED02C005900D92A432B107D9F716E0C2
:10879000A4E2B2E001C01D92AD3AB107E1F70E9438
:1087A0007C470C9412680C940000E9E6F0E08081AC
:1087B00082608083E89A08951F93CF93DF9360913E
:1087C0004D02635067FD9FC080914A02CCE0D0E02B
:1087D000C81BD109CF5ADD4F809149028D3209F073
:1087E0007FC0683009F08DC083EC80933D028AE53C
:1087F00080930001109224028881807641F0CE019E
:108800000E944648282F8F3F09F459C05FC09A81C3
:10881000109246028981882321F41092470222E0B7
:1088200047C0853019F490934E0241C0863081F5DF
:108830008B81813019F480EA90E004C0823041F4E9
:1088400082EB90E090934C0280934B0222E11CC09B
:108850008330C9F4992341F480E790E090934C026F
:1088600080934B0224E010C0913019F484E790E02B
:1088700004C0923041F48AE890E090934C028093D7
:108880004B0226E101C020E080E4809324021EC058
:10889000883021F421E080E592E00CC0893019F4A1
:1088A0009093500204C08A3011F421E001C020E00E
:1088B00086E492E090934C0280934B0207C088813B
:1088C00087FD2E8180E88093240206C08F81882353
:1088D00019F48E81821708F0822F8093010111C054
:1088E0008091240287FF0DC0CE010E94ED4B8F3F87
:1088F00021F48EE18093000104C0882311F01092CE
:10890000010110924D028091000184FF4AC08091C4
:1089100001018F3F09F445C0182F893008F018E095
:10892000811B8093010180913D0298E88927809303
:108930003D02112341F120914B0230914C02809174
:10894000240286FF0DC0AEE3B2E080E090E0F901C2
:10895000E80FF91FE491ED9301961817C1F708C0CD
:10896000912FD901EEE3F2E08D9181939150E1F7DF
:108970001150812F90E01F5F0196820F931F9093FB
:108980004C0280934B028EE392E0612F0E94F444EC
:10899000612F6C5F6C3019F08FEF80930101609351
:1089A000000194E189B1847131F49150D9F71092AA
:1089B0004E0210924802DF91CF911F910895A82F87
:1089C000B92F80E090E041E050EA60956F5F58F485
:1089D0002D9138EF82279795879510F0842795275A
:1089E0003F5FC8F3F3CF0895EADF8D939D93089519
:1089F000CF93CFB7CF93DF93C3954C9BE9F74C9BB5
:108A000011C04C9B0FC04C9B0DC04C9B0BC04C9B92
:108A100009C04C9B07C04C9B05C04C9B03C04C9BA2
:108A200001C081C06F93C0914A02DD27CF5ADD4F4C
:108A30002F9320E400C065E04C9B03C02F916F9101
:108A4000DECF0F931F934F9345E55F9355E53F931B
:108A50003BE014E009B104712EC06A95C9F03150B1
:108A6000D8F109B1047101130BC00894279529931B
:108A700020E4555500F46A9569F701E069B10BC02F
:108A8000102F66E02695299320E4555518F3E2CF80
:108A90000FEF69B10000162F455500F0404066E029
:108AA00014710030E2F221F0000009B1047103C03A
:108AB00009B10471A9F0011309C00894279568F25F
:108AC00000C06A95A9F700E069B1E5CF102F66E014
:108AD000269528F20000ECCF11E01CBB002717C040
:108AE0003B503195C31BD04011E01CBB0881033CB7
:108AF000F9F00B34E9F0209148021981110F12139B
:108B0000EDCF093651F10D3211F0013E39F70093E6
:108B10004F023F915F914F911F910F912F916F9154
:108B2000CCB3C0FD69CFDF91CF91CFBFCF91189566
:108B300020914F02222369F310914D02112329F550
:108B400034302AF130934D022093490210914A02A9
:108B50003BE0311B30934A021AC000914D020130B4
:108B6000A4F40AE53091000134FD12C00093000125
:108B7000CDE3D2E011C0052710E000C00BB919C049
:108B8000052710E0221F00C01DC04AE502C032EDDB
:108B9000432FC4E1D0E032E01AB114615C9A0BB10A
:108BA0001AB954E120E869E420FF05270BB927959D
:108BB000179500C000001C3FF0F66695A8F7A1F7D6
:108BC00020FF05270BB92795179500001C3FC0F61D
:108BD00029913A9541F70B7E10914E02110F0BB976
:108BE000C651D04011F01093480211E01CBB006147
:108BF0001AB11B7E402F4B7E55E05A95F1F70BB909
:108C00001AB94BB986CF1092250210922602109203
:108C10002702109228021092290210922A02109222
:108C20002B0210922C0281E080930B0110922D02F6
:108C300010922E021092300210922F0208951F936C
:108C4000CF93DF9310E0C5E4D3E000D0ADB7BEB75B
:108C50001296DC93CE9311970E9430561F5F0F90AF
:108C60000F90183291F700D08CEF92E0EDB7FEB77D
:108C7000928381830E94305683EB92E0ADB7BEB7FA
:108C800012969C938E9311970E9430568AE692E03A
:108C9000EDB7FEB7928381830E94305680E292E066
:108CA000ADB7BEB712969C938E9311970E94305623
:108CB00086ED91E0EDB7FEB7928381830E94305636
:108CC0008DE891E0ADB7BEB712969C938E93119745
:108CD0000E9430568BE891E0EDB7FEB79283818316
:108CE0000E9430568CE591E0ADB7BEB712969C93CA
:108CF0008E9311970E9430568AE591E0EDB7FEB74A
:108D0000928381830E94305600D000D0EDB7FEB729
:108D1000319684E491E0ADB7BEB712969C938E93E2
:108D2000119782E091E09383828386E091E09583BE
:108D300084830E943056EDB7FEB736960FB6F8948E
:108D4000FEBF0FBEEDBFDF91CF911F91089500D000
:108D500086EA93E0EDB7FEB7928381830E94305696
:108D6000549AF89486E993E0EDB7FEB79283818335
:108D70000E9430562AE00F900F9044EF51E012C04D
:108D800047983F9886E990E0FA013197F1F701970B
:108D9000D9F747983F9A8EE591E0FA013197F1F7BC
:108DA0000197D9F7215061F747983F98549800D020
:108DB00089E893E0EDB7FEB7928381830E94305635
:108DC0000F900F900895AF92BF92CF92DF92EF92E3
:108DD000FF920F931F936C0100D087E793E0EDB7EC
:108DE000FEB7928381830E94305685E693E0EDB70B
:108DF000FEB7928381830E9430565D985E9A209AD6
:108E00008CE593E0EDB7FEB7928381830E943056E4
:108E10005E9A0F900F9083E399E043E759E760E093
:108E200070E000E010E020E030E00E94155500D036
:108E30008AE593E0EDB7FEB7928381830E943056B6
:108E40005E985F985D9A2098289A87E493E0EDB742
:108E5000FEB7928381830E9430560F900F900E943C
:108E6000A259EE24FF24C701B6010E9479635B0179
:108E70006C0120E030E44CE955E40E949B617B01E9
:108E80008C0120E030E040E85FE30E94F562882337
:108E90001CF461E070E024C0C801B70120E03FEF9E
:108EA0004FE757E40E9495621816B4F4C601B50165
:108EB00020E030E040E251E40E949B610E94C55FE7
:108EC00084EF91E005C0FC013197F1F761507040EB
:108ED00061157105C1F707C0C801B7010E94C55FE0
:108EE000CB010197F1F71F910F91FF90EF90DF9069
:108EF000CF90BF90AF9008954F925F926F927F9204
:108F00008F929F92AF92BF92CF92DF92EF92FF9299
:108F10000F931F93CF93DF930E94654C8CE091E0F9
:108F20009093AA068093A9060E941F460E94184D9E
:108F30000E9461565B9A53980E94135982E390E015
:108F40000E94E346109225021092260210922702F8
:108F5000109228021092290210922A0210922B02DB
:108F600010922C0281E080930B0110922D0210923E
:108F70002E021092300210922F020E94D5430E94BE
:108F8000A74652E3452E51E0552E41E2642E41E0C2
:108F9000742E37E1832E31E0932E24E0A22E21E0BF
:108FA000B22E93EFC92E90E0D92E80EEE82E80E00D
:108FB000F82E06ED10E0C4ECD0E05D985E9A209AA1
:108FC00000D0EDB7FEB7528241820E9430565E9AC1
:108FD000EDB7FEB7728261820E9430565F98789436
:108FE000EDB7FEB7928281820E9430560F900F90AB
:108FF00002C00E94DC4380910B018630D1F760E013
:109000000E943D5800D0EDB7FEB7B282A1820E9407
:1090100030560F900F900E9483595F9800D0EDB7A3
:10902000FEB7D282C1820E9430565D9A2098289A5B
:10903000EDB7FEB7F282E1820E9430560F900F909A
:109040000E9420590E94A25900D0EDB7FEB71283AA
:1090500001830E9430560F900F9002C00E94DC43A3
:1090600080910B018730D1F700D0EDB7FEB7D283E6
:10907000C1830E9430560F900F900E9461560E944B
:10908000135984EF91E00E94E34697CFCF92DF928D
:10909000EF92FF920F931F93CF93DF93EC0189819F
:1090A000863009F0A1C010926B0210922D022DB7EC
:1090B0003EB7285030400FB6F8943EBF0FBE2DBFCC
:1090C000EDB7FEB7319692E0C92ED12CADB7BEB741
:1090D0001296DC92CE92119782E595E0938382837B
:1090E0008A819B81958384838C819D8197838683EC
:1090F0000E940A5381E0E82EF12C012D112D0A80E7
:1091000004C0EE0CFF1C001F111F0A94D2F7E0925E
:109110009802F092990200939A0210939B022C817C
:109120003D8130936D0220936C0240E050E0C80115
:10913000B7010E947F676093290270932A0280938F
:109140002B0290932C0210926E02109293021092B6
:10915000300210922F0200D000D000D0EDB7FEB741
:109160003196ADB7BEB71296DC92CE9211978AE0D7
:1091700095E093838283E482F5820683178380914E
:109180006C0290916D029187808780912902909165
:109190002A02A0912B02B0912C0282879387A48788
:1091A000B5870E940A53EDB7FEB73E960FB6F89406
:1091B000FEBF0FBEEDBF83E060E00E943D5880E03F
:1091C00060916C020E943D58809125029091260288
:1091D000A0912702B09128020097A105B10509F0DE
:1091E0009FC20E94D9549CC2873009F06FC083E0AF
:1091F00080930B018A819B81A0E0B0E07C01DD249B
:10920000CC248C819D81A0E0B0E0C82AD92AEA2A2A
:10921000FB2AC0922502D0922602E0922702F09209
:1092200028028E8180932D02C114D104E104F1043F
:1092300009F447C0209198023091990240919A0216
:1092400050919B02C701B6010E949E67611571058E
:1092500081059105B1F510916B020E94F5542DB76F
:109260003EB72C5030400FB6F8943EBF0FBE2DBF16
:10927000EDB7FEB7319622E030E0ADB7BEB712963B
:109280003C932E9311972EEC34E033832283148386
:109290001582C682D782E086F186938782870E94F4
:1092A0000A5380916B028F5F80936B02EDB7FEB71C
:1092B0003C960FB6F894FEBF0FBEEDBF0E94D95486
:1092C0002DC2C701B6010E94C24E28C2883009F0E3
:1092D000A0C083E080930B016A817B8180E090E0F5
:1092E000CB01772766272C813D8140E050E0622B3F
:1092F000732B842B952B6093250270932602809309
:109300002702909328022E8120932D0224E630E03C
:1093100040E050E00E947F672091290230912A02AC
:1093200040912B0250912C020E949E6720936E0266
:1093300080919302281721F085E0622F0E943D580A
:1093400080916E02809393026091250270912602B3
:1093500080912702909128020E94E656C090250233
:10936000D0902602E0902702F0902802C114D10488
:10937000E104F10409F4D2C12091980230919902DC
:1093800040919A0250919B02C701B6010E949E67CC
:10939000611571058105910509F0C0C110916B023D
:1093A0000E94F5542DB73EB72C5030400FB6F894BC
:1093B0003EBF0FBE2DBFEDB7FEB7319622E030E0C5
:1093C000ADB7BEB712963C932E93119722E934E0C5
:1093D0003383228314831582C682D782E086F18686
:1093E000938782870E940A5380916B028F5F8093DC
:1093F0006B02EDB7FEB73C960FB6F894FEBF0FBEFA
:10940000EDBF0E94D95481E060916B020E943D58EB
:1094100085C18930C1F580910B018330C1F000D046
:1094200000D082E090E0ADB7BEB712969C938E93C9
:10943000119782E594E014969C938E9313970E9463
:109440000A5320E00F900F900F900F9070C100D042
:1094500000D082E090E0EDB7FEB7928381838CE389
:1094600094E0948383830E940A5381E080930B01EC
:109470000F900F900F900F900E946E4D84E060E06F
:109480000E943D584DC1843009F053C02A813B8170
:1094900040E050E0A901332722278C819D81A0E084
:1094A000B0E0282B392B4A2B5B2B209325023093DD
:1094B000260240932702509328028DB79EB7089743
:1094C0000FB6F8949EBF0FBE8DBFEDB7FEB73196B5
:1094D00082E090E0ADB7BEB712969C938E93119741
:1094E00084E294E093838283248335834683578385
:1094F0000E940A53EDB7FEB738960FB6F894FEBF38
:109500000FBEEDBF20912502309126024091270227
:1095100050912802E0909802F090990200919A02EE
:1095200010919B0260E070E080E090E00E94155294
:10953000F7C08A30A1F486E080930B0100D000D000
:1095400082E090E0ADB7BEB712969C938E931197D0
:1095500084E194E014969C938E93139711C08B3002
:10956000B9F487E080930B0100D000D082E090E056
:10957000EDB7FEB79283818385E094E09483838383
:109580000E940A5320E00F900F900F900F90C9C0D7
:109590008C3011F500D000D082E090E0ADB7BEB7BE
:1095A00012969C938E93119785EF93E014969C935B
:1095B0008E9313970E940A532DE088E190E00FB636
:1095C000F894A895809360000FBE209360000F90E0
:1095D0000F900F900F90FFCF853009F0A1C08093BE
:1095E0000B012A813B8140E050E0A901332722276B
:1095F0008C819D81A0E0B0E0282B392B4A2B5B2B7E
:10960000209325023093260240932702509328028C
:10961000EDB7FEB73A970FB6F894FEBF0FBEEDBF99
:10962000319602E010E0ADB7BEB712961C930E93D0
:10963000119783ED93E0938382832483358346835C
:1096400057838E819F81918780870E940A538E81E4
:109650009F81A0E0B0E062E0880F991FAA1FBB1FA6
:109660006A95D1F78093670290936802A09369028C
:10967000B0936A0282E080932E0200D0EDB7FEB76D
:109680003196ADB7BEB712961C930E93119780EB2F
:1096900093E0938382838091250290912602A0918A
:1096A0002702B091280284839583A683B783809193
:1096B000670290916802A0916902B0916A02808766
:1096C0009187A287B3870E940A53EDB7FEB73C96F5
:1096D0000FB6F894FEBF0FBEEDBF609125027091EA
:1096E00026028091270290912802209167023091F2
:1096F00068024091690250916A0203E912E00E94F7
:10970000E251809331029093320280936F029093E2
:10971000700281E080930B0122E003C02FEF01C0B3
:1097200020E084E992E090934C0280934B02822FD8
:10973000DF91CF911F910F91FF90EF90DF90CF902D
:109740000895DF92EF92FF920F931F93D82EE92E88
:1097500020912E02F62E261708F4F22E2F192093B0
:109760002E020F2D10E08DB79EB708970FB6F89414
:109770009EBF0FBE8DBFEDB7FEB7319684E090E07F
:10978000ADB7BEB712969C938E9311978FE695E076
:109790009383828315830483268317820E940A534E
:1097A0002D2D3E2DC901FC018DB79EB708960FB631
:1097B000F8949EBF0FBE8DBFD801A159BD4F02C006
:1097C0008C9181938E2F8D198F15D0F38F2D1F9132
:1097D0000F91FF90EF90DF900895FF920F931F93EA
:1097E000CF93DF93182FF92E062F20912D022617E5
:1097F000F0F400D000D000D0EDB7FEB7319687EE80
:1098000095E0ADB7BEB712969C938E9311972283C5
:109810001382648315820E94305600912D028DB709
:109820009EB706960FB6F8949EBF0FBE8DBF80916F
:109830000B01833009F042C020912D02201B2093A0
:109840002D02ADB7BEB71C970FB6F894BEBF0FBEC2
:10985000ADBFEDB7FEB7319684E090E012969C93D1
:109860008E93119788E995E09383828380912502F6
:1098700090912602A0912702B091280284839583BB
:10988000A683B78300871186228713860E940A5316
:10989000212F3F2DC901EC01102F8DB79EB70C96DB
:1098A0000FB6F8949EBF0FBE8DBF06C089910E946F
:1098B0006C4D0E94544D11501123C1F7802FDF9140
:1098C000CF911F910F91FF90089582E08093C00087
:1098D00088E98093C10084E18093C40008951F92B9
:1098E0000F920FB60F9211248F939F939091C60001
:1098F0008091C00084FD07C090939C0280919D02DE
:10990000846080939D029F918F910F900FBE0F9066
:109910001F901895982F8091C00085FFFCCF9093E1
:10992000C6000895FC0190818091C00085FFFCCFA6
:109930009093C600992311F03196F5CF0895FC015C
:1099400094913196992339F08091C00085FFFCCF26
:109950009093C600F5CF0895982F8A3039F48091FE
:10996000C00085FFFCCF8DE08093C6008091C000D1
:1099700085FFFCCF9093C60080E090E00895FC0145
:109980001082758364837383628341834783468334
:109990000895FC0190818181981710F080E008956E
:1099A000A481B5816D938781815019F48181A81BB1
:1099B000B1098783B583A4839FB7F89480818F5FB3
:1099C00080839FBF81E00895FC0180818823E9F3B3
:1099D000A281B3812D918681815019F48181A81BC8
:1099E000B109B383A28386839FB7F89480818150A5
:1099F00080839FBF822F0895FC018081882319F402
:109A00002FEF3FEF13C0A281B3812D91868181504A
:109A100019F48181A81BB109B383A28386839FB700
:109A2000F8948081815080839FBF30E0C901089500
:109A300011B812B887B1856787B987B1857F87B9B3
:109A400088B1877988B988B1856088B984B18F6019
:109A500084B985B18F6085B98AB1806E8AB95E9A02
:109A60008BB18F758BB90895809133029091340238
:109A7000A0913502B09136020196A11DB11D8093CF
:109A8000330290933402A0933502B09336022A9A9F
:109A90004098409A2A980000000000000000000052
:109AA0000000089580B108958091330290913402AE
:109AB000A0913502B09136020196A11DB11D80938F
:109AC000330290933402A0933502B0933602299A60
:109AD0004098409A2998089582B9089500D000D0FE
:109AE00088E090E0EDB7FEB79283818389E097E04C
:109AF000948383830E940A53299A289A11B812B832
:109B00000F900F900F900F90089500D000D088E034
:109B100090E0EDB7FEB7928381838EE597E0948362
:109B200083830E940A532A9A289A11B812B80F9078
:109B30000F900F900F9008952091330230913402CE
:109B4000409135025091360220933702309338020B
:109B50004093390250933A028DB79EB708970FB6DB
:109B6000F8949EBF0FBE8DBFEDB7FEB7319688E06B
:109B700090E0ADB7BEB712969C938E9311978FEB82
:109B800097E09383828324833583468357830E949F
:109B90000A538DB79EB708960FB6F8949EBF0FBEB6
:109BA0008DBF08954F925F926F927F928F929F9296
:109BB000AF92BF92CF92DF92EF92FF921F93CF931B
:109BC000DF936B017C018DB79EB708970FB6F894B1
:109BD0009EBF0FBE8DBFEDB7FEB7319680E290E01D
:109BE000ADB7BEB712969C938E93119789EE97E00E
:109BF00093838283C482D582E682F7820E940A53CD
:109C000018E1EDB7FEB738960FB6F894FEBF0FBE59
:109C1000EDBF21E0822E912CA12CB12CC0E2D0E02E
:109C200095EE492E97E0592E87EE682E87E0782E24
:109C30001150D501C401012E04C0880F991FAA1F1D
:109C4000BB1F0A94D2F78C219D21AE21BF21009722
:109C5000A105B10581F000D000D0ADB7BEB7129616
:109C6000DC93CE93119714967C926E9213970E9478
:109C70000A53449A0BC0449800D000D0EDB7FEB709
:109C8000D283C183548243820E940A530F900F9063
:109C90000F900F90459A4598112351F600D000D0AF
:109CA00080E290E0ADB7BEB712969C938E93119769
:109CB00083EE97E014969C938E9313970E940A5319
:109CC000469A46984298429A0F900F900F900F90A4
:109CD000DF91CF911F91FF90EF90DF90CF90BF90D9
:109CE000AF909F908F907F906F905F904F9008956E
:109CF000DF92EF92FF920F931F937B018C01D42E82
:109D00008DB79EB70A970FB6F8949EBF0FBE8DBF52
:109D1000EDB7FEB7319680E190E0ADB7BEB71296D1
:109D20009C938E93119786EE96E093838283E482D0
:109D3000F58206831783408711860E940A538FEFAE
:109D400081B92898299A2A9A8DB79EB70A960FB694
:109D5000F8949EBF0FBE8DBFC801B7010E94D24DBF
:109D60002998D2B8299A00000000000000000000E5
:109D70000000289A11B812B81F910F91FF90EF9030
:109D8000DF900895EF92FF920F931F937B018C0158
:109D90008DB79EB708970FB6F8949EBF0FBE8DBFC4
:109DA000EDB7FEB7319688E090E0ADB7BEB712963A
:109DB0009C938E9311978EE197E093838283E48244
:109DC000F582068317830E940A53E0923302F092D1
:109DD000340200933502109336028FEF81B9289830
:109DE000299A2A9A8DB79EB708960FB6F8949EBF07
:109DF0000FBE8DBFC801B7010E94D24D29981F9197
:109E00000F91FF90EF9008957F928F929F92AF9263
:109E1000BF92CF92DF92EF92FF920F931F93CF9357
:109E2000DF93162FB72EA82E992E69017A01702E76
:109E30008DB79EB70C970FB6F8949EBF0FBE8DBF1F
:109E4000EDB7FEB7319688E090E0ADB7BEB7129699
:109E50009C938E93119788E496E093838283648326
:109E60007583A682978220873187428753870E9415
:109E70000A538DB79EB70C960FB6F8949EBF0FBECF
:109E80008DBF612F7B2D8A2D992D0E94C24E812F6F
:109E90009B2DAA2DB92D4C015D01C80CD91CEA1CC3
:109EA000FB1C08E010E0CAE2D6E049C0C501B401DD
:109EB0002FEF3FE040E050E00E949E676115710582
:109EC00081059105F9F4ADB7BEB718970FB6F894B0
:109ED000BEBF0FBEADBFEDB7FEB7319612961C9355
:109EE0000E931197D383C28384829582A682B78210
:109EF0000E940A538DB79EB708960FB6F8949EBF7E
:109F00000FBE8DBF72B88091330290913402A09140
:109F10003502B09136020196A11DB11D8093330226
:109F200090933402A0933502B0933602299A409858
:109F3000409A29980894811C911CA11CB11C8C1476
:109F40009D04AE04BF0408F4B1CF0E946E4DDF91B2
:109F5000CF911F910F91FF90EF90DF90CF90BF9026
:109F6000AF909F908F907F9008958F929F92AF9225
:109F7000BF92CF92DF92EF92FF920F931F93D62E54
:109F8000C72EB82EA92E942E852E780189018DB763
:109F90009EB70E970FB6F8949EBF0FBE8DBFEDB75C
:109FA000FEB7319688E090E0ADB7BEB712969C93AD
:109FB0008E9311978AEA96E09383828364837583F4
:109FC000B682A78240875187E286F3860487158789
:109FD0000E940A538DB79EB70E960FB6F8949EBF97
:109FE0000FBE8DBF6D2D7C2D8B2D9A2D0E94C24EE4
:109FF0008D2D9C2DAB2DBA2DAC01BD01292D382DF9
:10A00000C901FC0198018701040F151F261F371F86
:10A010001DC0819182B98091330290913402A09148
:10A020003502B09136020196A11DB11D8093330215
:10A0300090933402A0933502B0933602299A409847
:10A04000409A29984F5F5F4F6F4F7F4F40175107DE
:10A0500062077307F0F20E946E4D1F910F91FF90FF
:10A06000EF90DF90CF90BF90AF909F908F9008952A
:10A070008DB79EB708970FB6F8949EBF0FBE8DBFE1
:10A08000EDB7FEB7319688E090E0ADB7BEB7129657
:10A090009C938E93119788E997E0938382838091B4
:10A0A000370290913802A0913902B0913A0284832C
:10A0B0009583A683B7830E940A538DB79EB70896EF
:10A0C0000FB6F8949EBF0FBE8DBF6091370270919E
:10A0D00038028091390290913A020E94C24E08954E
:10A0E000EF92FF920F931F937B018C018DB79EB768
:10A0F00008970FB6F8949EBF0FBE8DBFEDB7FEB7A1
:10A10000319680E190E0ADB7BEB712969C938E93E6
:10A11000119784E497E093838283E482F582068337
:10A1200017830E940A5311B812B82898299A2A9ABC
:10A130008DB79EB708960FB6F8949EBF0FBE8DBF21
:10A14000C801B7010E94D24D2A980000000000000B
:10A1500000000000000080B12A9A289A11B812B8B5
:10A160001F910F91FF90EF900895EF92FF920F9340
:10A170001F937B018C018DB79EB708970FB6F8949B
:10A180009EBF0FBE8DBFEDB7FEB7319688E090E061
:10A19000ADB7BEB712969C938E93119783E797E065
:10A1A00093838283E482F582068317830E940A5395
:10A1B000E0923302F092340200933502109336029B
:10A1C00011B812B82898299A2A9A8DB79EB708967E
:10A1D0000FB6F8949EBF0FBE8DBFC801B7010E9495
:10A1E000D24D2A980000000000000000000000008E
:10A1F0001F910F91FF90EF9008958F929F92AF92D1
:10A20000BF92CF92DF92EF92FF920F931F93CF9363
:10A21000DF93D62EC72EB82EA92E942E852E780128
:10A2200089018DB79EB70E970FB6F8949EBF0FBEEB
:10A230008DBFEDB7FEB7319688E090E0ADB7BEB701
:10A2400012969C938E9311978EE696E09383828369
:10A2500064837583B682A78240875187E286F3863E
:10A26000048715870E940A538DB79EB70E960FB6C6
:10A27000F8949EBF0FBE8DBF6D2D7C2D8B2D9A2D1A
:10A280000E94B5508D2D9C2DAB2DBA2D5C016D011A
:10A29000292D382DC901EC01EA0CFB1C0C1D1D1DDC
:10A2A00009C080B189930E94344D0894A11CB11C4F
:10A2B000C11CD11CAE14BF04C006D10690F30E948D
:10A2C000854DDF91CF911F910F91FF90EF90DF901F
:10A2D000CF90BF90AF909F908F900895362F20E041
:10A2E0002827392780E090E061E270E1A901440F5E
:10A2F000551F37FF04C09A012627372701C09A014E
:10A3000001968830910591F7C90108950F931F9325
:10A31000CF93DF93EC0120E030E080E090E001E2B9
:10A3200010E119C0FE01E80FF91FF081E0E02E27CF
:10A330003F2740E050E0D901AA0FBB1F37FF04C000
:10A340009D012027312701C09D014F5F5F4F48309D
:10A35000510589F701968617970720F3C901DF9108
:10A36000CF911F910F9108950F931F93CF93DF9378
:10A370009C01EB01BA0140E050E001E210E119C09C
:10A38000FE01E40FF51FF081E0E02E273F2780E07B
:10A3900090E0D901AA0FBB1F37FF04C09D01202701
:10A3A000312701C09D0101968830910591F74F5FDB
:10A3B0005F4F4617570720F3C901DF91CF911F91D7
:10A3C0000F9108958F929F92AF92BF92CF92DF929A
:10A3D000EF92FF920F931F93CF93DF936B017C015A
:10A3E00049015A01E801860E971EA81EB91E09C030
:10A3F000C701B601AE0100E010E020E030E00E94AD
:10A40000FD50C814D904EA04FB0490F380E090E006
:10A41000DF91CF911F910F91FF90EF90DF90CF9040
:10A42000BF90AF909F908F9008952F923F924F9240
:10A430005F926F927F928F929F92AF92BF92CF92D4
:10A44000DF92EF92FF920F931F93CF93DF93D62E5D
:10A45000C72EB82EA92E39014A01170128010E94E2
:10A46000B5508DB79EB70C970FB6F8949EBF0FBE30
:10A470008DBFEDB7FEB7319680E490E0ADB7BEB7C3
:10A4800012969C938E93119788E798E0938382832A
:10A49000D482C582B682A7826086718682869386C0
:10A4A0000E940A532D2D3C2D4B2D5A2DC901DA0146
:10A4B0005C016D01C0E0D0E0FF248DB79EB70C9623
:10A4C0000FB6F8949EBF0FBE8DBF58C0A114B10443
:10A4D000C104D104A9F1C601B501A20191010E94F4
:10A4E0009E67611571058105910551F5ADB7BEB740
:10A4F0001C970FB6F894BEBF0FBEADBFEDB7FEB749
:10A50000319680E490E012969C938E931197ACE381
:10A51000B8E0B383A283F4821582A682B782C08694
:10A52000D186D387C2870E940A53F394C0E0D0E05B
:10A530008DB79EB70C960FB6F8949EBF0FBE8DBF19
:10A540000E94524D182F00E0C027D12780E090E0F4
:10A550009E01220F331FD7FF05C0C1E2D0E1C22701
:10A56000D32701C0E90101968830910589F70E943F
:10A57000344D0894A11CB11CC11CD11CA614B704F5
:10A58000C804D90408F4A2CFD601C5019F77A070F2
:10A59000B0700097A105B10539F5ADB7BEB71C97EE
:10A5A0000FB6F894BEBF0FBEADBFEDB7FEB7319684
:10A5B00080E490E012969C938E93119780E098E04F
:10A5C00093838283F4821582A682B782C086D18665
:10A5D000D387C2870E940A538DB79EB70C960FB6D9
:10A5E000F8949EBF0FBE8DBF0E94854DCE01DF91B6
:10A5F000CF911F910F91FF90EF90DF90CF90BF9080
:10A60000AF909F908F907F906F905F904F903F9012
:10A610002F900895DF93CF93CDB7DEB78D819E81C4
:10A6200020910A0130910B0182239323892B81F021
:10A630008EE992E06F81788540E051E00E94BF662C
:10A640009E01275F3F4F8EE992E0B9010E94176794
:10A65000CF91DF910895DF93CF93CDB7DEB78D8192
:10A660009E8120910A0130910B0182239323892B33
:10A6700041F09E01275F3F4F8F819885B9010E946D
:10A680001767CF91DF9108952F923F924F925F927B
:10A690006F927F928F929F92AF92BF92CF92DF92F2
:10A6A000EF92FF920F931F93CF93DF931B012C0127
:10A6B00039014A016801AA24BB2490E0AFC0F60129
:10A6C00040E050E020E030E08191280F311D4F5FE5
:10A6D0005F4F40315105C1F7232B11F491E098C031
:10A6E000992369F000D0EDEDF8E0ADB7BEB7129652
:10A6F000FC93EE9311970E9430560F900F9000D06C
:10A7000000D000D0E6EDF8E0ADB7BEB71296FC93EE
:10A71000EE931197E20CF31C041D151D1396ED9298
:10A72000FD920D931C9316970E943056E60100E0AF
:10A7300010E0EDB7FEB736960FB6F894FEBF0FBE29
:10A74000EDBF00D000D0EDB7FEB7319620ED38E078
:10A75000ADB7BEB712963C932E9311978991828321
:10A7600013820E9430560F5F1F4F0F900F900F9073
:10A770000F900031110529F700D0EDECF8E0ADB7EE
:10A78000BEB71296FC93EE9311970E943056E601E5
:10A7900000E010E00F900F909881892F81528E3544
:10A7A000B0F400D000D0EDB7FEB731962AEC38E017
:10A7B000ADB7BEB712963C932E9311979283138236
:10A7C0000E9430560F900F900F900F900DC000D048
:10A7D000E8ECF8E0ADB7BEB71296FC93EE93119794
:10A7E0000E9430560F900F900F5F1F4F219600313F
:10A7F000110591F600D0E5ECF8E0ADB7BEB71296C2
:10A80000FC93EE9311970E94305690E00F900F90BA
:10A8100020E130E0A20EB31EC20ED31E750100E08F
:10A8200010E0E614F7040805190508F448CFDF9195
:10A83000CF911F910F91FF90EF90DF90CF90BF903D
:10A84000AF909F908F907F906F905F904F903F90D0
:10A850002F9008956F927F928F929F92AF92BF92A6
:10A86000CF92DF92EF92FF920F931F93CF93DF93DC
:10A87000162F072FF82EE92E49015A010E94B550D4
:10A88000212F302F4F2D5E2DC901DA016C017D0182
:10A890008DEB682E88E0782EC7EBD8E040C0D7015A
:10A8A000C6018F709070A070B0700097A105B105BF
:10A8B000C9F400D000D000D0ADB7BEB712967C92DC
:10A8C0006E921197EDB7FEB7C382D482E582F6820D
:10A8D0000E9430568DB79EB706960FB6F8949EBF6D
:10A8E0000FBE8DBF0E94524D182F0E94344D00D0D4
:10A8F00000D0EDB7FEB73196ADB7BEB71296DC9378
:10A90000CE931197128313820E9430560894C11C73
:10A91000D11CE11CF11C0F900F900F900F90C814E8
:10A92000D904EA04FB0408F4BACF00D085EB98E020
:10A93000EDB7FEB7928381830E9430560F900F903F
:10A940000E94854DDF91CF911F910F91FF90EF9065
:10A95000DF90CF90BF90AF909F908F907F906F903F
:10A9600008951F920F920FB60F9211248F939F9309
:10A9700080919E0390919F03019790939F038093F2
:10A980009E03892B79F484EF91E090939F03809349
:10A990009E038091A0039091A10301969093A1033F
:10A9A0008093A0039F918F910F900FBE0F901F90E7
:10A9B000189589E0809381008FE39CE9909389004A
:10A9C0008093880010928500109284001092A10359
:10A9D0001092A00384EF91E090939F0380939E03D5
:10A9E00082E080936F00789408950F931F930091F5
:10A9F000A0031091A10320919E0330919F0340E09A
:10AA000050E064EF71E080E090E0621B730B840B18
:10AA1000950B24EF31E040E050E00E94C067020F48
:10AA2000131FC8011F910F9108954F925F926F926B
:10AA30007F928F929F92AF92BF92CF92DF92EF92CE
:10AA4000FF920F931F93CF93DF933C016A017B0129
:10AA5000480159012DB73EB72A5030400FB6F8943F
:10AA60003EBF0FBE2DBFEDB7FEB7319682E199E034
:10AA7000ADB7BEB712969C938E93119742835383C2
:10AA80006483758386829782A086B1860E94305641
:10AA9000EDB7FEB73A960FB6F894FEBF0FBEEDBF06
:10AAA000C501B4010E94C24E870176010894E108F5
:10AAB000F1080109110917FDC1C0F894E3012196BD
:10AAC000F30184917894803931F50894E108F10814
:10AAD00001091109FFEFEF16FFEFFF06FFEF0F0768
:10AAE000FFEF1F0709F4AAC0F894FE01849178943F
:10AAF000882379F000D086EF98E0ADB7BEB7129604
:10AB00009C938E9311970E94305681E00F900F9086
:10AB100096C0219680E90E946C4D0E94544D6501BB
:10AB200054010894A11CB11CC11CD11C772494EFC2
:10AB3000492E98E0592E5CC00894E108F1080109FB
:10AB40001109F894FE01219694907894D801C701D8
:10AB50009370A070B0700097A105B10549F400D0C2
:10AB6000EDB7FEB7528241820E9430560F900F908F
:10AB7000F0E99F1691F50894E108F108010911091F
:10AB80002FEFE2162FEFF2062FEF02072FEF12073B
:10AB900009F454C0F894FE0121968490789488209A
:10ABA00011F0982C12C080E90E946C4D0E94544D07
:10ABB0000894A11CB11CC11CD11C80E9782E18C0BE
:10ABC000872D0E946C4D0E94544D9A94C9F78A9427
:10ABD000A80CB11CC11CD11C0BC0892D0E946C4D4E
:10ABE0000E94544D0894A11CB11CC11CD11C792C8D
:10ABF0001E141F04100611060CF49ECF0E946E4D09
:10AC000000D000D000D080EE98E0ADB7BEB712966D
:10AC10009C938E931197EDB7FEB7A382B482C58241
:10AC2000D6820E94305680E02DB73EB72A5F3F4F54
:10AC30000FB6F8943EBF0FBE2DBF01C081E0DF917B
:10AC4000CF911F910F91FF90EF90DF90CF90BF9029
:10AC5000AF909F908F907F906F905F904F900895EE
:10AC6000EF92FF920F931F93DF93CF93CDB7DEB791
:10AC70008E01075F1F4FF801619171918F0182EA88
:10AC8000E82E83E0F82EC70140E051E00E94BF6645
:10AC9000C701B8010E941767CF91DF911F910F91F3
:10ACA000FF90EF900895DF93CF93CDB7DEB7FE010D
:10ACB000359681919191BF010E941767CF91DF91E5
:10ACC000089581E080931A0180931B0108955E9896
:10ACD0005F985D9A2098289A88EC90E024EF31E004
:10ACE000F9013197F1F70197D9F75D985E9A209AAB
:10ACF0005E9A5F98089560E070E080E090E00E94C6
:10AD000070508093A20461E070E080E090E00E94C7
:10AD100070508093A60662E070E080E090E00E94B0
:10AD200070508093A40608950F931F930E949C4D2A
:10AD300000D000D080E890E0EDB7FEB79283818329
:10AD40008FEA93E8948383830E940A530F900F90B5
:10AD50000F900F9060E070E180E090E043EA55E0F2
:10AD600000E011E020E030E00E94FD500E943850E9
:10AD700010921A011F910F9108950F931F930E9433
:10AD80009C4D00D000D080E890E0EDB7FEB79283F4
:10AD9000818380EE93E8948383830E940A530F900B
:10ADA0000F900F900F9060E070E080E090E043EA39
:10ADB00054E000E011E020E030E00E94FD500E94ED
:10ADC000385010921B011F910F9108959B01AC0107
:10ADD000213081E0380780E0480780E0580750F1D3
:10ADE00080911B01882331F1ADB7BEB718970FB61C
:10ADF000F894BEBF0FBEADBFEDB7FEB7319680E889
:10AE000090E012969C938E93119784E594E8938337
:10AE1000828324833583468357830E940A538DB7E8
:10AE20009EB708960FB6F8949EBF0FBE8DBF0E94C6
:10AE3000BD5631C0213091E1390790E0490790E0DB
:10AE4000590758F180911A01882339F1ADB7BEB77F
:10AE500018970FB6F894BEBF0FBEADBFEDB7FEB7E3
:10AE6000319680E890E012969C938E93119781E141
:10AE700094E89383828324833583468357830E9497
:10AE80000A538DB79EB708960FB6F8949EBF0FBEB3
:10AE90008DBF0E94945680E0089581E00895EF925E
:10AEA000FF920F931F93CF93DF93EC018B017A01F5
:10AEB00080911A018823C9F000D000D080E890E08A
:10AEC000ADB7BEB712969C938E93119788ED92E81A
:10AED00014969C938E9313970E940A5321E030E0BE
:10AEE0000F900F900F900F9077C00E949C4D60E0E4
:10AEF00070E180E090E00E947050853A29F00E9455
:10AF0000385021E030E068C061E070E180E090E01E
:10AF10000E947050888362E070E180E090E00E94BF
:10AF20007050F80180832DB73EB72C5030400FB6DB
:10AF3000F8943EBF0FBE2DBFEDB7FEB7319620E8A7
:10AF400030E0ADB7BEB712963C932E93119726EA28
:10AF500032E83383228321E030E1358324839881F2
:10AF60009683178222E030E131872087828713861B
:10AF70000E940A53EDB7FEB73C960FB6F894FEBF99
:10AF80000FBEEDBFD8010C9110E020E030E063E08F
:10AF900070E180E090E0A7010E94FD5060E070E168
:10AFA00080E090E04AE50E94784E5E985F985D9A56
:10AFB0002098289A88EC90E024EF31E0F90131974D
:10AFC000F1F70197D9F75D985E9A209A5E9A5F989B
:10AFD0000E94385020E030E0C901DF91CF911F91ED
:10AFE0000F91FF90EF9008956EEF7FEF80E090E07B
:10AFF0004091A3060E94784E6FEF7FEF80E090E0D3
:10B000004091A5060E94784E08956EEF7FEF80E094
:10B0100090E00E9470508093A3066FEF7FEF80E076
:10B0200090E00E9470508093A50664EE7FEF80E070
:10B0300090E040E00E94784E65EE7FEF80E090E087
:10B0400040E00E94784E089560E070E080E090E07B
:10B050004091A2040E94784E61E070E080E090E0B0
:10B060004091A6060E94784E62E070E080E090E099
:10B070004091A4060E94784E08950F931F93182FB5
:10B08000062F80911B018823B1F000D000D080E80A
:10B0900090E0ADB7BEB712969C938E9311978DE258
:10B0A00093E814969C938E9313970E940A530F90E3
:10B0B0000F900F900F90EDB7FEB73C970FB6F89436
:10B0C000FEBF0FBEEDBF319680E890E0ADB7BEB7D2
:10B0D00012969C938E93119789EF92E893838283C3
:10B0E00081E090E0958384831683178282E090E06C
:10B0F00091878087028713860E940A53EDB7FEB7B7
:10B100003C960FB6F894FEBF0FBEEDBF0E949C4D5B
:10B110000E947B560E94055860E070E080E090E05D
:10B1200045EA0E94784E61E070E080E090E0412FB7
:10B130000E94784E62E070E080E090E0402F0E9434
:10B14000784E5E985F985D9A2098289A88EC90E0F7
:10B1500024EF31E0F9013197F1F70197D9F75D98C4
:10B160005E9A209A2B9823985E9A5F980E942458A2
:10B170000E94F4570E9438501F910F9108950F9329
:10B180001F9380911A01882309F500D000D080E830
:10B1900090E0EDB7FEB7928381838EE493E89483C9
:10B1A00083830E940A530F900F900F900F9060E0DE
:10B1B00070E180E090E043EA55E000E011E020E03B
:10B1C00030E00E94B54F81E080931A011F910F91EA
:10B1D00008950F931F9380911B01882309F500D0D8
:10B1E00000D080E890E0EDB7FEB7928381838DE7D1
:10B1F00093E8948383830E940A530F900F900F90DB
:10B200000F9060E070E080E090E043EA54E000E0FE
:10B2100011E020E030E00E94B54F81E080931B01F7
:10B220001F910F910895F894E3E7F0E08081886022
:10B230008083E8E6F0E080818860808378940895D8
:10B24000F894E3E7F0E08081877F80837894089525
:10B25000F894549A28E088E190E00FB6F894A89505
:10B26000809360000FBE20936000FFCF1F920F926B
:10B270000FB60F9211242F933F934F935F936F93C9
:10B280007F938F939F93AF93BF93EF93FF934B99CC
:10B2900021C000D088EA94E8EDB7FEB7928381839D
:10B2A0000E94305687E994E8EDB7FEB79283818318
:10B2B0000E943056F894549A28E088E190E00FB646
:10B2C000F894A895809360000FBE209360000F90C3
:10B2D0000F90FFCFFF91EF91BF91AF919F918F9111
:10B2E0007F916F915F914F913F912F910F900FBE82
:10B2F0000F901F901895239A2B9885E88A95F1F75F
:10B300002B9A239808958091980290919902A09188
:10B310009A02B0919B0280509048A040B04029F41E
:10B320005E9A00D082ED94E804C05E9800D081EC73
:10B3300094E8EDB7FEB7928381830E9430560F9058
:10B340000F90089500D084EE94E8EDB7FEB7928395
:10B3500081830E943056F894539A5B9880E197E27B
:10B360000197F1F75B9A539878940F900F90089596
:10B370002F923F924F925F926F927F928F929F9205
:10B38000AF92BF92CF92DF92EF92FF920F931F93F3
:10B39000DF93CF9300D000D0CDB7DEB769837A8337
:10B3A0008B839C8339014A01170128018DB79EB711
:10B3B0000A970FB6F8949EBF0FBE8DBFEDB7FEB7CC
:10B3C000319680EE95E8ADB7BEB712969C938E93FA
:10B3D0001197B981B2838A8183839B819483AC81E5
:10B3E000A58326833783408751870E943056EDB767
:10B3F000FEB73A960FB6F894FEBF0FBEEDBF698157
:10B400007A818B819C810E94C24E29813A814B8135
:10B410005C81C901DA017C018D0195E5D92E87EAAD
:10B42000A82E85E8B82E35C0C801B701A201910148
:10B430000E949E67611571058105910511F5D394F0
:10B440008DB79EB708970FB6F8949EBF0FBE8DBFFD
:10B45000EDB7FEB73196ADB7BEB71296BC92AE92BD
:10B460001197E282F38204831583D68217820E94A9
:10B470003056EDB7FEB738960FB6F894FEBF0FBE44
:10B48000EDBF8D2D0E946C4D0894E11CF11C011D37
:10B49000111DE614F7040805190530F20E946E4DDF
:10B4A00029813A814B815C81C901DA015C016D011E
:10B4B0003EC086017501E20CF31C041D151D8DB7FD
:10B4C0009EB70A970FB6F8949EBF0FBE8DBFEDB71B
:10B4D000FEB7319687E695E8ADB7BEB712969C9356
:10B4E0008E931197A282B382C482D582E682F782BC
:10B4F000008711870E943056ADB7BEB71A960FB6B7
:10B50000F894BEBF0FBEADBFC601B501A80197013B
:10B510000E942A5400D085E295E8EDB7FEB79283E9
:10B5200081830E943056570168010F900F90A61436
:10B53000B704C804D90408F4BCCF69817A818B812F
:10B540009C81A4019301820171010E9415520F9008
:10B550000F900F900F90CF91DF911F910F91FF905F
:10B56000EF90DF90CF90BF90AF909F908F907F90A3
:10B570006F905F904F903F902F900895AF92BF9241
:10B58000CF92DF92EF92FF920F931F93CF93DF93AF
:10B59000162F072FF82EE92E59016A010E94B55087
:10B5A000212F302F4F2D5E2DC901DA017C018D0135
:10B5B000CBE1D6E82EC00E94524D8F3F19F12DB736
:10B5C0003EB7285030400FB6F8943EBF0FBE2DBF97
:10B5D000EDB7FEB73196ADB7BEB71296DC93CE93FA
:10B5E0001197E282F38204831583868317820E9477
:10B5F00030562DB73EB7285F3F4F0FB6F8943EBF89
:10B600000FBE2DBF0E94344D0894E11CF11C011D9A
:10B61000111DEA14FB040C051D0568F20E94854DFE
:10B62000DF91CF911F910F91FF90EF90DF90CF901E
:10B63000BF90AF900895EF92FF920F931F9300D0A9
:10B6400084E195E8EDB7FEB7928381830E9430567E
:10B650005D985E9A209A0F900F9060E070E080E015
:10B6600090E02FEF3FEF48E050E00FEF0E94044FD3
:10B6700000D085E095E8EDB7FEB7928381830E9404
:10B6800030560F900F9060E070E080E090E02FEF78
:10B690003FEF48E050E0E12CE0E8FE2E012D112DB7
:10B6A0000E94155200D084EF94E8EDB7FEB7928364
:10B6B00081830E9430560F900F9060E070E080E030
:10B6C00090E02FEF3FEF48E050E00E94BE5A00D0DC
:10B6D00080EF94E8EDB7FEB7928381830E943056E5
:10B6E0000F900F901F910F91FF90EF900895EF92A0
:10B6F000FF920F931F93CF93DF935D985E9A209AEA
:10B7000060E070E080E090E00E94C24E00E010E057
:10B7100004C00E946C4D0E94544D802F0F5F1F4F3C
:10B7200020E802301207A9F70E946E4D60E070E039
:10B7300080E090E00E94B550EE24FF248701C0E332
:10B74000D6E80E94524DADB7BEB718970FB6F89421
:10B75000BEBF0FBEADBFEDB7FEB731961296DC93FC
:10B76000CE931197E282F382048315838683178236
:10B770000E9430562DB73EB7285F3F4F0FB6F89462
:10B780003EBF0FBE2DBF0E94344D0894E11CF11C3A
:10B79000011D111D31E0E31630E8F30630E0030728
:10B7A00030E0130771F60E94854DDF91CF911F9114
:10B7B0000F91FF90EF900895EF92FF920F931F93D8
:10B7C000CF93DF935D985E9A209AF1E0EF2EF12CF3
:10B7D000012D112D0AC0C801B7014E2D0E94784ECF
:10B7E0000894E11CF11C011D111D21E0E21621E06D
:10B7F000F20620E0020720E0120769F7EE24FF249A
:10B800008701C1E4D6E80894E11CF11C011D111D5B
:10B81000C801B7010E947050ADB7BEB718970FB6F8
:10B82000F894BEBF0FBEADBFEDB7FEB7319612960E
:10B83000DC93CE931197E282F3820483158386838F
:10B8400017820E9430562DB73EB7285F3F4F0FB684
:10B85000F8943EBF0FBE2DBF30E0E31631E0F30693
:10B8600030E0030730E0130771F6DF91CF911F91AD
:10B870000F91FF90EF900895A1E1B0E0E2E4FCE5C4
:10B880000C94DB673C017F876E876A01FC0117829D
:10B890001682838181FD03C06FEF7FEF71C39E012C
:10B8A0002F5F3F4F398B288BF3012381EE85FF8576
:10B8B00023FD859123FF8191FF87EE87882309F47B
:10B8C0005CC3853251F4EE85FF8523FD859123FF0E
:10B8D0008191FF87EE87853229F490E0B3010E94C1
:10B8E000EB66E2CF982F10E0882499241032B0F450
:10B8F0009B3269F09C3228F4903251F0933271F40B
:10B900000BC09D3239F0903349F4116028C01260A9
:10B91000146025C0186023C0106121C017FD2AC023
:10B92000892F80538A3078F416FF06C0FAE09F9E74
:10B93000902C1124980E13C03AE0839E802C112481
:10B94000880E10620CC09E3221F416FD16C31064DE
:10B9500006C09C3611F4106802C0983659F4EE8582
:10B96000FF8523FD959123FF9191FF87EE87992312
:10B9700009F0BCCF892F8554833020F4812F80615A
:10B98000905E07C0892F8556833008F0A1C1812FB2
:10B990008F7E86FD02C076E0972E6FE3F62EF822AA
:10B9A000953619F4F0E4FF2A07C0963619F420E81A
:10B9B000F22A02C091109A94F7FE0BC03BE33915AE
:10B9C00020F427E05CE3B52E0EC0B92CB39427E039
:10B9D0000AC047E0491528F427E0BB2447E0942E2D
:10B9E00002C0292DBB24C60104969D878C87F601D1
:10B9F0006081718182819381AE014F5F5F4F0B2D1A
:10BA00000E94E7656C010981202E332400FF04C0E9
:10BA100003FD02C01DE209C0F1FE02C01BE205C029
:10BA2000F2FC02C010E001C010E2C1018C70907005
:10BA3000892BB9F1112311F483E001C084E088154A
:10BA400010F088240AC0881AF3FC07C080E290E056
:10BA5000B3010E94EB668A94C9F7112329F0812F64
:10BA600090E0B3010E94EB6623FE03C007E516E8F1
:10BA70000EC00BE516E80BC0E114F10409F080528A
:10BA800090E0B3010E94EB660F5F1F4F05C0EF2CE3
:10BA9000FF24F0E1EF22FF24F8018491882361F76D
:10BAA00014C1F7FE12C0BC0C24FE04C08A8181338D
:10BAB00009F4BA941B141CF0BB24B3942DC0F8E015
:10BAC000FB1550F538E0B32E27C0F6FC25C0892DB4
:10BAD00090E08C159D054CF02CEFC2162FEFD2068E
:10BAE00024F030E8F32A01C09A94992049F0E2E06A
:10BAF000F0E0EC0FFD1FE90DF11D80818033A1F313
:10BB0000F7FE0AC0B92CB394892D90E0C816D90667
:10BB100014F0992401C09C18F7FC03C025E030E024
:10BB200009C01C141D041CF021E030E003C0960184
:10BB30002F5F3F4F112311F02F5F3F4F992029F0C6
:10BB4000892D90E00196280F391F882D90E0281745
:10BB5000390714F0882401C0821A4F2C5524C201E1
:10BB600089709070892B39F008C080E290E0B301B1
:10BB70000E94EB668A948820C1F7112329F0812F57
:10BB800090E0B3010E94EB6643FE07C008C080E36B
:10BB900090E0B3010E94EB668A948820C1F7F7FE1B
:10BBA00046C08601D7FE02C000E010E0760108948E
:10BBB000E11CF11CE01AF10A41E050E04C0F5D1F5E
:10BBC000E40EF51E26014B185108892D90E0AA2499
:10BBD000BB24A81AB90A5FEF0F3F150729F48EE2BC
:10BBE00090E0B3010E94EB66C016D10634F0401617
:10BBF00051061CF4F701808101C080E30150104020
:10BC00000894E11CF11C0A151B052CF090E0B3010F
:10BC10000E94EB66E0CF0C151D0539F49A8196332E
:10BC200018F4953311F424FE81E390E04BC08A812F
:10BC3000813309F00F7E90E0B3010E94EB669920FA
:10BC4000A1F08EE290E0B3010E94EB6612E0E1E029
:10BC5000F0E0EC0FFD1FE10FF11D1F5F808190E010
:10BC6000B3010E94EB669A9491F744FC03C085E609
:10BC700090E002C085E490E0B3010E94EB66D7FC3F
:10BC800005C0C114D10441F404FF06C0D094C1948E
:10BC9000D108D3948DE201C08BE290E0B3010E9401
:10BCA000EB6680E305C08F5F26EF3FEFC20ED31E29
:10BCB0003AE0C316D104BCF790E0B3010E94EB66F2
:10BCC000C601C096B3010E94EB66CC84DD8452C1EC
:10BCD000933631F0933799F0933509F059C023C06A
:10BCE000F601808189835E010894A11CB11C22E0C9
:10BCF00030E0C20ED31E21E0E22EF12C12C0F6017C
:10BD0000A080B18016FD03C06FEF7FEF02C0692DE8
:10BD100070E022E030E0C20ED31EC5010E94E06652
:10BD20007C011F7713C0F601A080B18016FD03C00F
:10BD30006FEF7FEF02C0692D70E022E030E0C20EAD
:10BD4000D31EC5010E94D5667C01106813FF07C091
:10BD50001BC080E290E0B3010E94EB668A94882DBC
:10BD600090E0E816F906A8F30FC0F50117FD8591DC
:10BD700017FF81915F0190E0B3010E94EB66811093
:10BD80008A940894E108F108E114F10471F7F2C013
:10BD9000943611F0993689F517FF08C0F601208115
:10BDA00031814281538184E090E00AC0F6018081B4
:10BDB00091819C01442737FD4095542F82E090E00B
:10BDC000C80ED91E9FE6F92EF12257FF09C05095E3
:10BDD0004095309521953F4F4F4F5F4F90E8F92A9E
:10BDE000CA01B901AE014F5F5F4F2AE030E00E9407
:10BDF0002167E82EE889EE1A41C0953721F41F7EAD
:10BE00002AE030E01CC0197F9F3661F0903720F4A3
:10BE1000983509F0B2C00FC0903739F0983709F063
:10BE2000ACC004C028E030E00AC0106114FD14600A
:10BE300020E130E004C014FD166020E132E017FF7D
:10BE400008C0F601608171818281938144E050E0F5
:10BE500008C0F60180819181BC0180E090E042E061
:10BE600050E0C40ED51EAE014F5F5F4F0E942167A8
:10BE7000E82E5889E51A8FE7F82EF122F6FE0BC05E
:10BE80008EEFF822E91438F4F4FE07C0F2FC05C086
:10BE90009FEEF92202C01E2D01C0192DF4FE0DC027
:10BEA000FE01EE0DF11D8081803319F4E9EEFE22D2
:10BEB00008C01F5FF2FE05C003C08F2D867809F011
:10BEC0001F5F0F2DF3FC14C0F0FE0FC0181510F00B
:10BED0009E2C0BC09E2C980C911A182D06C080E247
:10BEE00090E0B3010E94EB661F5F1815C0F304C019
:10BEF000181510F4811A01C0882404FF0FC080E3D4
:10BF000090E0B3010E94EB6602FF1DC001FD03C07B
:10BF100088E790E00EC088E590E00BC0802F86781F
:10BF200091F001FF02C08BE201C080E2F7FC8DE2DC
:10BF300090E0B3010E94EB6606C080E390E0B3019D
:10BF40000E94EB669A94E914C0F3EA94E1E0F0E011
:10BF5000EC0FFD1FEE0DF11D808190E0B3010E94FA
:10BF6000EB66EE2091F706C080E290E0B3010E94FC
:10BF7000EB668A948820C1F797CCF30166817781BC
:10BF8000CB016196E2E10C94F767EF92FF920F9379
:10BF90001F937B018C0120E030E040E05FE40E94D1
:10BFA000C56288238CF0C801B70120E030E040E092
:10BFB0005FE40E943D610E9425639B01AC0120501B
:10BFC00030404040504806C0C801B7010E94256378
:10BFD0009B01AC01B901CA011F910F91FF90EF9035
:10BFE0000895A0E0B0E0E7EFFFE50C94DB67DC012B
:10BFF0002B01FA019C91923008F439C1EB01888140
:10C00000823008F433C1943069F4843009F02FC1D0
:10C0100011969C9111978981981709F428C1ACE178
:10C02000B1E025C1843009F421C18230A9F49230F5
:10C0300009F01DC19A01AD0188E0EA010990AE0145
:10C04000E90109929E018150C1F7E20189811196AF
:10C050009C918923818308C1923009F407C112960B
:10C060002D903C901397EB018A819B811496AD90A3
:10C07000BD90CD90DC901797EC80FD800E811F81E4
:10C080009101281B390BB90137FF04C066277727B8
:10C09000621B730B603271050CF061C0121613063F
:10C0A0006CF537014801062E04C096948794779466
:10C0B00067940A94D2F721E030E040E050E004C0F9
:10C0C000220F331F441F551F6A95D2F7215030406D
:10C0D000404050402E213F2140235123211531055E
:10C0E0004105510521F021E030E040E050E07901C8
:10C0F0008A01E628F728082919293CC0232BD1F109
:10C10000260E371E35014601062E04C096948794EC
:10C11000779467940A94D2F721E030E040E050E051
:10C1200004C0220F331F441F551F6A95D2F72150B8
:10C130003040404050402A213B214C215D212115B7
:10C1400031054105510521F021E030E040E050E0AB
:10C1500059016A01A628B728C828D9280BC082151A
:10C1600093052CF01C01AA24BB24650103C0EE2416
:10C17000FF24870111969C91D20111968C919817FA
:10C1800009F445C0992339F0A80197012A193B0900
:10C190004C095D0906C0A60195012E193F09400B07
:10C1A000510B57FD08C011823382228224833583CC
:10C1B000468357831DC081E0818333822282882792
:10C1C0009927DC01821B930BA40BB50B8483958309
:10C1D000A683B7830DC0220F331F441F551F24832E
:10C1E000358346835783828193810197938382832A
:10C1F0002481358146815781DA01C9010197A1095E
:10C20000B1098F5F9F4FAF4FBF4328F30BC091839E
:10C2100033822282EA0CFB1C0C1D1D1DE482F58278
:10C220000683178383E0808324813581468157818B
:10C2300057FF1AC0C901AA2797FDA095BA2F817090
:10C240009070A070B0705695479537952795822BC2
:10C25000932BA42BB52B84839583A683B7838281EC
:10C260009381019693838283DF0101C0D201CD01C6
:10C27000CDB7DEB7E2E10C94F767A0E2B0E0E3E40B
:10C28000F1E60C94E76769837A838B839C832D8323
:10C290003E834F835887E9E0EE2EF12CEC0EFD1E15
:10C2A000CE010196B7010E9416658E010F5E1F4FE9
:10C2B000CE010596B8010E9416658A8991E089270A
:10C2C0008A8BC701B801AE01475E5F4F0E94F15FE4
:10C2D0000E944164A096E6E00C940368A0E2B0E0FE
:10C2E000E4E7F1E60C94E76769837A838B839C83A8
:10C2F0002D833E834F835887F9E0EF2EF12CEC0E0F
:10C30000FD1ECE010196B7010E9416658E010F5EDB
:10C310001F4FCE010596B8010E941665C701B801EE
:10C32000AE01475E5F4F0E94F15F0E944164A0969C
:10C33000E6E00C940368A0E2B0E0E1EAF1E60C94D8
:10C34000DB6769837A838B839C832D833E834F8352
:10C350005887CE010196BE01675F7F4F0E94166528
:10C36000CE010596BE016F5E7F4F0E9416659985CE
:10C37000923088F089898230C8F0943019F4823084
:10C3800051F404C0843029F4923081F48CE191E0BE
:10C39000C6C0923049F420E09A858A89981321E03A
:10C3A0002A87CE010996BBC0823049F420E09A85E5
:10C3B0008A89981321E02A8BCE014196B0C02D8442
:10C3C0003E844F8458886D887E888F88988CEE24B0
:10C3D000FF248701AA24BB24650140E050E060E00F
:10C3E00070E0E0E0F0E0C10181709070892BE9F02D
:10C3F000E60CF71C081D191D9A01AB012A0D3B1D07
:10C400004C1D5D1D80E090E0A0E0B0E0E614F70474
:10C410000805190520F481E090E0A0E0B0E0BA0141
:10C42000A901480F591F6A1F7B1FAA0CBB1CCC1CFB
:10C43000DD1C97FE08C081E090E0A0E0B0E0A82AF3
:10C44000B92ACA2ADB2A3196E032F10549F0660C96
:10C45000771C881C991C5694479437942794C3CF13
:10C46000FA85EA892B893C898B859C85280F391FA1
:10C470002E5F3F4F17C0CA0181709070892B61F009
:10C4800016950795F794E79480E090E0A0E0B0E877
:10C49000E82AF92A0A2B1B2B76956795579547951D
:10C4A0002F5F3F4F77FDE7CF0CC0440F551F661F2E
:10C4B000771F17FD4160EE0CFF1C001F111F21505C
:10C4C0003040403090E0590790E0690790E47907E8
:10C4D00060F32B8F3C8FDB01CA018F779070A070C7
:10C4E000B07080349105A105B10561F447FD0AC023
:10C4F000E114F1040105110529F0405C5F4F6F4F15
:10C500007F4F40781A8EFE1711F081E08A8F4D8F91
:10C510005E8F6F8F78A383E0898FCE0149960E944A
:10C520004164A096E2E10C94F767A8E1B0E0EBE982
:10C53000F2E60C94E76769837A838B839C832D836F
:10C540003E834F83588789E0E82EF12CEC0EFD1EC8
:10C55000CE010196B7010E9416658E010F5E1F4F36
:10C56000CE010596B8010E9416658985823040F09B
:10C570008989823028F0C701B8010E948E6501C008
:10C580008FEF6896E6E00C940368A8E1B0E0EBEC6E
:10C59000F2E60C94E76769837A838B839C832D830F
:10C5A0003E834F83588789E0E82EF12CEC0EFD1E68
:10C5B000CE010196B7010E9416658E010F5E1F4FD6
:10C5C000CE010596B8010E9416658985823040F03B
:10C5D0008989823028F0C701B8010E948E6501C0A8
:10C5E0008FEF6896E6E00C940368A8E1B0E0EBEF0B
:10C5F000F2E60C94E76769837A838B839C832D83AF
:10C600003E834F83588789E0E82EF12CEC0EFD1E07
:10C61000CE010196B7010E9416658E010F5E1F4F75
:10C62000CE010596B8010E9416658985823040F0DA
:10C630008989823028F0C701B8010E948E6501C047
:10C6400081E06896E6E00C940368ACE0B0E0EBE2D1
:10C65000F3E60C94EB6769837A838B839C83CE012A
:10C660000196BE016B5F7F4F0E9416658D818230FF
:10C6700061F1823050F1843021F48E81882351F1B0
:10C680002EC02F81388537FD20C06E812F313105B6
:10C690001CF06623F9F023C08EE190E0821B930B1F
:10C6A00029853A854B855C8504C056954795379515
:10C6B00027958A95D2F76623B1F05095409530952D
:10C6C00021953F4F4F4F5F4F0EC020E030E040E0DC
:10C6D00050E009C02FEF3FEF4FEF5FE704C020E0CD
:10C6E00030E040E050E8B901CA012C96E2E00C9439
:10C6F0000768A8E0B0E0EFE7F3E60C94E3677B019E
:10C700008C01611571058105910519F482E0898319
:10C7100060C083E089838EE1C82ED12CDC82CB827D
:10C72000ED82FE820F831887C801B7010E94F26371
:10C73000FC013197F7FF3BC0222733272E1B3F0B0D
:10C7400057016801022E04C0D694C794B794A794E9
:10C750000A94D2F740E050E060E070E081E090E0C1
:10C76000A0E0B0E004C0880F991FAA1FBB1F2A9544
:10C77000D2F70197A109B1098E219F21A023B123EE
:10C780000097A105B10521F041E050E060E070E0C4
:10C790004A295B296C297D294D835E836F837887C5
:10C7A0008EE190E08E1B9F0B9C838B8312C0309791
:10C7B00081F00E2E04C0EE0CFF1C001F111F0A9406
:10C7C000D2F7ED82FE820F831887CE1ADF0ADC8251
:10C7D000CB821A82CE0101960E9441642896EAE03B
:10C7E0000C94FF67EF92FF920F931F937B018C01D4
:10C7F00080E0E81680E0F80681E0080780E018078E
:10C8000088F48FEFE816F1040105110531F028F0E6
:10C8100088E090E0A0E0B0E017C080E090E0A0E009
:10C82000B0E012C080E0E81680E0F80680E008077B
:10C8300081E0180728F088E190E0A0E0B0E004C0B3
:10C8400080E190E0A0E0B0E020E230E040E050E0A5
:10C85000281B390B4A0B5B0B04C016950795F79400
:10C86000E7948A95D2F7F701EC5DFE4F8081281B93
:10C87000310941095109C9011F910F91FF90EF90B2
:10C880000895DF92EF92FF920F931F93FC01E480D3
:10C89000F58006811781D1808081823048F480E064
:10C8A00090E0A0E1B0E0E82AF92A0A2B1B2BA5C0F2
:10C8B000843009F49FC0823021F4EE24FF248701E4
:10C8C00005C0E114F1040105110519F4E0E0F0E000
:10C8D00096C0628173819FEF623879070CF05BC06C
:10C8E00022E83FEF261B370B2A3131052CF020E0E0
:10C8F00030E040E050E02AC0B801A701022E04C099
:10C9000076956795579547950A94D2F781E090E020
:10C91000A0E0B0E004C0880F991FAA1FBB1F2A9592
:10C92000D2F70197A109B1098E219F21A023B1233C
:10C930000097A105B10521F081E090E0A0E0B0E012
:10C940009A01AB01282B392B4A2B5B2BDA01C90149
:10C950008F779070A070B07080349105A105B105FB
:10C9600039F427FF09C0205C3F4F4F4F5F4F04C091
:10C97000215C3F4F4F4F5F4FE0E0F0E02030A0E000
:10C980003A07A0E04A07A0E45A0710F0E1E0F0E01F
:10C9900079018A0127C06038710564F5FB01E1580F
:10C9A000FF4FD801C7018F779070A070B0708034AE
:10C9B0009105A105B10539F4E7FE0DC080E490E0D2
:10C9C000A0E0B0E004C08FE390E0A0E0B0E0E80EAB
:10C9D000F91E0A1F1B1F17FF05C016950795F79430
:10C9E000E794319687E016950795F794E7948A9532
:10C9F000D1F705C0EE24FF248701EFEFF0E06E2FA2
:10CA0000679566276795902F9F77D794DD24D794F5
:10CA10008E2F8695492F462B582F5D29B701CA01C5
:10CA20001F910F91FF90EF90DF900895FC01DB01C3
:10CA3000408151812281622F6F7770E0221F22276F
:10CA4000221F9381892F880F822B282F30E0991F76
:10CA50009927991F11969C93119721153105A9F5D6
:10CA6000411551056105710511F482E037C082E876
:10CA70009FEF13969C938E9312979A01AB0167E0F8
:10CA8000220F331F441F551F6A95D1F783E08C9303
:10CA90000DC0220F331F441F551F12968D919C917C
:10CAA0001397019713969C938E931297203080E0F2
:10CAB000380780E0480780E4580758F314962D9310
:10CAC0003D934D935C93179708952F3F310579F46B
:10CAD000411551056105710519F484E08C930895A1
:10CAE00064FF03C081E08C9312C01C9210C02F57CA
:10CAF000304013963C932E93129783E08C9387E0FB
:10CB0000440F551F661F771F8A95D1F770641496DE
:10CB10004D935D936D937C93179708951F93DC015C
:10CB2000FB019C91923008F447C08081823008F468
:10CB300043C0943051F411961C91843099F5818151
:10CB4000682F70E0611B71093FC0843021F0923082
:10CB500031F48230B9F18181882389F12DC0119699
:10CB60001C9111978230F1F081811817D9F4129637
:10CB70002D913C911397828193818217930794F0B2
:10CB800028173907BCF014968D919D910D90BC919A
:10CB9000A02D2481358146815781281739074A07FE
:10CBA0005B0718F4112341F00AC082179307A4070A
:10CBB000B50740F4112319F061E070E005C06FEF94
:10CBC0007FEF02C060E070E0CB011F910895283034
:10CBD00008F027E03327DA01990F311D87FD9160B6
:10CBE00000966105710539F432602E5F3D9330E3A4
:10CBF0002A95E1F708959F3F30F08038710561056F
:10CC000009F03C5F3C5F3D93913008F08068911DD6
:10CC1000DF93CF931F930F93FF92EF92192F987F7B
:10CC20009695E92F96959695E90FFF27E754F947D2
:10CC300099273327EE24FF24A701E70105900894E4
:10CC4000079428F4360FE71EF81E491F511D660F82
:10CC5000771F881F991F0694A1F70590079428F461
:10CC6000E70EF81E491F561FC11D770F881F991F19
:10CC7000661F0694A1F70590079428F4F80E491F43
:10CC8000561FC71FD11D880F991F661F771F069457
:10CC9000A1F70590079420F4490F561FC71FD81F0E
:10CCA000990F661F771F881F0694A9F78491109526
:10CCB000177041F0D695C79557954795F794E79427
:10CCC0001A95C1F7EFE5F6E868941590159135913E
:10CCD0006591959105907FE27395E118F10A430BF8
:10CCE000560BC90BD009C0F7E10CF11E431F561FAC
:10CCF000C91FD01D7EF4703311F48A95E6CFE894F5
:10CD0000015030F0080F0AF40027021708F4202F12
:10CD10002395022F7A3328F079E37D932A95E9F75A
:10CD200010C07D932A9589F6069497956795379557
:10CD300017951794E118F10A430B560BC90BD0094C
:10CD400098F023957E9173957A3308F070E37C9385
:10CD50002013B8F77E9170617D9330F0839571E375
:10CD60007D9370E32A95E1F71124EF90FF900F91E6
:10CD70001F91CF91DF91992787FD90950895DC0150
:10CD8000FB014115510549F04150504029F00590F3
:10CD90000D92002029F0F8CF1C9205900020E9F7B1
:10CDA000E61BF70B3197CF010895FC010590615008
:10CDB00070400110D8F7809590958E0F9F1F0895B1
:10CDC000FC016150704001900110D8F7809590955A
:10CDD0008E0F9F1F08950F931F93CF93DF938C01A6
:10CDE000EB018B8181FF1BC082FF0DC02E813F8133
:10CDF0008C819D812817390764F4E881F9810193BA
:10CE0000F983E88306C0E885F985802F0995892B89
:10CE100031F48E819F8101969F838E8302C00FEF34
:10CE20001FEFC801DF91CF911F910F9108959C01D1
:10CE3000AB018091A9069091AA06B9010E943C5CC1
:10CE40000895FA01AA27283051F1203181F1E894A0
:10CE50006F936E7F6E5F7F4F8F4F9F4FAF4FB1E0ED
:10CE60003ED0B4E03CD0670F781F891F9A1FA11DE8
:10CE7000680F791F8A1F911DA11D6A0F711D811DE9
:10CE8000911DA11D20D009F468943F912AE0269FAE
:10CE900011243019305D3193DEF6CF010895462F0D
:10CEA0004770405D4193B3E00FD0C9F7F6CF462FEE
:10CEB0004F70405D4A3318F0495D31FD4052419357
:10CEC00002D0A9F7EACFB4E0A69597958795779514
:10CED0006795BA95C9F700976105710508959B019B
:10CEE000AC010A2E06945795479537952795BA9524
:10CEF000C9F7620F731F841F951FA01D0895629FBD
:10CF0000D001739FF001829FE00DF11D649FE00D41
:10CF1000F11D929FF00D839FF00D749FF00D659FA2
:10CF2000F00D9927729FB00DE11DF91F639FB00DA1
:10CF3000E11DF91FBD01CF0111240895A1E21A2EB0
:10CF4000AA1BBB1BFD010DC0AA1FBB1FEE1FFF1FAD
:10CF5000A217B307E407F50720F0A21BB30BE40BFD
:10CF6000F50B661F771F881F991F1A9469F7609544
:10CF70007095809590959B01AC01BD01CF010895FE
:10CF800097FB092E05260ED057FD04D0D7DF0AD017
:10CF9000001C38F450954095309521953F4F4F4FE8
:10CFA0005F4F0895F6F790958095709561957F4F46
:10CFB0008F4F9F4F08952F923F924F925F926F92A3
:10CFC0007F928F929F92AF92BF92CF92DF92EF9219
:10CFD000FF920F931F93CF93DF93CDB7DEB7CA1B9A
:10CFE000DB0B0FB6F894DEBF0FBECDBF09942A88C5
:10CFF000398848885F846E847D848C849B84AA846D
:10D00000B984C884DF80EE80FD800C811B81AA81F9
:10D01000B981CE0FD11D0FB6F894DEBF0FBECDBFC4
:08D02000ED010895F894FFCF23
:10D028005AFF322E3600312E3000C30100000002B4
:10D0380000000000AC4C00000000010100000000EE
:10D0480000000000000102020303030304040404B7
:10D05800040404040505050505050505050505057C
:10D06800050505050606060606060606060606065C
:10D078000606060606060606060606060606060648
:10D08800060606060707070707070707070707072C
:10D098000707070707070707070707070707070718
:10D0A8000707070707070707070707070707070708
:10D0B80007070707070707070707070707070707F8
:10D0C80007070707080808080808080808080808DC
:10D0D80008080808080808080808080808080808C8
:10D0E80008080808080808080808080808080808B8
:10D0F80008080808080808080808080808080808A8
:10D108000808080808080808080808080808080897
:10D118000808080808080808080808080808080887
:10D128000808080808080808080808080808080877
:10D138000808080808080808080808080808080867
:04D1480008080808C3
:00000001FF
